Component: ARM Compiler 5.06 update 6 (build 750) Tool: armlink [4d35ed]

==============================================================================

Section Cross References

    startup_stm32f10x_hd.o(STACK) refers (Special) to heapauxi.o(.text) for __use_two_region_memory
    startup_stm32f10x_hd.o(HEAP) refers (Special) to heapauxi.o(.text) for __use_two_region_memory
    startup_stm32f10x_hd.o(RESET) refers (Special) to heapauxi.o(.text) for __use_two_region_memory
    startup_stm32f10x_hd.o(RESET) refers to startup_stm32f10x_hd.o(STACK) for __initial_sp
    startup_stm32f10x_hd.o(RESET) refers to startup_stm32f10x_hd.o(.text) for Reset_Handler
    startup_stm32f10x_hd.o(RESET) refers to uip_kernel_isr_cm.o(CODE) for uipPendSVHandler
    startup_stm32f10x_hd.o(RESET) refers to uip_kernel_time.o(i.uipSystemCounterHandler) for uipSystemCounterHandler
    startup_stm32f10x_hd.o(RESET) refers to chip_uip_interrupt.o(i.WWDG_IRQHandler) for WWDG_IRQHandler
    startup_stm32f10x_hd.o(RESET) refers to chip_uip_interrupt.o(i.PVD_IRQHandler) for PVD_IRQHandler
    startup_stm32f10x_hd.o(RESET) refers to chip_uip_interrupt.o(i.TAMPER_IRQHandler) for TAMPER_IRQHandler
    startup_stm32f10x_hd.o(RESET) refers to chip_uip_interrupt.o(i.RTC_IRQHandler) for RTC_IRQHandler
    startup_stm32f10x_hd.o(RESET) refers to chip_uip_interrupt.o(i.FLASH_IRQHandler) for FLASH_IRQHandler
    startup_stm32f10x_hd.o(RESET) refers to chip_uip_interrupt.o(i.RCC_IRQHandler) for RCC_IRQHandler
    startup_stm32f10x_hd.o(RESET) refers to chip_uip_interrupt.o(i.EXTI0_IRQHandler) for EXTI0_IRQHandler
    startup_stm32f10x_hd.o(RESET) refers to chip_uip_interrupt.o(i.EXTI1_IRQHandler) for EXTI1_IRQHandler
    startup_stm32f10x_hd.o(RESET) refers to chip_uip_interrupt.o(i.EXTI2_IRQHandler) for EXTI2_IRQHandler
    startup_stm32f10x_hd.o(RESET) refers to chip_uip_interrupt.o(i.EXTI3_IRQHandler) for EXTI3_IRQHandler
    startup_stm32f10x_hd.o(RESET) refers to chip_uip_interrupt.o(i.EXTI4_IRQHandler) for EXTI4_IRQHandler
    startup_stm32f10x_hd.o(RESET) refers to chip_uip_interrupt.o(i.DMA1_Channel1_IRQHandler) for DMA1_Channel1_IRQHandler
    startup_stm32f10x_hd.o(RESET) refers to chip_uip_interrupt.o(i.DMA1_Channel2_IRQHandler) for DMA1_Channel2_IRQHandler
    startup_stm32f10x_hd.o(RESET) refers to chip_uip_interrupt.o(i.DMA1_Channel3_IRQHandler) for DMA1_Channel3_IRQHandler
    startup_stm32f10x_hd.o(RESET) refers to chip_uip_interrupt.o(i.DMA1_Channel4_IRQHandler) for DMA1_Channel4_IRQHandler
    startup_stm32f10x_hd.o(RESET) refers to chip_uip_interrupt.o(i.DMA1_Channel5_IRQHandler) for DMA1_Channel5_IRQHandler
    startup_stm32f10x_hd.o(RESET) refers to chip_uip_interrupt.o(i.DMA1_Channel6_IRQHandler) for DMA1_Channel6_IRQHandler
    startup_stm32f10x_hd.o(RESET) refers to chip_uip_interrupt.o(i.DMA1_Channel7_IRQHandler) for DMA1_Channel7_IRQHandler
    startup_stm32f10x_hd.o(RESET) refers to chip_uip_interrupt.o(i.ADC1_2_IRQHandler) for ADC1_2_IRQHandler
    startup_stm32f10x_hd.o(RESET) refers to chip_uip_interrupt.o(i.USB_HP_CAN1_TX_IRQHandler) for USB_HP_CAN1_TX_IRQHandler
    startup_stm32f10x_hd.o(RESET) refers to chip_uip_interrupt.o(i.USB_LP_CAN1_RX0_IRQHandler) for USB_LP_CAN1_RX0_IRQHandler
    startup_stm32f10x_hd.o(RESET) refers to chip_uip_interrupt.o(i.CAN1_RX1_IRQHandler) for CAN1_RX1_IRQHandler
    startup_stm32f10x_hd.o(RESET) refers to chip_uip_interrupt.o(i.CAN1_SCE_IRQHandler) for CAN1_SCE_IRQHandler
    startup_stm32f10x_hd.o(RESET) refers to chip_uip_interrupt.o(i.EXTI9_5_IRQHandler) for EXTI9_5_IRQHandler
    startup_stm32f10x_hd.o(RESET) refers to chip_uip_interrupt.o(i.TIM1_BRK_IRQHandler) for TIM1_BRK_IRQHandler
    startup_stm32f10x_hd.o(RESET) refers to chip_uip_interrupt.o(i.TIM1_UP_IRQHandler) for TIM1_UP_IRQHandler
    startup_stm32f10x_hd.o(RESET) refers to chip_uip_interrupt.o(i.TIM1_TRG_COM_IRQHandler) for TIM1_TRG_COM_IRQHandler
    startup_stm32f10x_hd.o(RESET) refers to chip_uip_interrupt.o(i.TIM1_CC_IRQHandler) for TIM1_CC_IRQHandler
    startup_stm32f10x_hd.o(RESET) refers to chip_uip_interrupt.o(i.TIM2_IRQHandler) for TIM2_IRQHandler
    startup_stm32f10x_hd.o(RESET) refers to chip_uip_interrupt.o(i.TIM3_IRQHandler) for TIM3_IRQHandler
    startup_stm32f10x_hd.o(RESET) refers to chip_uip_interrupt.o(i.TIM4_IRQHandler) for TIM4_IRQHandler
    startup_stm32f10x_hd.o(RESET) refers to chip_uip_interrupt.o(i.I2C1_EV_IRQHandler) for I2C1_EV_IRQHandler
    startup_stm32f10x_hd.o(RESET) refers to chip_uip_interrupt.o(i.I2C1_ER_IRQHandler) for I2C1_ER_IRQHandler
    startup_stm32f10x_hd.o(RESET) refers to chip_uip_interrupt.o(i.I2C2_EV_IRQHandler) for I2C2_EV_IRQHandler
    startup_stm32f10x_hd.o(RESET) refers to chip_uip_interrupt.o(i.I2C2_ER_IRQHandler) for I2C2_ER_IRQHandler
    startup_stm32f10x_hd.o(RESET) refers to chip_uip_interrupt.o(i.SPI1_IRQHandler) for SPI1_IRQHandler
    startup_stm32f10x_hd.o(RESET) refers to chip_uip_interrupt.o(i.SPI2_IRQHandler) for SPI2_IRQHandler
    startup_stm32f10x_hd.o(RESET) refers to chip_uip_interrupt.o(i.USART1_IRQHandler) for USART1_IRQHandler
    startup_stm32f10x_hd.o(RESET) refers to chip_uip_interrupt.o(i.USART2_IRQHandler) for USART2_IRQHandler
    startup_stm32f10x_hd.o(RESET) refers to chip_uip_interrupt.o(i.USART3_IRQHandler) for USART3_IRQHandler
    startup_stm32f10x_hd.o(RESET) refers to chip_uip_interrupt.o(i.EXTI15_10_IRQHandler) for EXTI15_10_IRQHandler
    startup_stm32f10x_hd.o(RESET) refers to chip_uip_interrupt.o(i.RTCAlarm_IRQHandler) for RTCAlarm_IRQHandler
    startup_stm32f10x_hd.o(RESET) refers to chip_uip_interrupt.o(i.USBWakeUp_IRQHandler) for USBWakeUp_IRQHandler
    startup_stm32f10x_hd.o(RESET) refers to chip_uip_interrupt.o(i.TIM8_BRK_IRQHandler) for TIM8_BRK_IRQHandler
    startup_stm32f10x_hd.o(RESET) refers to chip_uip_interrupt.o(i.TIM8_UP_IRQHandler) for TIM8_UP_IRQHandler
    startup_stm32f10x_hd.o(RESET) refers to chip_uip_interrupt.o(i.TIM8_TRG_COM_IRQHandler) for TIM8_TRG_COM_IRQHandler
    startup_stm32f10x_hd.o(RESET) refers to chip_uip_interrupt.o(i.TIM8_CC_IRQHandler) for TIM8_CC_IRQHandler
    startup_stm32f10x_hd.o(RESET) refers to chip_uip_interrupt.o(i.ADC3_IRQHandler) for ADC3_IRQHandler
    startup_stm32f10x_hd.o(RESET) refers to chip_uip_interrupt.o(i.FSMC_IRQHandler) for FSMC_IRQHandler
    startup_stm32f10x_hd.o(RESET) refers to chip_uip_interrupt.o(i.SDIO_IRQHandler) for SDIO_IRQHandler
    startup_stm32f10x_hd.o(RESET) refers to chip_uip_interrupt.o(i.TIM5_IRQHandler) for TIM5_IRQHandler
    startup_stm32f10x_hd.o(RESET) refers to chip_uip_interrupt.o(i.SPI3_IRQHandler) for SPI3_IRQHandler
    startup_stm32f10x_hd.o(RESET) refers to chip_uip_interrupt.o(i.UART4_IRQHandler) for UART4_IRQHandler
    startup_stm32f10x_hd.o(RESET) refers to chip_uip_interrupt.o(i.UART5_IRQHandler) for UART5_IRQHandler
    startup_stm32f10x_hd.o(RESET) refers to chip_uip_interrupt.o(i.TIM6_IRQHandler) for TIM6_IRQHandler
    startup_stm32f10x_hd.o(RESET) refers to chip_uip_interrupt.o(i.TIM7_IRQHandler) for TIM7_IRQHandler
    startup_stm32f10x_hd.o(RESET) refers to chip_uip_interrupt.o(i.DMA2_Channel1_IRQHandler) for DMA2_Channel1_IRQHandler
    startup_stm32f10x_hd.o(RESET) refers to chip_uip_interrupt.o(i.DMA2_Channel2_IRQHandler) for DMA2_Channel2_IRQHandler
    startup_stm32f10x_hd.o(RESET) refers to chip_uip_interrupt.o(i.DMA2_Channel3_IRQHandler) for DMA2_Channel3_IRQHandler
    startup_stm32f10x_hd.o(RESET) refers to chip_uip_interrupt.o(i.DMA2_Channel4_5_IRQHandler) for DMA2_Channel4_5_IRQHandler
    startup_stm32f10x_hd.o(.text) refers (Special) to heapauxi.o(.text) for __use_two_region_memory
    startup_stm32f10x_hd.o(.text) refers to system_stm32f10x_cl.o(i.SystemInit) for SystemInit
    startup_stm32f10x_hd.o(.text) refers to __main.o(!!!main) for __main
    startup_stm32f10x_hd.o(.text) refers to startup_stm32f10x_hd.o(HEAP) for Heap_Mem
    startup_stm32f10x_hd.o(.text) refers to startup_stm32f10x_hd.o(STACK) for Stack_Mem
    system_stm32f10x_cl.o(i.SystemInit) refers to dflt_clz.o(x$fpl$dflt) for __aeabi_i2d
    system_stm32f10x_cl.o(i.SystemInit) refers to dmul.o(x$fpl$dmul) for __aeabi_dmul
    system_stm32f10x_cl.o(i.SystemInit) refers to dfixu.o(x$fpl$dfixu) for __aeabi_d2uiz
    system_stm32f10x_cl.o(i.SystemInit) refers to system_stm32f10x_cl.o(.data) for SystemFrequency_SysClk
    chip_uip_interrupt.o(i.ADC1_2_IRQHandler) refers to uip_kernel_isr_engine.o(i.uipInterruptServiceEngine) for uipInterruptServiceEngine
    chip_uip_interrupt.o(i.ADC1_2_IRQHandler) refers to uip_kernel_common.o(.data) for uipIntTableID
    chip_uip_interrupt.o(i.ADC3_IRQHandler) refers to uip_kernel_isr_engine.o(i.uipInterruptServiceEngine) for uipInterruptServiceEngine
    chip_uip_interrupt.o(i.ADC3_IRQHandler) refers to uip_kernel_common.o(.data) for uipIntTableID
    chip_uip_interrupt.o(i.CAN1_RX1_IRQHandler) refers to uip_kernel_isr_engine.o(i.uipInterruptServiceEngine) for uipInterruptServiceEngine
    chip_uip_interrupt.o(i.CAN1_RX1_IRQHandler) refers to uip_kernel_common.o(.data) for uipIntTableID
    chip_uip_interrupt.o(i.CAN1_SCE_IRQHandler) refers to uip_kernel_isr_engine.o(i.uipInterruptServiceEngine) for uipInterruptServiceEngine
    chip_uip_interrupt.o(i.CAN1_SCE_IRQHandler) refers to uip_kernel_common.o(.data) for uipIntTableID
    chip_uip_interrupt.o(i.Chip_UIP_InterruptInit) refers to chip_uip_interrupt.o(i.Chip_UIP_InterruptRegisterHandler) for Chip_UIP_InterruptRegisterHandler
    chip_uip_interrupt.o(i.Chip_UIP_InterruptInit) refers to app_int_cfg.o(.bss) for UIP_Exc_VectorTable
    chip_uip_interrupt.o(i.Chip_UIP_InterruptInit) refers to chip_uip_interrupt.o(i.Chip_UIP_InterruptNullHandler) for Chip_UIP_InterruptNullHandler
    chip_uip_interrupt.o(i.Chip_UIP_InterruptRegisterHandler) refers to app_int_cfg.o(.bss) for UIP_Exc_VectorTable
    chip_uip_interrupt.o(i.Chip_UIP_InterruptRemoveHandler) refers to chip_uip_interrupt.o(i.Chip_UIP_InterruptRegisterHandler) for Chip_UIP_InterruptRegisterHandler
    chip_uip_interrupt.o(i.Chip_UIP_InterruptRemoveHandler) refers to chip_uip_interrupt.o(i.Chip_UIP_InterruptNullHandler) for Chip_UIP_InterruptNullHandler
    chip_uip_interrupt.o(i.Chip_UIP_Kernel_Tick_ISR_Handler) refers to uip_kernel_time.o(i.uipSystemCounterHandler) for uipSystemCounterHandler
    chip_uip_interrupt.o(i.DMA1_Channel1_IRQHandler) refers to uip_kernel_isr_engine.o(i.uipInterruptServiceEngine) for uipInterruptServiceEngine
    chip_uip_interrupt.o(i.DMA1_Channel1_IRQHandler) refers to uip_kernel_common.o(.data) for uipIntTableID
    chip_uip_interrupt.o(i.DMA1_Channel2_IRQHandler) refers to uip_kernel_isr_engine.o(i.uipInterruptServiceEngine) for uipInterruptServiceEngine
    chip_uip_interrupt.o(i.DMA1_Channel2_IRQHandler) refers to uip_kernel_common.o(.data) for uipIntTableID
    chip_uip_interrupt.o(i.DMA1_Channel3_IRQHandler) refers to uip_kernel_isr_engine.o(i.uipInterruptServiceEngine) for uipInterruptServiceEngine
    chip_uip_interrupt.o(i.DMA1_Channel3_IRQHandler) refers to uip_kernel_common.o(.data) for uipIntTableID
    chip_uip_interrupt.o(i.DMA1_Channel4_IRQHandler) refers to uip_kernel_isr_engine.o(i.uipInterruptServiceEngine) for uipInterruptServiceEngine
    chip_uip_interrupt.o(i.DMA1_Channel4_IRQHandler) refers to uip_kernel_common.o(.data) for uipIntTableID
    chip_uip_interrupt.o(i.DMA1_Channel5_IRQHandler) refers to uip_kernel_isr_engine.o(i.uipInterruptServiceEngine) for uipInterruptServiceEngine
    chip_uip_interrupt.o(i.DMA1_Channel5_IRQHandler) refers to uip_kernel_common.o(.data) for uipIntTableID
    chip_uip_interrupt.o(i.DMA1_Channel6_IRQHandler) refers to uip_kernel_isr_engine.o(i.uipInterruptServiceEngine) for uipInterruptServiceEngine
    chip_uip_interrupt.o(i.DMA1_Channel6_IRQHandler) refers to uip_kernel_common.o(.data) for uipIntTableID
    chip_uip_interrupt.o(i.DMA1_Channel7_IRQHandler) refers to uip_kernel_isr_engine.o(i.uipInterruptServiceEngine) for uipInterruptServiceEngine
    chip_uip_interrupt.o(i.DMA1_Channel7_IRQHandler) refers to uip_kernel_common.o(.data) for uipIntTableID
    chip_uip_interrupt.o(i.DMA2_Channel1_IRQHandler) refers to uip_kernel_isr_engine.o(i.uipInterruptServiceEngine) for uipInterruptServiceEngine
    chip_uip_interrupt.o(i.DMA2_Channel1_IRQHandler) refers to uip_kernel_common.o(.data) for uipIntTableID
    chip_uip_interrupt.o(i.DMA2_Channel2_IRQHandler) refers to uip_kernel_isr_engine.o(i.uipInterruptServiceEngine) for uipInterruptServiceEngine
    chip_uip_interrupt.o(i.DMA2_Channel2_IRQHandler) refers to uip_kernel_common.o(.data) for uipIntTableID
    chip_uip_interrupt.o(i.DMA2_Channel3_IRQHandler) refers to uip_kernel_isr_engine.o(i.uipInterruptServiceEngine) for uipInterruptServiceEngine
    chip_uip_interrupt.o(i.DMA2_Channel3_IRQHandler) refers to uip_kernel_common.o(.data) for uipIntTableID
    chip_uip_interrupt.o(i.DMA2_Channel4_5_IRQHandler) refers to uip_kernel_isr_engine.o(i.uipInterruptServiceEngine) for uipInterruptServiceEngine
    chip_uip_interrupt.o(i.DMA2_Channel4_5_IRQHandler) refers to uip_kernel_common.o(.data) for uipIntTableID
    chip_uip_interrupt.o(i.EXTI0_IRQHandler) refers to uip_kernel_isr_engine.o(i.uipInterruptServiceEngine) for uipInterruptServiceEngine
    chip_uip_interrupt.o(i.EXTI0_IRQHandler) refers to uip_kernel_common.o(.data) for uipIntTableID
    chip_uip_interrupt.o(i.EXTI15_10_IRQHandler) refers to uip_kernel_isr_engine.o(i.uipInterruptServiceEngine) for uipInterruptServiceEngine
    chip_uip_interrupt.o(i.EXTI15_10_IRQHandler) refers to uip_kernel_common.o(.data) for uipIntTableID
    chip_uip_interrupt.o(i.EXTI1_IRQHandler) refers to uip_kernel_isr_engine.o(i.uipInterruptServiceEngine) for uipInterruptServiceEngine
    chip_uip_interrupt.o(i.EXTI1_IRQHandler) refers to uip_kernel_common.o(.data) for uipIntTableID
    chip_uip_interrupt.o(i.EXTI2_IRQHandler) refers to uip_kernel_isr_engine.o(i.uipInterruptServiceEngine) for uipInterruptServiceEngine
    chip_uip_interrupt.o(i.EXTI2_IRQHandler) refers to uip_kernel_common.o(.data) for uipIntTableID
    chip_uip_interrupt.o(i.EXTI3_IRQHandler) refers to uip_kernel_isr_engine.o(i.uipInterruptServiceEngine) for uipInterruptServiceEngine
    chip_uip_interrupt.o(i.EXTI3_IRQHandler) refers to uip_kernel_common.o(.data) for uipIntTableID
    chip_uip_interrupt.o(i.EXTI4_IRQHandler) refers to uip_kernel_isr_engine.o(i.uipInterruptServiceEngine) for uipInterruptServiceEngine
    chip_uip_interrupt.o(i.EXTI4_IRQHandler) refers to uip_kernel_common.o(.data) for uipIntTableID
    chip_uip_interrupt.o(i.EXTI9_5_IRQHandler) refers to uip_kernel_isr_engine.o(i.uipInterruptServiceEngine) for uipInterruptServiceEngine
    chip_uip_interrupt.o(i.EXTI9_5_IRQHandler) refers to uip_kernel_common.o(.data) for uipIntTableID
    chip_uip_interrupt.o(i.FLASH_IRQHandler) refers to uip_kernel_isr_engine.o(i.uipInterruptServiceEngine) for uipInterruptServiceEngine
    chip_uip_interrupt.o(i.FLASH_IRQHandler) refers to uip_kernel_common.o(.data) for uipIntTableID
    chip_uip_interrupt.o(i.FSMC_IRQHandler) refers to uip_kernel_isr_engine.o(i.uipInterruptServiceEngine) for uipInterruptServiceEngine
    chip_uip_interrupt.o(i.FSMC_IRQHandler) refers to uip_kernel_common.o(.data) for uipIntTableID
    chip_uip_interrupt.o(i.I2C1_ER_IRQHandler) refers to uip_kernel_isr_engine.o(i.uipInterruptServiceEngine) for uipInterruptServiceEngine
    chip_uip_interrupt.o(i.I2C1_ER_IRQHandler) refers to uip_kernel_common.o(.data) for uipIntTableID
    chip_uip_interrupt.o(i.I2C1_EV_IRQHandler) refers to uip_kernel_isr_engine.o(i.uipInterruptServiceEngine) for uipInterruptServiceEngine
    chip_uip_interrupt.o(i.I2C1_EV_IRQHandler) refers to uip_kernel_common.o(.data) for uipIntTableID
    chip_uip_interrupt.o(i.I2C2_ER_IRQHandler) refers to uip_kernel_isr_engine.o(i.uipInterruptServiceEngine) for uipInterruptServiceEngine
    chip_uip_interrupt.o(i.I2C2_ER_IRQHandler) refers to uip_kernel_common.o(.data) for uipIntTableID
    chip_uip_interrupt.o(i.I2C2_EV_IRQHandler) refers to uip_kernel_isr_engine.o(i.uipInterruptServiceEngine) for uipInterruptServiceEngine
    chip_uip_interrupt.o(i.I2C2_EV_IRQHandler) refers to uip_kernel_common.o(.data) for uipIntTableID
    chip_uip_interrupt.o(i.InterruptHandler) refers to uip_kernel_common.o(.data) for uipIntTableID
    chip_uip_interrupt.o(i.InterruptHandler) refers to app_int_cfg.o(.bss) for UIP_Exc_VectorTable
    chip_uip_interrupt.o(i.InterruptHandler) refers to app_int_cfg.o(.data) for AppIntNumber
    chip_uip_interrupt.o(i.PVD_IRQHandler) refers to uip_kernel_isr_engine.o(i.uipInterruptServiceEngine) for uipInterruptServiceEngine
    chip_uip_interrupt.o(i.PVD_IRQHandler) refers to uip_kernel_common.o(.data) for uipIntTableID
    chip_uip_interrupt.o(i.RCC_IRQHandler) refers to uip_kernel_isr_engine.o(i.uipInterruptServiceEngine) for uipInterruptServiceEngine
    chip_uip_interrupt.o(i.RCC_IRQHandler) refers to uip_kernel_common.o(.data) for uipIntTableID
    chip_uip_interrupt.o(i.RTCAlarm_IRQHandler) refers to uip_kernel_isr_engine.o(i.uipInterruptServiceEngine) for uipInterruptServiceEngine
    chip_uip_interrupt.o(i.RTCAlarm_IRQHandler) refers to uip_kernel_common.o(.data) for uipIntTableID
    chip_uip_interrupt.o(i.RTC_IRQHandler) refers to uip_kernel_isr_engine.o(i.uipInterruptServiceEngine) for uipInterruptServiceEngine
    chip_uip_interrupt.o(i.RTC_IRQHandler) refers to uip_kernel_common.o(.data) for uipIntTableID
    chip_uip_interrupt.o(i.SDIO_IRQHandler) refers to uip_kernel_isr_engine.o(i.uipInterruptServiceEngine) for uipInterruptServiceEngine
    chip_uip_interrupt.o(i.SDIO_IRQHandler) refers to uip_kernel_common.o(.data) for uipIntTableID
    chip_uip_interrupt.o(i.SPI1_IRQHandler) refers to uip_kernel_isr_engine.o(i.uipInterruptServiceEngine) for uipInterruptServiceEngine
    chip_uip_interrupt.o(i.SPI1_IRQHandler) refers to uip_kernel_common.o(.data) for uipIntTableID
    chip_uip_interrupt.o(i.SPI2_IRQHandler) refers to uip_kernel_isr_engine.o(i.uipInterruptServiceEngine) for uipInterruptServiceEngine
    chip_uip_interrupt.o(i.SPI2_IRQHandler) refers to uip_kernel_common.o(.data) for uipIntTableID
    chip_uip_interrupt.o(i.SPI3_IRQHandler) refers to uip_kernel_isr_engine.o(i.uipInterruptServiceEngine) for uipInterruptServiceEngine
    chip_uip_interrupt.o(i.SPI3_IRQHandler) refers to uip_kernel_common.o(.data) for uipIntTableID
    chip_uip_interrupt.o(i.TAMPER_IRQHandler) refers to uip_kernel_isr_engine.o(i.uipInterruptServiceEngine) for uipInterruptServiceEngine
    chip_uip_interrupt.o(i.TAMPER_IRQHandler) refers to uip_kernel_common.o(.data) for uipIntTableID
    chip_uip_interrupt.o(i.TIM1_BRK_IRQHandler) refers to uip_kernel_isr_engine.o(i.uipInterruptServiceEngine) for uipInterruptServiceEngine
    chip_uip_interrupt.o(i.TIM1_BRK_IRQHandler) refers to uip_kernel_common.o(.data) for uipIntTableID
    chip_uip_interrupt.o(i.TIM1_CC_IRQHandler) refers to uip_kernel_isr_engine.o(i.uipInterruptServiceEngine) for uipInterruptServiceEngine
    chip_uip_interrupt.o(i.TIM1_CC_IRQHandler) refers to uip_kernel_common.o(.data) for uipIntTableID
    chip_uip_interrupt.o(i.TIM1_TRG_COM_IRQHandler) refers to uip_kernel_isr_engine.o(i.uipInterruptServiceEngine) for uipInterruptServiceEngine
    chip_uip_interrupt.o(i.TIM1_TRG_COM_IRQHandler) refers to uip_kernel_common.o(.data) for uipIntTableID
    chip_uip_interrupt.o(i.TIM1_UP_IRQHandler) refers to uip_kernel_isr_engine.o(i.uipInterruptServiceEngine) for uipInterruptServiceEngine
    chip_uip_interrupt.o(i.TIM1_UP_IRQHandler) refers to uip_kernel_common.o(.data) for uipIntTableID
    chip_uip_interrupt.o(i.TIM2_IRQHandler) refers to uip_kernel_isr_engine.o(i.uipInterruptServiceEngine) for uipInterruptServiceEngine
    chip_uip_interrupt.o(i.TIM2_IRQHandler) refers to uip_kernel_common.o(.data) for uipIntTableID
    chip_uip_interrupt.o(i.TIM3_IRQHandler) refers to uip_kernel_isr_engine.o(i.uipInterruptServiceEngine) for uipInterruptServiceEngine
    chip_uip_interrupt.o(i.TIM3_IRQHandler) refers to uip_kernel_common.o(.data) for uipIntTableID
    chip_uip_interrupt.o(i.TIM4_IRQHandler) refers to uip_kernel_isr_engine.o(i.uipInterruptServiceEngine) for uipInterruptServiceEngine
    chip_uip_interrupt.o(i.TIM4_IRQHandler) refers to uip_kernel_common.o(.data) for uipIntTableID
    chip_uip_interrupt.o(i.TIM5_IRQHandler) refers to uip_kernel_isr_engine.o(i.uipInterruptServiceEngine) for uipInterruptServiceEngine
    chip_uip_interrupt.o(i.TIM5_IRQHandler) refers to uip_kernel_common.o(.data) for uipIntTableID
    chip_uip_interrupt.o(i.TIM6_IRQHandler) refers to uip_kernel_isr_engine.o(i.uipInterruptServiceEngine) for uipInterruptServiceEngine
    chip_uip_interrupt.o(i.TIM6_IRQHandler) refers to uip_kernel_common.o(.data) for uipIntTableID
    chip_uip_interrupt.o(i.TIM7_IRQHandler) refers to uip_kernel_isr_engine.o(i.uipInterruptServiceEngine) for uipInterruptServiceEngine
    chip_uip_interrupt.o(i.TIM7_IRQHandler) refers to uip_kernel_common.o(.data) for uipIntTableID
    chip_uip_interrupt.o(i.TIM8_BRK_IRQHandler) refers to uip_kernel_isr_engine.o(i.uipInterruptServiceEngine) for uipInterruptServiceEngine
    chip_uip_interrupt.o(i.TIM8_BRK_IRQHandler) refers to uip_kernel_common.o(.data) for uipIntTableID
    chip_uip_interrupt.o(i.TIM8_CC_IRQHandler) refers to uip_kernel_isr_engine.o(i.uipInterruptServiceEngine) for uipInterruptServiceEngine
    chip_uip_interrupt.o(i.TIM8_CC_IRQHandler) refers to uip_kernel_common.o(.data) for uipIntTableID
    chip_uip_interrupt.o(i.TIM8_TRG_COM_IRQHandler) refers to uip_kernel_isr_engine.o(i.uipInterruptServiceEngine) for uipInterruptServiceEngine
    chip_uip_interrupt.o(i.TIM8_TRG_COM_IRQHandler) refers to uip_kernel_common.o(.data) for uipIntTableID
    chip_uip_interrupt.o(i.TIM8_UP_IRQHandler) refers to uip_kernel_isr_engine.o(i.uipInterruptServiceEngine) for uipInterruptServiceEngine
    chip_uip_interrupt.o(i.TIM8_UP_IRQHandler) refers to uip_kernel_common.o(.data) for uipIntTableID
    chip_uip_interrupt.o(i.UART4_IRQHandler) refers to uip_kernel_isr_engine.o(i.uipInterruptServiceEngine) for uipInterruptServiceEngine
    chip_uip_interrupt.o(i.UART4_IRQHandler) refers to uip_kernel_common.o(.data) for uipIntTableID
    chip_uip_interrupt.o(i.UART5_IRQHandler) refers to uip_kernel_isr_engine.o(i.uipInterruptServiceEngine) for uipInterruptServiceEngine
    chip_uip_interrupt.o(i.UART5_IRQHandler) refers to uip_kernel_common.o(.data) for uipIntTableID
    chip_uip_interrupt.o(i.USART1_IRQHandler) refers to uip_kernel_isr_engine.o(i.uipInterruptServiceEngine) for uipInterruptServiceEngine
    chip_uip_interrupt.o(i.USART1_IRQHandler) refers to uip_kernel_common.o(.data) for uipIntTableID
    chip_uip_interrupt.o(i.USART2_IRQHandler) refers to uip_kernel_isr_engine.o(i.uipInterruptServiceEngine) for uipInterruptServiceEngine
    chip_uip_interrupt.o(i.USART2_IRQHandler) refers to uip_kernel_common.o(.data) for uipIntTableID
    chip_uip_interrupt.o(i.USART3_IRQHandler) refers to uip_kernel_isr_engine.o(i.uipInterruptServiceEngine) for uipInterruptServiceEngine
    chip_uip_interrupt.o(i.USART3_IRQHandler) refers to uip_kernel_common.o(.data) for uipIntTableID
    chip_uip_interrupt.o(i.USBWakeUp_IRQHandler) refers to uip_kernel_isr_engine.o(i.uipInterruptServiceEngine) for uipInterruptServiceEngine
    chip_uip_interrupt.o(i.USBWakeUp_IRQHandler) refers to uip_kernel_common.o(.data) for uipIntTableID
    chip_uip_interrupt.o(i.USB_HP_CAN1_TX_IRQHandler) refers to uip_kernel_isr_engine.o(i.uipInterruptServiceEngine) for uipInterruptServiceEngine
    chip_uip_interrupt.o(i.USB_HP_CAN1_TX_IRQHandler) refers to uip_kernel_common.o(.data) for uipIntTableID
    chip_uip_interrupt.o(i.USB_LP_CAN1_RX0_IRQHandler) refers to uip_kernel_isr_engine.o(i.uipInterruptServiceEngine) for uipInterruptServiceEngine
    chip_uip_interrupt.o(i.USB_LP_CAN1_RX0_IRQHandler) refers to uip_kernel_common.o(.data) for uipIntTableID
    chip_uip_interrupt.o(i.WWDG_IRQHandler) refers to uip_kernel_isr_engine.o(i.uipInterruptServiceEngine) for uipInterruptServiceEngine
    chip_uip_interrupt.o(i.WWDG_IRQHandler) refers to uip_kernel_common.o(.data) for uipIntTableID
    chip_uip_interrupt.o(i.uipInterruptHandlingCallback) refers to chip_uip_interrupt.o(i.InterruptHandler) for InterruptHandler
    chip_uip_interrupt.o(i.uipInterruptHandlingCallback) refers to uip_kernel_common.o(.data) for uipLowPowerMode
    hardware_init.o(i.Hardware_Init) refers to stm32f1xx_hal_cortex.o(i.HAL_NVIC_SetPriorityGrouping) for HAL_NVIC_SetPriorityGrouping
    hardware_init.o(i.Hardware_Init) refers to chip_uip_interrupt.o(i.Chip_UIP_InterruptInit) for Chip_UIP_InterruptInit
    hardware_init.o(i.Kernel_System_Tick_Init) refers to stm32f1xx_hal_rcc.o(i.HAL_RCC_GetHCLKFreq) for HAL_RCC_GetHCLKFreq
    hardware_init.o(i.Kernel_System_Tick_Init) refers to stm32f1xx_hal_cortex.o(i.HAL_SYSTICK_Config) for HAL_SYSTICK_Config
    hardware_init.o(i.Kernel_System_Tick_Init) refers to stm32f1xx_hal_cortex.o(i.HAL_SYSTICK_CLKSourceConfig) for HAL_SYSTICK_CLKSourceConfig
    hardware_init.o(i.Kernel_System_Tick_Init) refers to stm32f1xx_hal_cortex.o(i.HAL_NVIC_SetPriority) for HAL_NVIC_SetPriority
    hardware_init.o(i.STM32_OSC_Init) refers to stm32f1xx_hal_rcc.o(i.HAL_RCC_OscConfig) for HAL_RCC_OscConfig
    hardware_init.o(i.STM32_OSC_Init) refers to stm32f1xx_hal_rcc.o(i.HAL_RCC_ClockConfig) for HAL_RCC_ClockConfig
    system_stm32f1xx.o(i.SystemCoreClockUpdate) refers to system_stm32f1xx.o(.data) for SystemCoreClock
    system_stm32f1xx.o(i.SystemCoreClockUpdate) refers to system_stm32f1xx.o(.constdata) for AHBPrescTable
    app_cfg.o(.data) refers to app_cfg.o(.bss) for AppMsgBuf
    app_cfg.o(.data) refers to demo.o(i.TASK_0) for TASK_0
    app_cfg.o(.data) refers to demo.o(i.TASK_1) for TASK_1
    app_cfg.o(.data) refers to demo.o(i.TASK_2) for TASK_2
    app_cfg.o(.data) refers to demo.o(i.TASK_3) for TASK_3
    app_cfg.o(.data) refers to demo.o(i.TASK_4) for TASK_4
    app_cfg.o(.data) refers to demo.o(i.AppIdleTask) for AppIdleTask
    demo.o(i.TASK_0) refers to uip_kernel_event.o(i.UIP_WaitEvent) for UIP_WaitEvent
    demo.o(i.TASK_0) refers to uip_kernel_event.o(i.UIP_ClearEvent) for UIP_ClearEvent
    demo.o(i.TASK_1) refers to uip_kernel_event.o(i.UIP_WaitEvent) for UIP_WaitEvent
    demo.o(i.TASK_1) refers to uip_kernel_event.o(i.UIP_ClearEvent) for UIP_ClearEvent
    demo.o(i.TASK_2) refers to uip_kernel_event.o(i.UIP_WaitEvent) for UIP_WaitEvent
    demo.o(i.TASK_2) refers to uip_kernel_event.o(i.UIP_ClearEvent) for UIP_ClearEvent
    demo.o(i.TASK_2) refers to uip_kernel_resource.o(i.UIP_GetResource) for UIP_GetResource
    demo.o(i.TASK_2) refers to uip_kernel_resource.o(i.UIP_ReleaseResource) for UIP_ReleaseResource
    demo.o(i.TASK_3) refers to uip_kernel_resource.o(i.UIP_GetResource) for UIP_GetResource
    demo.o(i.TASK_3) refers to uip_kernel_event.o(i.UIP_SetEvent) for UIP_SetEvent
    demo.o(i.TASK_3) refers to uip_kernel_resource.o(i.UIP_ReleaseResource) for UIP_ReleaseResource
    demo.o(i.TASK_4) refers to uip_kernel_message.o(i.UIP_ReceiveMessage) for UIP_ReceiveMessage
    demo.o(i.TASK_4) refers to uip_kernel_task.o(i.UIP_TerminateTask) for UIP_TerminateTask
    demo.o(i.main) refers to hardware_init.o(i.Hardware_Init) for Hardware_Init
    demo.o(i.main) refers to uip_kernel_common.o(i.StartOS) for StartOS
    demo.o(i.main) refers to uip_kernel_common.o(.data) for uipIdleTaskID
    demo.o(i.uipAppInitialize) refers to uip_kernel_common.o(i.uipTaskInitialize) for uipTaskInitialize
    demo.o(i.uipAppInitialize) refers to uip_kernel_common.o(i.uipAlarmInitialize) for uipAlarmInitialize
    demo.o(i.uipAppInitialize) refers to uip_kernel_common.o(i.uipResInitialize) for uipResInitialize
    demo.o(i.uipAppInitialize) refers to uip_kernel_common.o(i.uipMsgInitialize) for uipMsgInitialize
    demo.o(i.uipAppInitialize) refers to hardware_init.o(i.Kernel_System_Tick_Init) for Kernel_System_Tick_Init
    demo.o(i.uipAppInitialize) refers to app_cfg.o(.data) for AppTaskNumber
    uip_kernel_common.o(i.StartOS) refers to uip_kernel_isr_cm.o(CODE) for uipDisableAllInterrupts
    uip_kernel_common.o(i.StartOS) refers to uip_kernel_common.o(i.uipKernelInitialize) for uipKernelInitialize
    uip_kernel_common.o(i.StartOS) refers to demo.o(i.uipAppInitialize) for uipAppInitialize
    uip_kernel_common.o(i.StartOS) refers to uip_kernel_scheduler.o(.data) for uipSystemMode
    uip_kernel_common.o(i.uipAlarmInfoInit) refers to uip_kernel_common.o(.data) for uipAlarmNumber
    uip_kernel_common.o(i.uipAlarmInitialize) refers to uip_kernel_common.o(.data) for uipAlarmNumber
    uip_kernel_common.o(i.uipKernelInitialize) refers to uip_kernel_common.o(.data) for uipTCBArray
    uip_kernel_common.o(i.uipKernelInitialize) refers to uip_kernel_common.o(.bss) for uipPriorityToTaskID
    uip_kernel_common.o(i.uipKernelInitialize) refers to uip_kernel_scheduler.o(.bss) for uipPrioGrpArray
    uip_kernel_common.o(i.uipKernelInitialize) refers to uip_kernel_scheduler.o(.data) for uipSchedulerLock
    uip_kernel_common.o(i.uipMsgInfoInit) refers to uip_kernel_common.o(.data) for uipMsgNumber
    uip_kernel_common.o(i.uipMsgInitialize) refers to uip_kernel_common.o(.data) for uipMsgNumber
    uip_kernel_common.o(i.uipResInfoInit) refers to uip_kernel_common.o(.data) for uipResNumber
    uip_kernel_common.o(i.uipResInitialize) refers to uip_kernel_common.o(.data) for uipResNumber
    uip_kernel_common.o(i.uipTaskInfoInit) refers to uip_kernel_common.o(.data) for uipTaskNumber
    uip_kernel_common.o(i.uipTaskInitialize) refers to uip_kernel_common.o(i.uipTaskStackInit) for uipTaskStackInit
    uip_kernel_common.o(i.uipTaskInitialize) refers to uip_kernel_common.o(.data) for uipTaskNumber
    uip_kernel_common.o(i.uipTaskInitialize) refers to uip_kernel_common.o(.bss) for uipInitTaskStackPtr
    uip_kernel_common.o(i.uipTaskInitialize) refers to uip_kernel_scheduler.o(.data) for uipPrioGroup
    uip_kernel_common.o(i.uipTaskInitialize) refers to uip_kernel_scheduler.o(.bss) for uipPrioGrpArray
    uip_kernel_event.o(i.UIP_ClearEvent) refers to uip_kernel_isr_cm.o(CODE) for uipDisableAllInterrupts
    uip_kernel_event.o(i.UIP_ClearEvent) refers to uip_kernel_scheduler.o(.data) for uipNestedInterrupts
    uip_kernel_event.o(i.UIP_GetEvent) refers to uip_kernel_isr_cm.o(CODE) for uipDisableAllInterrupts
    uip_kernel_event.o(i.UIP_GetEvent) refers to uip_kernel_scheduler.o(.data) for uipSchedulerLock
    uip_kernel_event.o(i.UIP_GetEvent) refers to uip_kernel_common.o(.data) for uipTCBArray
    uip_kernel_event.o(i.UIP_SetEvent) refers to uip_kernel_isr_cm.o(CODE) for uipDisableAllInterrupts
    uip_kernel_event.o(i.UIP_SetEvent) refers to uip_kernel_scheduler.o(i.uipGetNextPriority) for uipGetNextPriority
    uip_kernel_event.o(i.UIP_SetEvent) refers to uip_kernel_common.o(.data) for uipTCBArray
    uip_kernel_event.o(i.UIP_SetEvent) refers to uip_kernel_scheduler.o(.data) for uipPrioGroup
    uip_kernel_event.o(i.UIP_SetEvent) refers to uip_kernel_scheduler.o(.bss) for uipPrioGrpArray
    uip_kernel_event.o(i.UIP_SetEvent) refers to uip_kernel_common.o(.bss) for uipPriorityToTaskID
    uip_kernel_event.o(i.UIP_WaitEvent) refers to uip_kernel_isr_cm.o(CODE) for uipDisableAllInterrupts
    uip_kernel_event.o(i.UIP_WaitEvent) refers to uip_kernel_scheduler.o(i.uipClearPrioGrpAndArrayBit) for uipClearPrioGrpAndArrayBit
    uip_kernel_event.o(i.UIP_WaitEvent) refers to uip_kernel_scheduler.o(i.uipGetNextTask) for uipGetNextTask
    uip_kernel_event.o(i.UIP_WaitEvent) refers to uip_kernel_scheduler.o(.data) for uipNestedInterrupts
    uip_kernel_isr_cm.o(CODE) refers to uip_kernel_scheduler.o(i.uipPreContexSwitch) for uipPreContexSwitch
    uip_kernel_isr_cm.o(CODE) refers to uip_kernel_scheduler.o(.data) for uipCurrentTaskTCBPtr
    uip_kernel_isr_engine.o(i.uipInterruptServiceEngine) refers to uip_kernel_isr_cm.o(CODE) for uipDisableAllInterrupts
    uip_kernel_isr_engine.o(i.uipInterruptServiceEngine) refers to chip_uip_interrupt.o(i.uipInterruptHandlingCallback) for uipInterruptHandlingCallback
    uip_kernel_isr_engine.o(i.uipInterruptServiceEngine) refers to uip_kernel_scheduler.o(i.uipGetNextTask) for uipGetNextTask
    uip_kernel_isr_engine.o(i.uipInterruptServiceEngine) refers to uip_kernel_scheduler.o(.data) for uipSystemMode
    uip_kernel_isr_engine.o(i.uipInterruptServiceEngine) refers to uip_kernel_common.o(.data) for uipLowPowerMode
    uip_kernel_message.o(i.UIP_GetMessageStatus) refers to uip_kernel_common.o(.data) for uipMsgNumber
    uip_kernel_message.o(i.UIP_ReadFlag) refers to uip_kernel_common.o(.data) for uipMCBArray
    uip_kernel_message.o(i.UIP_ReceiveMessage) refers to uip_kernel_isr_cm.o(CODE) for uipDisableAllInterrupts
    uip_kernel_message.o(i.UIP_ReceiveMessage) refers to uip_kernel_common.o(.data) for uipMsgNumber
    uip_kernel_message.o(i.UIP_ResetFlag) refers to uip_kernel_isr_cm.o(CODE) for uipDisableAllInterrupts
    uip_kernel_message.o(i.UIP_ResetFlag) refers to uip_kernel_common.o(.data) for uipMCBArray
    uip_kernel_message.o(i.UIP_SendMessage) refers to uip_kernel_isr_cm.o(CODE) for uipDisableAllInterrupts
    uip_kernel_message.o(i.UIP_SendMessage) refers to uip_kernel_event.o(i.UIP_SetEvent) for UIP_SetEvent
    uip_kernel_message.o(i.UIP_SendMessage) refers to uip_kernel_task.o(i.UIP_ActivateTask) for UIP_ActivateTask
    uip_kernel_message.o(i.UIP_SendMessage) refers to uip_kernel_common.o(.data) for uipMsgNumber
    uip_kernel_message.o(i.UIP_StartCOM) refers to demo.o(i.uipCOMInit) for uipCOMInit
    uip_kernel_message.o(i.UIP_StopCOM) refers to uip_kernel_common.o(.data) for uipMCBArray
    uip_kernel_resource.o(i.UIP_GetResource) refers to uip_kernel_isr_cm.o(CODE) for uipDisableAllInterrupts
    uip_kernel_resource.o(i.UIP_GetResource) refers to uip_kernel_scheduler.o(.data) for uipNestedInterrupts
    uip_kernel_resource.o(i.UIP_GetResource) refers to uip_kernel_common.o(.data) for uipResNumber
    uip_kernel_resource.o(i.UIP_GetResource) refers to uip_kernel_scheduler.o(.bss) for uipPrioGrpArray
    uip_kernel_resource.o(i.UIP_GetResource) refers to uip_kernel_common.o(.bss) for uipPriorityToTaskID
    uip_kernel_resource.o(i.UIP_ReleaseResource) refers to uip_kernel_isr_cm.o(CODE) for uipDisableAllInterrupts
    uip_kernel_resource.o(i.UIP_ReleaseResource) refers to uip_kernel_scheduler.o(i.uipGetNextPriority) for uipGetNextPriority
    uip_kernel_resource.o(i.UIP_ReleaseResource) refers to uip_kernel_common.o(.data) for uipResNumber
    uip_kernel_resource.o(i.UIP_ReleaseResource) refers to uip_kernel_scheduler.o(.data) for uipCurrentTaskTCBPtr
    uip_kernel_resource.o(i.UIP_ReleaseResource) refers to uip_kernel_scheduler.o(.bss) for uipPrioGrpArray
    uip_kernel_resource.o(i.UIP_ReleaseResource) refers to uip_kernel_common.o(.bss) for uipPriorityToTaskID
    uip_kernel_scheduler.o(i.uipClearPrioGrpAndArrayBit) refers to uip_kernel_scheduler.o(.bss) for uipPrioGrpArray
    uip_kernel_scheduler.o(i.uipClearPrioGrpAndArrayBit) refers to uip_kernel_scheduler.o(.data) for uipPrioGroup
    uip_kernel_scheduler.o(i.uipGetNextPriority) refers to uip_kernel_scheduler.o(.data) for uipPrioGroup
    uip_kernel_scheduler.o(i.uipGetNextPriority) refers to uip_kernel_scheduler.o(.bss) for uipPrioGrpArray
    uip_kernel_scheduler.o(i.uipGetNextTask) refers to uip_kernel_scheduler.o(.data) for uipPrioGroup
    uip_kernel_scheduler.o(i.uipGetNextTask) refers to uip_kernel_scheduler.o(.bss) for uipPrioGrpArray
    uip_kernel_scheduler.o(i.uipGetNextTask) refers to uip_kernel_common.o(.bss) for uipPriorityToTaskID
    uip_kernel_scheduler.o(i.uipGetNextTask) refers to uip_kernel_common.o(.data) for uipTCBArray
    uip_kernel_scheduler.o(i.uipPreContexSwitch) refers to uip_kernel_scheduler.o(i.uipResetPrioGrpAndArrayBit) for uipResetPrioGrpAndArrayBit
    uip_kernel_scheduler.o(i.uipPreContexSwitch) refers to uip_kernel_scheduler.o(.data) for uipNextRunningTaskTCBPtr
    uip_kernel_scheduler.o(i.uipResetPrioGrpAndArrayBit) refers to uip_kernel_scheduler.o(.data) for uipCurrentTaskTCBPtr
    uip_kernel_scheduler.o(i.uipResetPrioGrpAndArrayBit) refers to uip_kernel_scheduler.o(.bss) for uipPrioGrpArray
    uip_kernel_task.o(i.UIP_ActivateTask) refers to uip_kernel_isr_cm.o(CODE) for uipDisableAllInterrupts
    uip_kernel_task.o(i.UIP_ActivateTask) refers to uip_kernel_common.o(.data) for uipTCBArray
    uip_kernel_task.o(i.UIP_ActivateTask) refers to uip_kernel_scheduler.o(.data) for uipPrioGroup
    uip_kernel_task.o(i.UIP_ActivateTask) refers to uip_kernel_scheduler.o(.bss) for uipPrioGrpArray
    uip_kernel_task.o(i.UIP_ChainTask) refers to uip_kernel_isr_cm.o(CODE) for uipDisableAllInterrupts
    uip_kernel_task.o(i.UIP_ChainTask) refers to uip_kernel_scheduler.o(i.uipClearPrioGrpAndArrayBit) for uipClearPrioGrpAndArrayBit
    uip_kernel_task.o(i.UIP_ChainTask) refers to uip_kernel_scheduler.o(i.uipGetNextTask) for uipGetNextTask
    uip_kernel_task.o(i.UIP_ChainTask) refers to uip_kernel_common.o(i.uipTaskStackInit) for uipTaskStackInit
    uip_kernel_task.o(i.UIP_ChainTask) refers to uip_kernel_scheduler.o(.data) for uipNestedInterrupts
    uip_kernel_task.o(i.UIP_ChainTask) refers to uip_kernel_common.o(.data) for uipTCBArray
    uip_kernel_task.o(i.UIP_ChainTask) refers to uip_kernel_scheduler.o(.bss) for uipPrioGrpArray
    uip_kernel_task.o(i.UIP_ChainTask) refers to uip_kernel_common.o(.bss) for uipInitTaskStackPtr
    uip_kernel_task.o(i.UIP_GetTaskID) refers to uip_kernel_scheduler.o(.data) for uipCurrentTaskTCBPtr
    uip_kernel_task.o(i.UIP_GetTaskState) refers to uip_kernel_isr_cm.o(CODE) for uipDisableAllInterrupts
    uip_kernel_task.o(i.UIP_GetTaskState) refers to uip_kernel_common.o(.data) for uipTCBArray
    uip_kernel_task.o(i.UIP_Schedule) refers to uip_kernel_isr_cm.o(CODE) for uipDisableAllInterrupts
    uip_kernel_task.o(i.UIP_Schedule) refers to uip_kernel_scheduler.o(i.uipGetNextPriority) for uipGetNextPriority
    uip_kernel_task.o(i.UIP_Schedule) refers to uip_kernel_scheduler.o(.data) for uipNestedInterrupts
    uip_kernel_task.o(i.UIP_Schedule) refers to uip_kernel_scheduler.o(.bss) for uipPrioGrpArray
    uip_kernel_task.o(i.UIP_Schedule) refers to uip_kernel_common.o(.bss) for uipPriorityToTaskID
    uip_kernel_task.o(i.UIP_Schedule) refers to uip_kernel_common.o(.data) for uipTCBArray
    uip_kernel_task.o(i.UIP_TerminateTask) refers to uip_kernel_isr_cm.o(CODE) for uipDisableAllInterrupts
    uip_kernel_task.o(i.UIP_TerminateTask) refers to uip_kernel_common.o(i.uipTaskStackInit) for uipTaskStackInit
    uip_kernel_task.o(i.UIP_TerminateTask) refers to uip_kernel_scheduler.o(i.uipClearPrioGrpAndArrayBit) for uipClearPrioGrpAndArrayBit
    uip_kernel_task.o(i.UIP_TerminateTask) refers to uip_kernel_scheduler.o(i.uipGetNextTask) for uipGetNextTask
    uip_kernel_task.o(i.UIP_TerminateTask) refers to uip_kernel_scheduler.o(.data) for uipNestedInterrupts
    uip_kernel_task.o(i.UIP_TerminateTask) refers to uip_kernel_common.o(.bss) for uipInitTaskStackPtr
    uip_kernel_task.o(i.UIP_TerminateTask) refers to uip_kernel_scheduler.o(.bss) for uipPrioGrpArray
    uip_kernel_time.o(i.UIP_CancelAlarm) refers to uip_kernel_isr_cm.o(CODE) for uipDisableAllInterrupts
    uip_kernel_time.o(i.UIP_CancelAlarm) refers to uip_kernel_common.o(.data) for uipAlarmNumber
    uip_kernel_time.o(i.UIP_GetAlarm) refers to uip_kernel_isr_cm.o(CODE) for uipDisableAllInterrupts
    uip_kernel_time.o(i.UIP_GetAlarm) refers to uip_kernel_common.o(.data) for uipAlarmNumber
    uip_kernel_time.o(i.UIP_GetAlarmBase) refers to uip_kernel_common.o(.data) for uipAlarmNumber
    uip_kernel_time.o(i.UIP_SetAbsAlarm) refers to uip_kernel_isr_cm.o(CODE) for uipDisableAllInterrupts
    uip_kernel_time.o(i.UIP_SetAbsAlarm) refers to uip_kernel_common.o(.data) for uipAlarmNumber
    uip_kernel_time.o(i.UIP_SetRelAlarm) refers to uip_kernel_isr_cm.o(CODE) for uipDisableAllInterrupts
    uip_kernel_time.o(i.UIP_SetRelAlarm) refers to uip_kernel_common.o(.data) for uipAlarmNumber
    uip_kernel_time.o(i.uipAlarmHandler) refers to uip_kernel_event.o(i.UIP_SetEvent) for UIP_SetEvent
    uip_kernel_time.o(i.uipAlarmHandler) refers to uip_kernel_task.o(i.UIP_ActivateTask) for UIP_ActivateTask
    uip_kernel_time.o(i.uipAlarmHandler) refers to uip_kernel_common.o(.data) for uipACBArray
    uip_kernel_time.o(i.uipGeneralCounterHandler) refers to uip_kernel_time.o(i.uipAlarmHandler) for uipAlarmHandler
    uip_kernel_time.o(i.uipGeneralCounterHandler) refers to uip_kernel_common.o(.data) for uipACBArray
    uip_kernel_time.o(i.uipGetCtrCurrentValue) refers to uip_kernel_isr_cm.o(CODE) for uipDisableAllInterrupts
    uip_kernel_time.o(i.uipGetCtrCurrentValue) refers to uip_kernel_common.o(.data) for uipAlarmNumber
    uip_kernel_time.o(i.uipSystemCounterHandler) refers to uip_kernel_time.o(i.uipAlarmHandler) for uipAlarmHandler
    uip_kernel_time.o(i.uipSystemCounterHandler) refers to uip_kernel_common.o(.bss) for uipSystemCounter
    uip_kernel_time.o(i.uipSystemCounterHandler) refers to uip_kernel_common.o(.data) for uipACBArray
    stm32f1xx_hal.o(i.HAL_DeInit) refers to stm32f1xx_hal.o(i.HAL_MspDeInit) for HAL_MspDeInit
    stm32f1xx_hal.o(i.HAL_Delay) refers to stm32f1xx_hal.o(i.HAL_GetTick) for HAL_GetTick
    stm32f1xx_hal.o(i.HAL_GetTick) refers to stm32f1xx_hal.o(.data) for uwTick
    stm32f1xx_hal.o(i.HAL_IncTick) refers to stm32f1xx_hal.o(.data) for uwTick
    stm32f1xx_hal.o(i.HAL_Init) refers to stm32f1xx_hal_cortex.o(i.HAL_NVIC_SetPriorityGrouping) for HAL_NVIC_SetPriorityGrouping
    stm32f1xx_hal.o(i.HAL_Init) refers to stm32f1xx_hal.o(i.HAL_InitTick) for HAL_InitTick
    stm32f1xx_hal.o(i.HAL_Init) refers to stm32f1xx_hal_msp.o(i.HAL_MspInit) for HAL_MspInit
    stm32f1xx_hal.o(i.HAL_InitTick) refers to stm32f1xx_hal_rcc.o(i.HAL_RCC_GetHCLKFreq) for HAL_RCC_GetHCLKFreq
    stm32f1xx_hal.o(i.HAL_InitTick) refers to stm32f1xx_hal_cortex.o(i.HAL_SYSTICK_Config) for HAL_SYSTICK_Config
    stm32f1xx_hal.o(i.HAL_InitTick) refers to stm32f1xx_hal_cortex.o(i.HAL_NVIC_SetPriority) for HAL_NVIC_SetPriority
    stm32f1xx_hal_cortex.o(i.HAL_NVIC_GetPriorityGrouping) refers to stm32f1xx_hal_cortex.o(i.NVIC_GetPriorityGrouping) for NVIC_GetPriorityGrouping
    stm32f1xx_hal_cortex.o(i.HAL_NVIC_SetPriority) refers to stm32f1xx_hal_cortex.o(i.NVIC_GetPriorityGrouping) for NVIC_GetPriorityGrouping
    stm32f1xx_hal_cortex.o(i.HAL_NVIC_SetPriority) refers to stm32f1xx_hal_cortex.o(i.NVIC_SetPriority) for NVIC_SetPriority
    stm32f1xx_hal_cortex.o(i.HAL_SYSTICK_Config) refers to stm32f1xx_hal_cortex.o(i.NVIC_SetPriority) for NVIC_SetPriority
    stm32f1xx_hal_cortex.o(i.HAL_SYSTICK_IRQHandler) refers to stm32f1xx_hal_cortex.o(i.HAL_SYSTICK_Callback) for HAL_SYSTICK_Callback
    stm32f1xx_hal_dma.o(i.HAL_DMA_Abort) refers to stm32f1xx_hal.o(i.HAL_GetTick) for HAL_GetTick
    stm32f1xx_hal_dma.o(i.HAL_DMA_PollForTransfer) refers to stm32f1xx_hal.o(i.HAL_GetTick) for HAL_GetTick
    stm32f1xx_hal_dma.o(i.HAL_DMA_Start) refers to stm32f1xx_hal_dma.o(i.DMA_SetConfig) for DMA_SetConfig
    stm32f1xx_hal_dma.o(i.HAL_DMA_Start_IT) refers to stm32f1xx_hal_dma.o(i.DMA_SetConfig) for DMA_SetConfig
    stm32f1xx_hal_flash.o(i.FLASH_Program_HalfWord) refers to stm32f1xx_hal_flash.o(.bss) for pFlash
    stm32f1xx_hal_flash.o(i.FLASH_SetErrorCode) refers to stm32f1xx_hal_flash.o(.bss) for pFlash
    stm32f1xx_hal_flash.o(i.FLASH_WaitForLastOperation) refers to stm32f1xx_hal.o(i.HAL_GetTick) for HAL_GetTick
    stm32f1xx_hal_flash.o(i.FLASH_WaitForLastOperation) refers to stm32f1xx_hal_flash.o(i.FLASH_SetErrorCode) for FLASH_SetErrorCode
    stm32f1xx_hal_flash.o(i.HAL_FLASH_GetError) refers to stm32f1xx_hal_flash.o(.bss) for pFlash
    stm32f1xx_hal_flash.o(i.HAL_FLASH_IRQHandler) refers to stm32f1xx_hal_flash.o(i.FLASH_SetErrorCode) for FLASH_SetErrorCode
    stm32f1xx_hal_flash.o(i.HAL_FLASH_IRQHandler) refers to stm32f1xx_hal_flash.o(i.HAL_FLASH_OperationErrorCallback) for HAL_FLASH_OperationErrorCallback
    stm32f1xx_hal_flash.o(i.HAL_FLASH_IRQHandler) refers to stm32f1xx_hal_flash.o(i.HAL_FLASH_EndOfOperationCallback) for HAL_FLASH_EndOfOperationCallback
    stm32f1xx_hal_flash.o(i.HAL_FLASH_IRQHandler) refers to stm32f1xx_hal_flash_ex.o(i.FLASH_PageErase) for FLASH_PageErase
    stm32f1xx_hal_flash.o(i.HAL_FLASH_IRQHandler) refers to stm32f1xx_hal_flash.o(i.FLASH_Program_HalfWord) for FLASH_Program_HalfWord
    stm32f1xx_hal_flash.o(i.HAL_FLASH_IRQHandler) refers to stm32f1xx_hal_flash.o(.bss) for pFlash
    stm32f1xx_hal_flash.o(i.HAL_FLASH_OB_Launch) refers to stm32f1xx_hal_cortex.o(i.HAL_NVIC_SystemReset) for HAL_NVIC_SystemReset
    stm32f1xx_hal_flash.o(i.HAL_FLASH_Program) refers to stm32f1xx_hal_flash.o(i.FLASH_WaitForLastOperation) for FLASH_WaitForLastOperation
    stm32f1xx_hal_flash.o(i.HAL_FLASH_Program) refers to llushr.o(.text) for __aeabi_llsr
    stm32f1xx_hal_flash.o(i.HAL_FLASH_Program) refers to stm32f1xx_hal_flash.o(i.FLASH_Program_HalfWord) for FLASH_Program_HalfWord
    stm32f1xx_hal_flash.o(i.HAL_FLASH_Program) refers to stm32f1xx_hal_flash.o(.bss) for pFlash
    stm32f1xx_hal_flash.o(i.HAL_FLASH_Program_IT) refers to stm32f1xx_hal_flash.o(i.FLASH_Program_HalfWord) for FLASH_Program_HalfWord
    stm32f1xx_hal_flash.o(i.HAL_FLASH_Program_IT) refers to stm32f1xx_hal_flash.o(.bss) for pFlash
    stm32f1xx_hal_flash_ex.o(i.FLASH_ErasePage) refers to stm32f1xx_hal_flash.o(i.FLASH_WaitForLastOperation) for FLASH_WaitForLastOperation
    stm32f1xx_hal_flash_ex.o(i.FLASH_MassErase) refers to stm32f1xx_hal_flash.o(.bss) for pFlash
    stm32f1xx_hal_flash_ex.o(i.FLASH_OB_DisableWRP) refers to stm32f1xx_hal_flash_ex.o(i.FLASH_OB_GetWRP) for FLASH_OB_GetWRP
    stm32f1xx_hal_flash_ex.o(i.FLASH_OB_DisableWRP) refers to stm32f1xx_hal_flash.o(i.FLASH_WaitForLastOperation) for FLASH_WaitForLastOperation
    stm32f1xx_hal_flash_ex.o(i.FLASH_OB_DisableWRP) refers to stm32f1xx_hal_flash_ex.o(i.HAL_FLASHEx_OBErase) for HAL_FLASHEx_OBErase
    stm32f1xx_hal_flash_ex.o(i.FLASH_OB_DisableWRP) refers to stm32f1xx_hal_flash.o(.bss) for pFlash
    stm32f1xx_hal_flash_ex.o(i.FLASH_OB_EnableWRP) refers to stm32f1xx_hal_flash_ex.o(i.FLASH_OB_GetWRP) for FLASH_OB_GetWRP
    stm32f1xx_hal_flash_ex.o(i.FLASH_OB_EnableWRP) refers to stm32f1xx_hal_flash.o(i.FLASH_WaitForLastOperation) for FLASH_WaitForLastOperation
    stm32f1xx_hal_flash_ex.o(i.FLASH_OB_EnableWRP) refers to stm32f1xx_hal_flash_ex.o(i.HAL_FLASHEx_OBErase) for HAL_FLASHEx_OBErase
    stm32f1xx_hal_flash_ex.o(i.FLASH_OB_EnableWRP) refers to stm32f1xx_hal_flash.o(.bss) for pFlash
    stm32f1xx_hal_flash_ex.o(i.FLASH_OB_ProgramData) refers to stm32f1xx_hal_flash.o(i.FLASH_WaitForLastOperation) for FLASH_WaitForLastOperation
    stm32f1xx_hal_flash_ex.o(i.FLASH_OB_ProgramData) refers to stm32f1xx_hal_flash.o(.bss) for pFlash
    stm32f1xx_hal_flash_ex.o(i.FLASH_OB_RDP_LevelConfig) refers to stm32f1xx_hal_flash.o(i.FLASH_WaitForLastOperation) for FLASH_WaitForLastOperation
    stm32f1xx_hal_flash_ex.o(i.FLASH_OB_RDP_LevelConfig) refers to stm32f1xx_hal_flash.o(.bss) for pFlash
    stm32f1xx_hal_flash_ex.o(i.FLASH_OB_UserConfig) refers to stm32f1xx_hal_flash.o(i.FLASH_WaitForLastOperation) for FLASH_WaitForLastOperation
    stm32f1xx_hal_flash_ex.o(i.FLASH_OB_UserConfig) refers to stm32f1xx_hal_flash.o(.bss) for pFlash
    stm32f1xx_hal_flash_ex.o(i.FLASH_PageErase) refers to stm32f1xx_hal_flash.o(.bss) for pFlash
    stm32f1xx_hal_flash_ex.o(i.HAL_FLASHEx_Erase) refers to stm32f1xx_hal_flash.o(i.FLASH_WaitForLastOperation) for FLASH_WaitForLastOperation
    stm32f1xx_hal_flash_ex.o(i.HAL_FLASHEx_Erase) refers to stm32f1xx_hal_flash_ex.o(i.FLASH_MassErase) for FLASH_MassErase
    stm32f1xx_hal_flash_ex.o(i.HAL_FLASHEx_Erase) refers to stm32f1xx_hal_flash_ex.o(i.FLASH_PageErase) for FLASH_PageErase
    stm32f1xx_hal_flash_ex.o(i.HAL_FLASHEx_Erase) refers to stm32f1xx_hal_flash.o(.bss) for pFlash
    stm32f1xx_hal_flash_ex.o(i.HAL_FLASHEx_Erase_IT) refers to stm32f1xx_hal_flash_ex.o(i.FLASH_MassErase) for FLASH_MassErase
    stm32f1xx_hal_flash_ex.o(i.HAL_FLASHEx_Erase_IT) refers to stm32f1xx_hal_flash_ex.o(i.FLASH_PageErase) for FLASH_PageErase
    stm32f1xx_hal_flash_ex.o(i.HAL_FLASHEx_Erase_IT) refers to stm32f1xx_hal_flash.o(.bss) for pFlash
    stm32f1xx_hal_flash_ex.o(i.HAL_FLASHEx_OBErase) refers to stm32f1xx_hal_flash_ex.o(i.FLASH_OB_GetRDP) for FLASH_OB_GetRDP
    stm32f1xx_hal_flash_ex.o(i.HAL_FLASHEx_OBErase) refers to stm32f1xx_hal_flash.o(i.FLASH_WaitForLastOperation) for FLASH_WaitForLastOperation
    stm32f1xx_hal_flash_ex.o(i.HAL_FLASHEx_OBErase) refers to stm32f1xx_hal_flash_ex.o(i.FLASH_OB_RDP_LevelConfig) for FLASH_OB_RDP_LevelConfig
    stm32f1xx_hal_flash_ex.o(i.HAL_FLASHEx_OBErase) refers to stm32f1xx_hal_flash.o(.bss) for pFlash
    stm32f1xx_hal_flash_ex.o(i.HAL_FLASHEx_OBGetConfig) refers to stm32f1xx_hal_flash_ex.o(i.FLASH_OB_GetWRP) for FLASH_OB_GetWRP
    stm32f1xx_hal_flash_ex.o(i.HAL_FLASHEx_OBGetConfig) refers to stm32f1xx_hal_flash_ex.o(i.FLASH_OB_GetRDP) for FLASH_OB_GetRDP
    stm32f1xx_hal_flash_ex.o(i.HAL_FLASHEx_OBGetConfig) refers to stm32f1xx_hal_flash_ex.o(i.FLASH_OB_GetUser) for FLASH_OB_GetUser
    stm32f1xx_hal_flash_ex.o(i.HAL_FLASHEx_OBProgram) refers to stm32f1xx_hal_flash_ex.o(i.FLASH_OB_EnableWRP) for FLASH_OB_EnableWRP
    stm32f1xx_hal_flash_ex.o(i.HAL_FLASHEx_OBProgram) refers to stm32f1xx_hal_flash_ex.o(i.FLASH_OB_DisableWRP) for FLASH_OB_DisableWRP
    stm32f1xx_hal_flash_ex.o(i.HAL_FLASHEx_OBProgram) refers to stm32f1xx_hal_flash_ex.o(i.FLASH_OB_RDP_LevelConfig) for FLASH_OB_RDP_LevelConfig
    stm32f1xx_hal_flash_ex.o(i.HAL_FLASHEx_OBProgram) refers to stm32f1xx_hal_flash_ex.o(i.FLASH_OB_UserConfig) for FLASH_OB_UserConfig
    stm32f1xx_hal_flash_ex.o(i.HAL_FLASHEx_OBProgram) refers to stm32f1xx_hal_flash_ex.o(i.FLASH_OB_ProgramData) for FLASH_OB_ProgramData
    stm32f1xx_hal_flash_ex.o(i.HAL_FLASHEx_OBProgram) refers to stm32f1xx_hal_flash.o(.bss) for pFlash
    stm32f1xx_hal_gpio.o(i.HAL_GPIO_EXTI_IRQHandler) refers to stm32f1xx_hal_gpio.o(i.HAL_GPIO_EXTI_Callback) for HAL_GPIO_EXTI_Callback
    stm32f1xx_hal_iwdg.o(i.HAL_IWDG_Init) refers to stm32f1xx_hal_msp.o(i.HAL_IWDG_MspInit) for HAL_IWDG_MspInit
    stm32f1xx_hal_iwdg.o(i.HAL_IWDG_Refresh) refers to stm32f1xx_hal.o(i.HAL_GetTick) for HAL_GetTick
    stm32f1xx_hal_pwr.o(i.HAL_PWR_EnterSTOPMode) refers to stm32f1xx_hal_pwr.o(i.PWR_OverloadWfe) for PWR_OverloadWfe
    stm32f1xx_hal_pwr.o(i.HAL_PWR_PVD_IRQHandler) refers to stm32f1xx_hal_pwr.o(i.HAL_PWR_PVDCallback) for HAL_PWR_PVDCallback
    stm32f1xx_hal_rcc.o(i.HAL_RCC_ClockConfig) refers to stm32f1xx_hal.o(i.HAL_GetTick) for HAL_GetTick
    stm32f1xx_hal_rcc.o(i.HAL_RCC_ClockConfig) refers to stm32f1xx_hal.o(i.HAL_InitTick) for HAL_InitTick
    stm32f1xx_hal_rcc.o(i.HAL_RCC_GetHCLKFreq) refers to stm32f1xx_hal_rcc.o(i.HAL_RCC_GetSysClockFreq) for HAL_RCC_GetSysClockFreq
    stm32f1xx_hal_rcc.o(i.HAL_RCC_GetHCLKFreq) refers to stm32f1xx_hal_rcc.o(.constdata) for aAPBAHBPrescTable
    stm32f1xx_hal_rcc.o(i.HAL_RCC_GetHCLKFreq) refers to system_stm32f1xx.o(.data) for SystemCoreClock
    stm32f1xx_hal_rcc.o(i.HAL_RCC_GetPCLK1Freq) refers to stm32f1xx_hal_rcc.o(i.HAL_RCC_GetHCLKFreq) for HAL_RCC_GetHCLKFreq
    stm32f1xx_hal_rcc.o(i.HAL_RCC_GetPCLK1Freq) refers to stm32f1xx_hal_rcc.o(.constdata) for aAPBAHBPrescTable
    stm32f1xx_hal_rcc.o(i.HAL_RCC_GetPCLK2Freq) refers to stm32f1xx_hal_rcc.o(i.HAL_RCC_GetHCLKFreq) for HAL_RCC_GetHCLKFreq
    stm32f1xx_hal_rcc.o(i.HAL_RCC_GetPCLK2Freq) refers to stm32f1xx_hal_rcc.o(.constdata) for aAPBAHBPrescTable
    stm32f1xx_hal_rcc.o(i.HAL_RCC_MCOConfig) refers to stm32f1xx_hal_gpio.o(i.HAL_GPIO_Init) for HAL_GPIO_Init
    stm32f1xx_hal_rcc.o(i.HAL_RCC_NMI_IRQHandler) refers to stm32f1xx_hal_rcc.o(i.HAL_RCC_CSSCallback) for HAL_RCC_CSSCallback
    stm32f1xx_hal_rcc.o(i.HAL_RCC_OscConfig) refers to stm32f1xx_hal.o(i.HAL_GetTick) for HAL_GetTick
    stm32f1xx_hal_rcc.o(i.HAL_RCC_OscConfig) refers to stm32f1xx_hal.o(i.HAL_Delay) for HAL_Delay
    stm32f1xx_hal_rcc_ex.o(i.HAL_RCCEx_GetPeriphCLKFreq) refers to stm32f1xx_hal_rcc.o(i.HAL_RCC_GetSysClockFreq) for HAL_RCC_GetSysClockFreq
    stm32f1xx_hal_rcc_ex.o(i.HAL_RCCEx_GetPeriphCLKFreq) refers to stm32f1xx_hal_rcc.o(i.HAL_RCC_GetPCLK2Freq) for HAL_RCC_GetPCLK2Freq
    stm32f1xx_hal_rcc_ex.o(i.HAL_RCCEx_PeriphCLKConfig) refers to stm32f1xx_hal.o(i.HAL_GetTick) for HAL_GetTick
    stm32f1xx_hal_msp.o(i.HAL_MspInit) refers to stm32f1xx_hal_cortex.o(i.HAL_NVIC_SetPriorityGrouping) for HAL_NVIC_SetPriorityGrouping
    stm32f1xx_hal_msp.o(i.HAL_MspInit) refers to stm32f1xx_hal_cortex.o(i.HAL_NVIC_SetPriority) for HAL_NVIC_SetPriority
    __main.o(!!!main) refers to __rtentry.o(.ARM.Collect$$rtentry$$00000000) for __rt_entry
    dfixu.o(x$fpl$dfixu) refers (Special) to usenofp.o(x$fpl$usenofp) for __I$use$fp
    dfixu.o(x$fpl$dfixu) refers to dnaninf.o(x$fpl$dnaninf) for __fpl_dnaninf
    dfixu.o(x$fpl$dfixur) refers (Special) to usenofp.o(x$fpl$usenofp) for __I$use$fp
    dfixu.o(x$fpl$dfixur) refers to dnaninf.o(x$fpl$dnaninf) for __fpl_dnaninf
    dflt_clz.o(x$fpl$dfltu) refers (Special) to usenofp.o(x$fpl$usenofp) for __I$use$fp
    dflt_clz.o(x$fpl$dflt) refers (Special) to usenofp.o(x$fpl$usenofp) for __I$use$fp
    dflt_clz.o(x$fpl$dfltn) refers (Special) to usenofp.o(x$fpl$usenofp) for __I$use$fp
    dmul.o(x$fpl$dmul) refers (Special) to usenofp.o(x$fpl$usenofp) for __I$use$fp
    dmul.o(x$fpl$dmul) refers to dretinf.o(x$fpl$dretinf) for __fpl_dretinf
    dmul.o(x$fpl$dmul) refers to dnaninf.o(x$fpl$dnaninf) for __fpl_dnaninf
    __rtentry.o(.ARM.Collect$$rtentry$$00000000) refers (Special) to __rtentry2.o(.ARM.Collect$$rtentry$$0000000A) for __rt_entry_li
    __rtentry.o(.ARM.Collect$$rtentry$$00000000) refers (Special) to __rtentry2.o(.ARM.Collect$$rtentry$$0000000D) for __rt_entry_main
    __rtentry.o(.ARM.Collect$$rtentry$$00000000) refers (Special) to __rtentry2.o(.ARM.Collect$$rtentry$$0000000C) for __rt_entry_postli_1
    __rtentry.o(.ARM.Collect$$rtentry$$00000000) refers (Special) to __rtentry2.o(.ARM.Collect$$rtentry$$00000009) for __rt_entry_postsh_1
    __rtentry.o(.ARM.Collect$$rtentry$$00000000) refers (Special) to __rtentry2.o(.ARM.Collect$$rtentry$$00000002) for __rt_entry_presh_1
    __rtentry.o(.ARM.Collect$$rtentry$$00000000) refers (Special) to __rtentry4.o(.ARM.Collect$$rtentry$$00000004) for __rt_entry_sh
    dnaninf.o(x$fpl$dnaninf) refers (Special) to usenofp.o(x$fpl$usenofp) for __I$use$fp
    dretinf.o(x$fpl$dretinf) refers (Special) to usenofp.o(x$fpl$usenofp) for __I$use$fp
    __rtentry2.o(.ARM.Collect$$rtentry$$00000008) refers to boardinit2.o(.text) for _platform_post_stackheap_init
    __rtentry2.o(.ARM.Collect$$rtentry$$0000000A) refers to libinit.o(.ARM.Collect$$libinit$$00000000) for __rt_lib_init
    __rtentry2.o(.ARM.Collect$$rtentry$$0000000B) refers to boardinit3.o(.text) for _platform_post_lib_init
    __rtentry2.o(.ARM.Collect$$rtentry$$0000000D) refers to demo.o(i.main) for main
    __rtentry2.o(.ARM.Collect$$rtentry$$0000000D) refers to exit.o(.text) for exit
    __rtentry2.o(.ARM.exidx) refers to __rtentry2.o(.ARM.Collect$$rtentry$$00000001) for .ARM.Collect$$rtentry$$00000001
    __rtentry2.o(.ARM.exidx) refers to __rtentry2.o(.ARM.Collect$$rtentry$$00000008) for .ARM.Collect$$rtentry$$00000008
    __rtentry2.o(.ARM.exidx) refers to __rtentry2.o(.ARM.Collect$$rtentry$$0000000A) for .ARM.Collect$$rtentry$$0000000A
    __rtentry2.o(.ARM.exidx) refers to __rtentry2.o(.ARM.Collect$$rtentry$$0000000B) for .ARM.Collect$$rtentry$$0000000B
    __rtentry2.o(.ARM.exidx) refers to __rtentry2.o(.ARM.Collect$$rtentry$$0000000D) for .ARM.Collect$$rtentry$$0000000D
    __rtentry4.o(.ARM.Collect$$rtentry$$00000004) refers to sys_stackheap_outer.o(.text) for __user_setup_stackheap
    __rtentry4.o(.ARM.exidx) refers to __rtentry4.o(.ARM.Collect$$rtentry$$00000004) for .ARM.Collect$$rtentry$$00000004
    sys_stackheap_outer.o(.text) refers to libspace.o(.text) for __user_perproc_libspace
    sys_stackheap_outer.o(.text) refers to startup_stm32f10x_hd.o(.text) for __user_initial_stackheap
    exit.o(.text) refers to rtexit.o(.ARM.Collect$$rtexit$$00000000) for __rt_exit
    libinit.o(.ARM.Collect$$libinit$$00000000) refers (Special) to libinit2.o(.ARM.Collect$$libinit$$0000002E) for __rt_lib_init_alloca_1
    libinit.o(.ARM.Collect$$libinit$$00000000) refers (Special) to libinit2.o(.ARM.Collect$$libinit$$0000002C) for __rt_lib_init_argv_1
    libinit.o(.ARM.Collect$$libinit$$00000000) refers (Special) to libinit2.o(.ARM.Collect$$libinit$$0000001B) for __rt_lib_init_atexit_1
    libinit.o(.ARM.Collect$$libinit$$00000000) refers (Special) to libinit2.o(.ARM.Collect$$libinit$$00000021) for __rt_lib_init_clock_1
    libinit.o(.ARM.Collect$$libinit$$00000000) refers (Special) to libinit2.o(.ARM.Collect$$libinit$$00000032) for __rt_lib_init_cpp_1
    libinit.o(.ARM.Collect$$libinit$$00000000) refers (Special) to libinit2.o(.ARM.Collect$$libinit$$00000030) for __rt_lib_init_exceptions_1
    libinit.o(.ARM.Collect$$libinit$$00000000) refers (Special) to libinit2.o(.ARM.Collect$$libinit$$00000002) for __rt_lib_init_fp_1
    libinit.o(.ARM.Collect$$libinit$$00000000) refers (Special) to libinit2.o(.ARM.Collect$$libinit$$0000001F) for __rt_lib_init_fp_trap_1
    libinit.o(.ARM.Collect$$libinit$$00000000) refers (Special) to libinit2.o(.ARM.Collect$$libinit$$00000023) for __rt_lib_init_getenv_1
    libinit.o(.ARM.Collect$$libinit$$00000000) refers (Special) to libinit2.o(.ARM.Collect$$libinit$$0000000A) for __rt_lib_init_heap_1
    libinit.o(.ARM.Collect$$libinit$$00000000) refers (Special) to libinit2.o(.ARM.Collect$$libinit$$00000011) for __rt_lib_init_lc_collate_1
    libinit.o(.ARM.Collect$$libinit$$00000000) refers (Special) to libinit2.o(.ARM.Collect$$libinit$$00000013) for __rt_lib_init_lc_ctype_1
    libinit.o(.ARM.Collect$$libinit$$00000000) refers (Special) to libinit2.o(.ARM.Collect$$libinit$$00000015) for __rt_lib_init_lc_monetary_1
    libinit.o(.ARM.Collect$$libinit$$00000000) refers (Special) to libinit2.o(.ARM.Collect$$libinit$$00000017) for __rt_lib_init_lc_numeric_1
    libinit.o(.ARM.Collect$$libinit$$00000000) refers (Special) to libinit2.o(.ARM.Collect$$libinit$$00000019) for __rt_lib_init_lc_time_1
    libinit.o(.ARM.Collect$$libinit$$00000000) refers (Special) to libinit2.o(.ARM.Collect$$libinit$$00000004) for __rt_lib_init_preinit_1
    libinit.o(.ARM.Collect$$libinit$$00000000) refers (Special) to libinit2.o(.ARM.Collect$$libinit$$0000000E) for __rt_lib_init_rand_1
    libinit.o(.ARM.Collect$$libinit$$00000000) refers (Special) to libinit2.o(.ARM.Collect$$libinit$$00000033) for __rt_lib_init_return
    libinit.o(.ARM.Collect$$libinit$$00000000) refers (Special) to libinit2.o(.ARM.Collect$$libinit$$0000001D) for __rt_lib_init_signal_1
    libinit.o(.ARM.Collect$$libinit$$00000000) refers (Special) to libinit2.o(.ARM.Collect$$libinit$$00000025) for __rt_lib_init_stdio_1
    libinit.o(.ARM.Collect$$libinit$$00000000) refers (Special) to libinit2.o(.ARM.Collect$$libinit$$0000000C) for __rt_lib_init_user_alloc_1
    libspace.o(.text) refers to libspace.o(.bss) for __libspace_start
    rtexit.o(.ARM.Collect$$rtexit$$00000000) refers (Special) to rtexit2.o(.ARM.Collect$$rtexit$$00000004) for __rt_exit_exit
    rtexit.o(.ARM.Collect$$rtexit$$00000000) refers (Special) to rtexit2.o(.ARM.Collect$$rtexit$$00000003) for __rt_exit_ls
    rtexit.o(.ARM.Collect$$rtexit$$00000000) refers (Special) to rtexit2.o(.ARM.Collect$$rtexit$$00000002) for __rt_exit_prels_1
    rtexit.o(.ARM.exidx) refers (Special) to rtexit2.o(.ARM.Collect$$rtexit$$00000004) for __rt_exit_exit
    rtexit.o(.ARM.exidx) refers (Special) to rtexit2.o(.ARM.Collect$$rtexit$$00000003) for __rt_exit_ls
    rtexit.o(.ARM.exidx) refers (Special) to rtexit2.o(.ARM.Collect$$rtexit$$00000002) for __rt_exit_prels_1
    rtexit.o(.ARM.exidx) refers to rtexit.o(.ARM.Collect$$rtexit$$00000000) for .ARM.Collect$$rtexit$$00000000
    libinit2.o(.ARM.Collect$$libinit$$00000010) refers to libinit2.o(.ARM.Collect$$libinit$$0000000F) for .ARM.Collect$$libinit$$0000000F
    libinit2.o(.ARM.Collect$$libinit$$00000012) refers to libinit2.o(.ARM.Collect$$libinit$$0000000F) for .ARM.Collect$$libinit$$0000000F
    libinit2.o(.ARM.Collect$$libinit$$00000014) refers to libinit2.o(.ARM.Collect$$libinit$$0000000F) for .ARM.Collect$$libinit$$0000000F
    libinit2.o(.ARM.Collect$$libinit$$00000016) refers to libinit2.o(.ARM.Collect$$libinit$$0000000F) for .ARM.Collect$$libinit$$0000000F
    libinit2.o(.ARM.Collect$$libinit$$00000018) refers to libinit2.o(.ARM.Collect$$libinit$$0000000F) for .ARM.Collect$$libinit$$0000000F
    libinit2.o(.ARM.Collect$$libinit$$00000026) refers to argv_veneer.o(.emb_text) for __ARM_argv_veneer
    libinit2.o(.ARM.Collect$$libinit$$00000027) refers to argv_veneer.o(.emb_text) for __ARM_argv_veneer
    rtexit2.o(.ARM.Collect$$rtexit$$00000003) refers to libshutdown.o(.ARM.Collect$$libshutdown$$00000000) for __rt_lib_shutdown
    rtexit2.o(.ARM.Collect$$rtexit$$00000004) refers to sys_exit.o(.text) for _sys_exit
    rtexit2.o(.ARM.exidx) refers to rtexit2.o(.ARM.Collect$$rtexit$$00000001) for .ARM.Collect$$rtexit$$00000001
    rtexit2.o(.ARM.exidx) refers to rtexit2.o(.ARM.Collect$$rtexit$$00000003) for .ARM.Collect$$rtexit$$00000003
    rtexit2.o(.ARM.exidx) refers to rtexit2.o(.ARM.Collect$$rtexit$$00000004) for .ARM.Collect$$rtexit$$00000004
    argv_veneer.o(.emb_text) refers to no_argv.o(.text) for __ARM_get_argv
    sys_exit.o(.text) refers (Special) to use_no_semi.o(.text) for __I$use$semihosting
    sys_exit.o(.text) refers (Special) to indicate_semi.o(.text) for __semihosting_library_function
    _get_argv_nomalloc.o(.text) refers (Special) to hrguard.o(.text) for __heap_region$guard
    _get_argv_nomalloc.o(.text) refers to defsig_rtmem_outer.o(.text) for __rt_SIGRTMEM
    _get_argv_nomalloc.o(.text) refers to sys_command.o(.text) for _sys_command_string
    libshutdown.o(.ARM.Collect$$libshutdown$$00000000) refers (Special) to libshutdown2.o(.ARM.Collect$$libshutdown$$00000002) for __rt_lib_shutdown_cpp_1
    libshutdown.o(.ARM.Collect$$libshutdown$$00000000) refers (Special) to libshutdown2.o(.ARM.Collect$$libshutdown$$00000007) for __rt_lib_shutdown_fp_trap_1
    libshutdown.o(.ARM.Collect$$libshutdown$$00000000) refers (Special) to libshutdown2.o(.ARM.Collect$$libshutdown$$0000000F) for __rt_lib_shutdown_heap_1
    libshutdown.o(.ARM.Collect$$libshutdown$$00000000) refers (Special) to libshutdown2.o(.ARM.Collect$$libshutdown$$00000010) for __rt_lib_shutdown_return
    libshutdown.o(.ARM.Collect$$libshutdown$$00000000) refers (Special) to libshutdown2.o(.ARM.Collect$$libshutdown$$0000000A) for __rt_lib_shutdown_signal_1
    libshutdown.o(.ARM.Collect$$libshutdown$$00000000) refers (Special) to libshutdown2.o(.ARM.Collect$$libshutdown$$00000004) for __rt_lib_shutdown_stdio_1
    libshutdown.o(.ARM.Collect$$libshutdown$$00000000) refers (Special) to libshutdown2.o(.ARM.Collect$$libshutdown$$0000000C) for __rt_lib_shutdown_user_alloc_1
    sys_command.o(.text) refers (Special) to use_no_semi.o(.text) for __I$use$semihosting
    sys_command.o(.text) refers (Special) to indicate_semi.o(.text) for __semihosting_library_function
    defsig_rtmem_outer.o(.text) refers to defsig_rtmem_inner.o(.text) for __rt_SIGRTMEM_inner
    defsig_rtmem_outer.o(.text) refers to defsig_exit.o(.text) for __sig_exit
    defsig_rtmem_formal.o(.text) refers to rt_raise.o(.text) for __rt_raise
    rt_raise.o(.text) refers to __raise.o(.text) for __raise
    rt_raise.o(.text) refers to sys_exit.o(.text) for _sys_exit
    defsig_exit.o(.text) refers to sys_exit.o(.text) for _sys_exit
    defsig_rtmem_inner.o(.text) refers to defsig_general.o(.text) for __default_signal_display
    __raise.o(.text) refers to defsig.o(CL$$defsig) for __default_signal_handler
    defsig_general.o(.text) refers to sys_wrch.o(.text) for _ttywrch
    sys_wrch.o(.text) refers (Special) to use_no_semi.o(.text) for __I$use$semihosting
    sys_wrch.o(.text) refers (Special) to indicate_semi.o(.text) for __semihosting_library_function
    defsig.o(CL$$defsig) refers to defsig_rtmem_inner.o(.text) for __rt_SIGRTMEM_inner
    defsig_abrt_inner.o(.text) refers to defsig_general.o(.text) for __default_signal_display
    defsig_fpe_inner.o(.text) refers to defsig_general.o(.text) for __default_signal_display
    defsig_rtred_inner.o(.text) refers to defsig_general.o(.text) for __default_signal_display
    defsig_stak_inner.o(.text) refers to defsig_general.o(.text) for __default_signal_display
    defsig_pvfn_inner.o(.text) refers to defsig_general.o(.text) for __default_signal_display
    defsig_cppl_inner.o(.text) refers to defsig_general.o(.text) for __default_signal_display
    defsig_segv_inner.o(.text) refers to defsig_general.o(.text) for __default_signal_display
    defsig_other.o(.text) refers to defsig_general.o(.text) for __default_signal_display


==============================================================================

Removing Unused input sections from the image.

    Removing system_stm32f10x_cl.o(.rev16_text), (4 bytes).
    Removing system_stm32f10x_cl.o(.revsh_text), (4 bytes).
    Removing chip_uip_interrupt.o(i.Chip_UIP_InterruptRemoveHandler), (24 bytes).
    Removing chip_uip_interrupt.o(i.Chip_UIP_Kernel_Tick_ISR_Handler), (12 bytes).
    Removing chip_uip_interrupt.o(i.Chip_UIP_Kernel_Tick_ISR_Handler_Callback), (6 bytes).
    Removing hardware_init.o(.rev16_text), (4 bytes).
    Removing hardware_init.o(.revsh_text), (4 bytes).
    Removing hardware_init.o(i.STM32_OSC_Init), (74 bytes).
    Removing hardware_init.o(.bss), (10 bytes).
    Removing system_stm32f1xx.o(.rev16_text), (4 bytes).
    Removing system_stm32f1xx.o(.revsh_text), (4 bytes).
    Removing system_stm32f1xx.o(i.SystemCoreClockUpdate), (172 bytes).
    Removing system_stm32f1xx.o(.constdata), (16 bytes).
    Removing demo.o(i.uipCOMInit), (4 bytes).
    Removing demo.o(.data), (16 bytes).
    Removing hook.o(i.COMErrorHook), (2 bytes).
    Removing hook.o(i.ErrorHook), (2 bytes).
    Removing hook.o(i.PostTaskHook), (2 bytes).
    Removing hook.o(i.PreTaskHook), (2 bytes).
    Removing hook.o(i.ShutdownHook), (2 bytes).
    Removing hook.o(i.StuipCOMExtension), (4 bytes).
    Removing hook.o(i.StuipupHook), (2 bytes).
    Removing app_int_cfg.o(i.Chip_STM32F103_UART1_ISR_Handler_Callback), (6 bytes).
    Removing uip_kernel_common.o(i.ShutdownOS), (2 bytes).
    Removing uip_kernel_common.o(i.uipAlarmInfoInit), (20 bytes).
    Removing uip_kernel_common.o(i.uipMsgInfoInit), (20 bytes).
    Removing uip_kernel_common.o(i.uipResInfoInit), (20 bytes).
    Removing uip_kernel_common.o(i.uipTaskInfoInit), (20 bytes).
    Removing uip_kernel_event.o(i.UIP_GetEvent), (116 bytes).
    Removing uip_kernel_message.o(i.UIP_CloseCOM), (4 bytes).
    Removing uip_kernel_message.o(i.UIP_GetMessageStatus), (88 bytes).
    Removing uip_kernel_message.o(i.UIP_ReadFlag), (24 bytes).
    Removing uip_kernel_message.o(i.UIP_ResetFlag), (40 bytes).
    Removing uip_kernel_message.o(i.UIP_SendMessage), (272 bytes).
    Removing uip_kernel_message.o(i.UIP_StartCOM), (12 bytes).
    Removing uip_kernel_message.o(i.UIP_StopCOM), (56 bytes).
    Removing uip_kernel_task.o(i.UIP_ChainTask), (388 bytes).
    Removing uip_kernel_task.o(i.UIP_GetTaskID), (28 bytes).
    Removing uip_kernel_task.o(i.UIP_GetTaskState), (68 bytes).
    Removing uip_kernel_task.o(i.UIP_Schedule), (272 bytes).
    Removing uip_kernel_time.o(i.UIP_CancelAlarm), (72 bytes).
    Removing uip_kernel_time.o(i.UIP_GetAlarm), (112 bytes).
    Removing uip_kernel_time.o(i.UIP_GetAlarmBase), (48 bytes).
    Removing uip_kernel_time.o(i.UIP_SetAbsAlarm), (136 bytes).
    Removing uip_kernel_time.o(i.UIP_SetRelAlarm), (180 bytes).
    Removing uip_kernel_time.o(i.uipGeneralCounterHandler), (88 bytes).
    Removing uip_kernel_time.o(i.uipGetCtrCurrentValue), (80 bytes).
    Removing stm32f1xx_hal.o(.rev16_text), (4 bytes).
    Removing stm32f1xx_hal.o(.revsh_text), (4 bytes).
    Removing stm32f1xx_hal.o(i.HAL_DBGMCU_DisableDBGSleepMode), (20 bytes).
    Removing stm32f1xx_hal.o(i.HAL_DBGMCU_DisableDBGStandbyMode), (20 bytes).
    Removing stm32f1xx_hal.o(i.HAL_DBGMCU_DisableDBGStopMode), (20 bytes).
    Removing stm32f1xx_hal.o(i.HAL_DBGMCU_EnableDBGSleepMode), (20 bytes).
    Removing stm32f1xx_hal.o(i.HAL_DBGMCU_EnableDBGStandbyMode), (20 bytes).
    Removing stm32f1xx_hal.o(i.HAL_DBGMCU_EnableDBGStopMode), (20 bytes).
    Removing stm32f1xx_hal.o(i.HAL_DeInit), (36 bytes).
    Removing stm32f1xx_hal.o(i.HAL_Delay), (26 bytes).
    Removing stm32f1xx_hal.o(i.HAL_GetDEVID), (16 bytes).
    Removing stm32f1xx_hal.o(i.HAL_GetHalVersion), (8 bytes).
    Removing stm32f1xx_hal.o(i.HAL_GetREVID), (28 bytes).
    Removing stm32f1xx_hal.o(i.HAL_GetTick), (12 bytes).
    Removing stm32f1xx_hal.o(i.HAL_IncTick), (16 bytes).
    Removing stm32f1xx_hal.o(i.HAL_Init), (40 bytes).
    Removing stm32f1xx_hal.o(i.HAL_InitTick), (36 bytes).
    Removing stm32f1xx_hal.o(i.HAL_MspDeInit), (2 bytes).
    Removing stm32f1xx_hal.o(i.HAL_MspInit), (2 bytes).
    Removing stm32f1xx_hal.o(i.HAL_ResumeTick), (18 bytes).
    Removing stm32f1xx_hal.o(i.HAL_SuspendTick), (18 bytes).
    Removing stm32f1xx_hal.o(.data), (4 bytes).
    Removing stm32f1xx_hal_adc.o(.rev16_text), (4 bytes).
    Removing stm32f1xx_hal_adc.o(.revsh_text), (4 bytes).
    Removing stm32f1xx_hal_adc_ex.o(.rev16_text), (4 bytes).
    Removing stm32f1xx_hal_adc_ex.o(.revsh_text), (4 bytes).
    Removing stm32f1xx_hal_can.o(.rev16_text), (4 bytes).
    Removing stm32f1xx_hal_can.o(.revsh_text), (4 bytes).
    Removing stm32f1xx_hal_cec.o(.rev16_text), (4 bytes).
    Removing stm32f1xx_hal_cec.o(.revsh_text), (4 bytes).
    Removing stm32f1xx_hal_cortex.o(.rev16_text), (4 bytes).
    Removing stm32f1xx_hal_cortex.o(.revsh_text), (4 bytes).
    Removing stm32f1xx_hal_cortex.o(i.HAL_NVIC_ClearPendingIRQ), (28 bytes).
    Removing stm32f1xx_hal_cortex.o(i.HAL_NVIC_DisableIRQ), (28 bytes).
    Removing stm32f1xx_hal_cortex.o(i.HAL_NVIC_EnableIRQ), (26 bytes).
    Removing stm32f1xx_hal_cortex.o(i.HAL_NVIC_GetActive), (40 bytes).
    Removing stm32f1xx_hal_cortex.o(i.HAL_NVIC_GetPendingIRQ), (40 bytes).
    Removing stm32f1xx_hal_cortex.o(i.HAL_NVIC_GetPriority), (148 bytes).
    Removing stm32f1xx_hal_cortex.o(i.HAL_NVIC_GetPriorityGrouping), (8 bytes).
    Removing stm32f1xx_hal_cortex.o(i.HAL_NVIC_SetPendingIRQ), (28 bytes).
    Removing stm32f1xx_hal_cortex.o(i.HAL_NVIC_SystemReset), (44 bytes).
    Removing stm32f1xx_hal_cortex.o(i.HAL_SYSTICK_Callback), (2 bytes).
    Removing stm32f1xx_hal_cortex.o(i.HAL_SYSTICK_IRQHandler), (8 bytes).
    Removing stm32f1xx_hal_crc.o(.rev16_text), (4 bytes).
    Removing stm32f1xx_hal_crc.o(.revsh_text), (4 bytes).
    Removing stm32f1xx_hal_dac.o(.rev16_text), (4 bytes).
    Removing stm32f1xx_hal_dac.o(.revsh_text), (4 bytes).
    Removing stm32f1xx_hal_dac_ex.o(.rev16_text), (4 bytes).
    Removing stm32f1xx_hal_dac_ex.o(.revsh_text), (4 bytes).
    Removing stm32f1xx_hal_dma.o(.rev16_text), (4 bytes).
    Removing stm32f1xx_hal_dma.o(.revsh_text), (4 bytes).
    Removing stm32f1xx_hal_dma.o(i.DMA_SetConfig), (32 bytes).
    Removing stm32f1xx_hal_dma.o(i.HAL_DMA_Abort), (98 bytes).
    Removing stm32f1xx_hal_dma.o(i.HAL_DMA_DeInit), (1120 bytes).
    Removing stm32f1xx_hal_dma.o(i.HAL_DMA_GetError), (6 bytes).
    Removing stm32f1xx_hal_dma.o(i.HAL_DMA_GetState), (8 bytes).
    Removing stm32f1xx_hal_dma.o(i.HAL_DMA_IRQHandler), (2312 bytes).
    Removing stm32f1xx_hal_dma.o(i.HAL_DMA_Init), (84 bytes).
    Removing stm32f1xx_hal_dma.o(i.HAL_DMA_PollForTransfer), (1916 bytes).
    Removing stm32f1xx_hal_dma.o(i.HAL_DMA_Start), (82 bytes).
    Removing stm32f1xx_hal_dma.o(i.HAL_DMA_Start_IT), (118 bytes).
    Removing stm32f1xx_hal_eth.o(.rev16_text), (4 bytes).
    Removing stm32f1xx_hal_eth.o(.revsh_text), (4 bytes).
    Removing stm32f1xx_hal_flash.o(.rev16_text), (4 bytes).
    Removing stm32f1xx_hal_flash.o(.revsh_text), (4 bytes).
    Removing stm32f1xx_hal_flash.o(i.FLASH_Program_HalfWord), (32 bytes).
    Removing stm32f1xx_hal_flash.o(i.FLASH_SetErrorCode), (104 bytes).
    Removing stm32f1xx_hal_flash.o(i.FLASH_WaitForLastOperation), (112 bytes).
    Removing stm32f1xx_hal_flash.o(i.HAL_FLASH_EndOfOperationCallback), (2 bytes).
    Removing stm32f1xx_hal_flash.o(i.HAL_FLASH_GetError), (12 bytes).
    Removing stm32f1xx_hal_flash.o(i.HAL_FLASH_IRQHandler), (384 bytes).
    Removing stm32f1xx_hal_flash.o(i.HAL_FLASH_Lock), (20 bytes).
    Removing stm32f1xx_hal_flash.o(i.HAL_FLASH_OB_Launch), (10 bytes).
    Removing stm32f1xx_hal_flash.o(i.HAL_FLASH_OB_Lock), (20 bytes).
    Removing stm32f1xx_hal_flash.o(i.HAL_FLASH_OB_Unlock), (44 bytes).
    Removing stm32f1xx_hal_flash.o(i.HAL_FLASH_OperationErrorCallback), (2 bytes).
    Removing stm32f1xx_hal_flash.o(i.HAL_FLASH_Program), (176 bytes).
    Removing stm32f1xx_hal_flash.o(i.HAL_FLASH_Program_IT), (124 bytes).
    Removing stm32f1xx_hal_flash.o(i.HAL_FLASH_Unlock), (44 bytes).
    Removing stm32f1xx_hal_flash.o(.bss), (32 bytes).
    Removing stm32f1xx_hal_flash_ex.o(.rev16_text), (4 bytes).
    Removing stm32f1xx_hal_flash_ex.o(.revsh_text), (4 bytes).
    Removing stm32f1xx_hal_flash_ex.o(i.FLASH_ErasePage), (96 bytes).
    Removing stm32f1xx_hal_flash_ex.o(i.FLASH_MassErase), (40 bytes).
    Removing stm32f1xx_hal_flash_ex.o(i.FLASH_OB_DisableWRP), (232 bytes).
    Removing stm32f1xx_hal_flash_ex.o(i.FLASH_OB_EnableWRP), (236 bytes).
    Removing stm32f1xx_hal_flash_ex.o(i.FLASH_OB_GetRDP), (28 bytes).
    Removing stm32f1xx_hal_flash_ex.o(i.FLASH_OB_GetUser), (28 bytes).
    Removing stm32f1xx_hal_flash_ex.o(i.FLASH_OB_GetWRP), (12 bytes).
    Removing stm32f1xx_hal_flash_ex.o(i.FLASH_OB_ProgramData), (76 bytes).
    Removing stm32f1xx_hal_flash_ex.o(i.FLASH_OB_RDP_LevelConfig), (124 bytes).
    Removing stm32f1xx_hal_flash_ex.o(i.FLASH_OB_UserConfig), (84 bytes).
    Removing stm32f1xx_hal_flash_ex.o(i.FLASH_PageErase), (40 bytes).
    Removing stm32f1xx_hal_flash_ex.o(i.HAL_FLASHEx_Erase), (176 bytes).
    Removing stm32f1xx_hal_flash_ex.o(i.HAL_FLASHEx_Erase_IT), (100 bytes).
    Removing stm32f1xx_hal_flash_ex.o(i.HAL_FLASHEx_OBErase), (96 bytes).
    Removing stm32f1xx_hal_flash_ex.o(i.HAL_FLASHEx_OBGetConfig), (28 bytes).
    Removing stm32f1xx_hal_flash_ex.o(i.HAL_FLASHEx_OBGetUserData), (72 bytes).
    Removing stm32f1xx_hal_flash_ex.o(i.HAL_FLASHEx_OBProgram), (200 bytes).
    Removing stm32f1xx_hal_gpio.o(.rev16_text), (4 bytes).
    Removing stm32f1xx_hal_gpio.o(.revsh_text), (4 bytes).
    Removing stm32f1xx_hal_gpio.o(i.HAL_GPIO_DeInit), (344 bytes).
    Removing stm32f1xx_hal_gpio.o(i.HAL_GPIO_EXTI_Callback), (2 bytes).
    Removing stm32f1xx_hal_gpio.o(i.HAL_GPIO_EXTI_IRQHandler), (28 bytes).
    Removing stm32f1xx_hal_gpio.o(i.HAL_GPIO_Init), (832 bytes).
    Removing stm32f1xx_hal_gpio.o(i.HAL_GPIO_LockPin), (46 bytes).
    Removing stm32f1xx_hal_gpio.o(i.HAL_GPIO_ReadPin), (16 bytes).
    Removing stm32f1xx_hal_gpio.o(i.HAL_GPIO_TogglePin), (8 bytes).
    Removing stm32f1xx_hal_gpio.o(i.HAL_GPIO_WritePin), (12 bytes).
    Removing stm32f1xx_hal_gpio_ex.o(.rev16_text), (4 bytes).
    Removing stm32f1xx_hal_gpio_ex.o(.revsh_text), (4 bytes).
    Removing stm32f1xx_hal_gpio_ex.o(i.HAL_GPIOEx_ConfigEventout), (24 bytes).
    Removing stm32f1xx_hal_gpio_ex.o(i.HAL_GPIOEx_DisableEventout), (20 bytes).
    Removing stm32f1xx_hal_gpio_ex.o(i.HAL_GPIOEx_EnableEventout), (20 bytes).
    Removing stm32f1xx_hal_hcd.o(.rev16_text), (4 bytes).
    Removing stm32f1xx_hal_hcd.o(.revsh_text), (4 bytes).
    Removing stm32f1xx_hal_i2c.o(.rev16_text), (4 bytes).
    Removing stm32f1xx_hal_i2c.o(.revsh_text), (4 bytes).
    Removing stm32f1xx_hal_i2s.o(.rev16_text), (4 bytes).
    Removing stm32f1xx_hal_i2s.o(.revsh_text), (4 bytes).
    Removing stm32f1xx_hal_irda.o(.rev16_text), (4 bytes).
    Removing stm32f1xx_hal_irda.o(.revsh_text), (4 bytes).
    Removing stm32f1xx_hal_iwdg.o(.rev16_text), (4 bytes).
    Removing stm32f1xx_hal_iwdg.o(.revsh_text), (4 bytes).
    Removing stm32f1xx_hal_iwdg.o(i.HAL_IWDG_GetState), (6 bytes).
    Removing stm32f1xx_hal_iwdg.o(i.HAL_IWDG_Init), (100 bytes).
    Removing stm32f1xx_hal_iwdg.o(i.HAL_IWDG_MspInit), (2 bytes).
    Removing stm32f1xx_hal_iwdg.o(i.HAL_IWDG_Refresh), (100 bytes).
    Removing stm32f1xx_hal_iwdg.o(i.HAL_IWDG_Start), (56 bytes).
    Removing stm32f1xx_hal_nand.o(.rev16_text), (4 bytes).
    Removing stm32f1xx_hal_nand.o(.revsh_text), (4 bytes).
    Removing stm32f1xx_hal_nor.o(.rev16_text), (4 bytes).
    Removing stm32f1xx_hal_nor.o(.revsh_text), (4 bytes).
    Removing stm32f1xx_hal_pccard.o(.rev16_text), (4 bytes).
    Removing stm32f1xx_hal_pccard.o(.revsh_text), (4 bytes).
    Removing stm32f1xx_hal_pcd.o(.rev16_text), (4 bytes).
    Removing stm32f1xx_hal_pcd.o(.revsh_text), (4 bytes).
    Removing stm32f1xx_hal_pcd_ex.o(.rev16_text), (4 bytes).
    Removing stm32f1xx_hal_pcd_ex.o(.revsh_text), (4 bytes).
    Removing stm32f1xx_hal_pwr.o(.rev16_text), (4 bytes).
    Removing stm32f1xx_hal_pwr.o(.revsh_text), (4 bytes).
    Removing stm32f1xx_hal_pwr.o(i.HAL_PWR_ConfigPVD), (180 bytes).
    Removing stm32f1xx_hal_pwr.o(i.HAL_PWR_DeInit), (28 bytes).
    Removing stm32f1xx_hal_pwr.o(i.HAL_PWR_DisableBkUpAccess), (28 bytes).
    Removing stm32f1xx_hal_pwr.o(i.HAL_PWR_DisablePVD), (24 bytes).
    Removing stm32f1xx_hal_pwr.o(i.HAL_PWR_DisableSEVOnPend), (20 bytes).
    Removing stm32f1xx_hal_pwr.o(i.HAL_PWR_DisableSleepOnExit), (20 bytes).
    Removing stm32f1xx_hal_pwr.o(i.HAL_PWR_DisableWakeUpPin), (28 bytes).
    Removing stm32f1xx_hal_pwr.o(i.HAL_PWR_EnableBkUpAccess), (24 bytes).
    Removing stm32f1xx_hal_pwr.o(i.HAL_PWR_EnablePVD), (24 bytes).
    Removing stm32f1xx_hal_pwr.o(i.HAL_PWR_EnableSEVOnPend), (20 bytes).
    Removing stm32f1xx_hal_pwr.o(i.HAL_PWR_EnableSleepOnExit), (20 bytes).
    Removing stm32f1xx_hal_pwr.o(i.HAL_PWR_EnableWakeUpPin), (28 bytes).
    Removing stm32f1xx_hal_pwr.o(i.HAL_PWR_EnterSLEEPMode), (32 bytes).
    Removing stm32f1xx_hal_pwr.o(i.HAL_PWR_EnterSTANDBYMode), (40 bytes).
    Removing stm32f1xx_hal_pwr.o(i.HAL_PWR_EnterSTOPMode), (84 bytes).
    Removing stm32f1xx_hal_pwr.o(i.HAL_PWR_PVDCallback), (2 bytes).
    Removing stm32f1xx_hal_pwr.o(i.HAL_PWR_PVD_IRQHandler), (32 bytes).
    Removing stm32f1xx_hal_pwr.o(i.PWR_OverloadWfe), (6 bytes).
    Removing stm32f1xx_hal_rcc.o(.rev16_text), (4 bytes).
    Removing stm32f1xx_hal_rcc.o(.revsh_text), (4 bytes).
    Removing stm32f1xx_hal_rcc.o(i.HAL_RCC_CSSCallback), (2 bytes).
    Removing stm32f1xx_hal_rcc.o(i.HAL_RCC_ClockConfig), (1076 bytes).
    Removing stm32f1xx_hal_rcc.o(i.HAL_RCC_DeInit), (80 bytes).
    Removing stm32f1xx_hal_rcc.o(i.HAL_RCC_DisableCSS), (28 bytes).
    Removing stm32f1xx_hal_rcc.o(i.HAL_RCC_EnableCSS), (24 bytes).
    Removing stm32f1xx_hal_rcc.o(i.HAL_RCC_GetClockConfig), (68 bytes).
    Removing stm32f1xx_hal_rcc.o(i.HAL_RCC_GetOscConfig), (212 bytes).
    Removing stm32f1xx_hal_rcc.o(i.HAL_RCC_GetPCLK1Freq), (44 bytes).
    Removing stm32f1xx_hal_rcc.o(i.HAL_RCC_GetPCLK2Freq), (44 bytes).
    Removing stm32f1xx_hal_rcc.o(i.HAL_RCC_MCOConfig), (100 bytes).
    Removing stm32f1xx_hal_rcc.o(i.HAL_RCC_NMI_IRQHandler), (32 bytes).
    Removing stm32f1xx_hal_rcc.o(i.HAL_RCC_OscConfig), (2440 bytes).
    Removing stm32f1xx_hal_rcc_ex.o(.rev16_text), (4 bytes).
    Removing stm32f1xx_hal_rcc_ex.o(.revsh_text), (4 bytes).
    Removing stm32f1xx_hal_rcc_ex.o(i.HAL_RCCEx_GetPeriphCLKConfig), (84 bytes).
    Removing stm32f1xx_hal_rcc_ex.o(i.HAL_RCCEx_GetPeriphCLKFreq), (360 bytes).
    Removing stm32f1xx_hal_rcc_ex.o(i.HAL_RCCEx_PeriphCLKConfig), (372 bytes).
    Removing stm32f1xx_hal_rtc.o(.rev16_text), (4 bytes).
    Removing stm32f1xx_hal_rtc.o(.revsh_text), (4 bytes).
    Removing stm32f1xx_hal_rtc_ex.o(.rev16_text), (4 bytes).
    Removing stm32f1xx_hal_rtc_ex.o(.revsh_text), (4 bytes).
    Removing stm32f1xx_hal_sd.o(.rev16_text), (4 bytes).
    Removing stm32f1xx_hal_sd.o(.revsh_text), (4 bytes).
    Removing stm32f1xx_hal_smartcard.o(.rev16_text), (4 bytes).
    Removing stm32f1xx_hal_smartcard.o(.revsh_text), (4 bytes).
    Removing stm32f1xx_hal_spi.o(.rev16_text), (4 bytes).
    Removing stm32f1xx_hal_spi.o(.revsh_text), (4 bytes).
    Removing stm32f1xx_hal_spi_ex.o(.rev16_text), (4 bytes).
    Removing stm32f1xx_hal_spi_ex.o(.revsh_text), (4 bytes).
    Removing stm32f1xx_hal_sram.o(.rev16_text), (4 bytes).
    Removing stm32f1xx_hal_sram.o(.revsh_text), (4 bytes).
    Removing stm32f1xx_hal_tim.o(.rev16_text), (4 bytes).
    Removing stm32f1xx_hal_tim.o(.revsh_text), (4 bytes).
    Removing stm32f1xx_hal_tim_ex.o(.rev16_text), (4 bytes).
    Removing stm32f1xx_hal_tim_ex.o(.revsh_text), (4 bytes).
    Removing stm32f1xx_hal_uart.o(.rev16_text), (4 bytes).
    Removing stm32f1xx_hal_uart.o(.revsh_text), (4 bytes).
    Removing stm32f1xx_hal_usart.o(.rev16_text), (4 bytes).
    Removing stm32f1xx_hal_usart.o(.revsh_text), (4 bytes).
    Removing stm32f1xx_hal_wwdg.o(.rev16_text), (4 bytes).
    Removing stm32f1xx_hal_wwdg.o(.revsh_text), (4 bytes).
    Removing stm32f1xx_ll_fsmc.o(.rev16_text), (4 bytes).
    Removing stm32f1xx_ll_fsmc.o(.revsh_text), (4 bytes).
    Removing stm32f1xx_ll_sdmmc.o(.rev16_text), (4 bytes).
    Removing stm32f1xx_ll_sdmmc.o(.revsh_text), (4 bytes).
    Removing stm32f1xx_ll_usb.o(.rev16_text), (4 bytes).
    Removing stm32f1xx_ll_usb.o(.revsh_text), (4 bytes).
    Removing stm32f1xx_hal_msp.o(.rev16_text), (4 bytes).
    Removing stm32f1xx_hal_msp.o(.revsh_text), (4 bytes).
    Removing stm32f1xx_hal_msp.o(i.HAL_IWDG_MspInit), (2 bytes).
    Removing stm32f1xx_hal_msp.o(i.HAL_MspInit), (52 bytes).
    Removing stm32f1xx_it.o(.rev16_text), (4 bytes).
    Removing stm32f1xx_it.o(.revsh_text), (4 bytes).

261 unused section(s) (total 19526 bytes) removed from the image.

==============================================================================

Image Symbol Table

    Local Symbols

    Symbol Name                              Value     Ov Type        Size  Object(Section)

    ../clib/angel/boardlib.s                 0x00000000   Number         0  boardinit3.o ABSOLUTE
    ../clib/angel/boardlib.s                 0x00000000   Number         0  boardinit2.o ABSOLUTE
    ../clib/angel/boardlib.s                 0x00000000   Number         0  boardinit1.o ABSOLUTE
    ../clib/angel/boardlib.s                 0x00000000   Number         0  boardshut.o ABSOLUTE
    ../clib/angel/dczerorl2.s                0x00000000   Number         0  __dczerorl2.o ABSOLUTE
    ../clib/angel/handlers.s                 0x00000000   Number         0  __scatter_zi.o ABSOLUTE
    ../clib/angel/kernel.s                   0x00000000   Number         0  rtexit.o ABSOLUTE
    ../clib/angel/kernel.s                   0x00000000   Number         0  __rtentry4.o ABSOLUTE
    ../clib/angel/kernel.s                   0x00000000   Number         0  __rtentry2.o ABSOLUTE
    ../clib/angel/kernel.s                   0x00000000   Number         0  __rtentry.o ABSOLUTE
    ../clib/angel/kernel.s                   0x00000000   Number         0  rtexit2.o ABSOLUTE
    ../clib/angel/rt.s                       0x00000000   Number         0  rt_raise.o ABSOLUTE
    ../clib/angel/scatter.s                  0x00000000   Number         0  __scatter.o ABSOLUTE
    ../clib/angel/startup.s                  0x00000000   Number         0  __main.o ABSOLUTE
    ../clib/angel/sys.s                      0x00000000   Number         0  sys_stackheap_outer.o ABSOLUTE
    ../clib/angel/sys.s                      0x00000000   Number         0  libspace.o ABSOLUTE
    ../clib/angel/sys.s                      0x00000000   Number         0  use_no_semi.o ABSOLUTE
    ../clib/angel/sys.s                      0x00000000   Number         0  indicate_semi.o ABSOLUTE
    ../clib/angel/sysapp.c                   0x00000000   Number         0  sys_command.o ABSOLUTE
    ../clib/angel/sysapp.c                   0x00000000   Number         0  sys_wrch.o ABSOLUTE
    ../clib/angel/sysapp.c                   0x00000000   Number         0  sys_exit.o ABSOLUTE
    ../clib/armsys.c                         0x00000000   Number         0  no_argv.o ABSOLUTE
    ../clib/armsys.c                         0x00000000   Number         0  _get_argv_nomalloc.o ABSOLUTE
    ../clib/armsys.c                         0x00000000   Number         0  argv_veneer.o ABSOLUTE
    ../clib/armsys.c                         0x00000000   Number         0  argv_veneer.o ABSOLUTE
    ../clib/heapalloc.c                      0x00000000   Number         0  hrguard.o ABSOLUTE
    ../clib/heapaux.c                        0x00000000   Number         0  heapauxi.o ABSOLUTE
    ../clib/libinit.s                        0x00000000   Number         0  libinit2.o ABSOLUTE
    ../clib/libinit.s                        0x00000000   Number         0  libinit.o ABSOLUTE
    ../clib/libinit.s                        0x00000000   Number         0  libshutdown.o ABSOLUTE
    ../clib/libinit.s                        0x00000000   Number         0  libshutdown2.o ABSOLUTE
    ../clib/longlong.s                       0x00000000   Number         0  llushr.o ABSOLUTE
    ../clib/signal.c                         0x00000000   Number         0  defsig_rtmem_formal.o ABSOLUTE
    ../clib/signal.c                         0x00000000   Number         0  defsig_rtmem_outer.o ABSOLUTE
    ../clib/signal.c                         0x00000000   Number         0  defsig_segv_inner.o ABSOLUTE
    ../clib/signal.c                         0x00000000   Number         0  defsig_rtmem_inner.o ABSOLUTE
    ../clib/signal.c                         0x00000000   Number         0  defsig_other.o ABSOLUTE
    ../clib/signal.c                         0x00000000   Number         0  defsig_cppl_inner.o ABSOLUTE
    ../clib/signal.c                         0x00000000   Number         0  defsig_pvfn_inner.o ABSOLUTE
    ../clib/signal.c                         0x00000000   Number         0  defsig_stak_inner.o ABSOLUTE
    ../clib/signal.c                         0x00000000   Number         0  defsig_rtred_inner.o ABSOLUTE
    ../clib/signal.c                         0x00000000   Number         0  defsig_fpe_inner.o ABSOLUTE
    ../clib/signal.c                         0x00000000   Number         0  defsig_abrt_inner.o ABSOLUTE
    ../clib/signal.c                         0x00000000   Number         0  defsig_exit.o ABSOLUTE
    ../clib/signal.c                         0x00000000   Number         0  defsig_general.o ABSOLUTE
    ../clib/signal.c                         0x00000000   Number         0  __raise.o ABSOLUTE
    ../clib/signal.s                         0x00000000   Number         0  defsig.o ABSOLUTE
    ../clib/stdlib.c                         0x00000000   Number         0  exit.o ABSOLUTE
    ../fplib/dfixu.s                         0x00000000   Number         0  dfixu.o ABSOLUTE
    ../fplib/dflt.s                          0x00000000   Number         0  dflt_clz.o ABSOLUTE
    ../fplib/dmul.s                          0x00000000   Number         0  dmul.o ABSOLUTE
    ../fplib/dnaninf.s                       0x00000000   Number         0  dnaninf.o ABSOLUTE
    ../fplib/dretinf.s                       0x00000000   Number         0  dretinf.o ABSOLUTE
    ../fplib/fpinit.s                        0x00000000   Number         0  fpinit.o ABSOLUTE
    ../fplib/usenofp.s                       0x00000000   Number         0  usenofp.o ABSOLUTE
    app\app_cfg.c                            0x00000000   Number         0  app_cfg.o ABSOLUTE
    app\app_int_cfg.c                        0x00000000   Number         0  app_int_cfg.o ABSOLUTE
    app\demo.c                               0x00000000   Number         0  demo.o ABSOLUTE
    app\hook.c                               0x00000000   Number         0  hook.o ABSOLUTE
    bsp\\hardware_init.c                     0x00000000   Number         0  hardware_init.o ABSOLUTE
    bsp\\system_stm32f1xx.c                  0x00000000   Number         0  system_stm32f1xx.o ABSOLUTE
    bsp\chip_uip_interrupt.c                 0x00000000   Number         0  chip_uip_interrupt.o ABSOLUTE
    bsp\hardware_init.c                      0x00000000   Number         0  hardware_init.o ABSOLUTE
    bsp\system_stm32f1xx.c                   0x00000000   Number         0  system_stm32f1xx.o ABSOLUTE
    dc.s                                     0x00000000   Number         0  dc.o ABSOLUTE
    startup\\system_stm32f10x_cl.c           0x00000000   Number         0  system_stm32f10x_cl.o ABSOLUTE
    startup\startup_stm32f10x_hd.s           0x00000000   Number         0  startup_stm32f10x_hd.o ABSOLUTE
    startup\system_stm32f10x_cl.c            0x00000000   Number         0  system_stm32f10x_cl.o ABSOLUTE
    stm32f1xx_hal_driver\\src\\stm32f1xx_hal.c 0x00000000   Number         0  stm32f1xx_hal.o ABSOLUTE
    stm32f1xx_hal_driver\\src\\stm32f1xx_hal_adc.c 0x00000000   Number         0  stm32f1xx_hal_adc.o ABSOLUTE
    stm32f1xx_hal_driver\\src\\stm32f1xx_hal_adc_ex.c 0x00000000   Number         0  stm32f1xx_hal_adc_ex.o ABSOLUTE
    stm32f1xx_hal_driver\\src\\stm32f1xx_hal_can.c 0x00000000   Number         0  stm32f1xx_hal_can.o ABSOLUTE
    stm32f1xx_hal_driver\\src\\stm32f1xx_hal_cec.c 0x00000000   Number         0  stm32f1xx_hal_cec.o ABSOLUTE
    stm32f1xx_hal_driver\\src\\stm32f1xx_hal_cortex.c 0x00000000   Number         0  stm32f1xx_hal_cortex.o ABSOLUTE
    stm32f1xx_hal_driver\\src\\stm32f1xx_hal_crc.c 0x00000000   Number         0  stm32f1xx_hal_crc.o ABSOLUTE
    stm32f1xx_hal_driver\\src\\stm32f1xx_hal_dac.c 0x00000000   Number         0  stm32f1xx_hal_dac.o ABSOLUTE
    stm32f1xx_hal_driver\\src\\stm32f1xx_hal_dac_ex.c 0x00000000   Number         0  stm32f1xx_hal_dac_ex.o ABSOLUTE
    stm32f1xx_hal_driver\\src\\stm32f1xx_hal_dma.c 0x00000000   Number         0  stm32f1xx_hal_dma.o ABSOLUTE
    stm32f1xx_hal_driver\\src\\stm32f1xx_hal_eth.c 0x00000000   Number         0  stm32f1xx_hal_eth.o ABSOLUTE
    stm32f1xx_hal_driver\\src\\stm32f1xx_hal_flash.c 0x00000000   Number         0  stm32f1xx_hal_flash.o ABSOLUTE
    stm32f1xx_hal_driver\\src\\stm32f1xx_hal_flash_ex.c 0x00000000   Number         0  stm32f1xx_hal_flash_ex.o ABSOLUTE
    stm32f1xx_hal_driver\\src\\stm32f1xx_hal_gpio.c 0x00000000   Number         0  stm32f1xx_hal_gpio.o ABSOLUTE
    stm32f1xx_hal_driver\\src\\stm32f1xx_hal_gpio_ex.c 0x00000000   Number         0  stm32f1xx_hal_gpio_ex.o ABSOLUTE
    stm32f1xx_hal_driver\\src\\stm32f1xx_hal_hcd.c 0x00000000   Number         0  stm32f1xx_hal_hcd.o ABSOLUTE
    stm32f1xx_hal_driver\\src\\stm32f1xx_hal_i2c.c 0x00000000   Number         0  stm32f1xx_hal_i2c.o ABSOLUTE
    stm32f1xx_hal_driver\\src\\stm32f1xx_hal_i2s.c 0x00000000   Number         0  stm32f1xx_hal_i2s.o ABSOLUTE
    stm32f1xx_hal_driver\\src\\stm32f1xx_hal_irda.c 0x00000000   Number         0  stm32f1xx_hal_irda.o ABSOLUTE
    stm32f1xx_hal_driver\\src\\stm32f1xx_hal_iwdg.c 0x00000000   Number         0  stm32f1xx_hal_iwdg.o ABSOLUTE
    stm32f1xx_hal_driver\\src\\stm32f1xx_hal_msp.c 0x00000000   Number         0  stm32f1xx_hal_msp.o ABSOLUTE
    stm32f1xx_hal_driver\\src\\stm32f1xx_hal_nand.c 0x00000000   Number         0  stm32f1xx_hal_nand.o ABSOLUTE
    stm32f1xx_hal_driver\\src\\stm32f1xx_hal_nor.c 0x00000000   Number         0  stm32f1xx_hal_nor.o ABSOLUTE
    stm32f1xx_hal_driver\\src\\stm32f1xx_hal_pccard.c 0x00000000   Number         0  stm32f1xx_hal_pccard.o ABSOLUTE
    stm32f1xx_hal_driver\\src\\stm32f1xx_hal_pcd.c 0x00000000   Number         0  stm32f1xx_hal_pcd.o ABSOLUTE
    stm32f1xx_hal_driver\\src\\stm32f1xx_hal_pcd_ex.c 0x00000000   Number         0  stm32f1xx_hal_pcd_ex.o ABSOLUTE
    stm32f1xx_hal_driver\\src\\stm32f1xx_hal_pwr.c 0x00000000   Number         0  stm32f1xx_hal_pwr.o ABSOLUTE
    stm32f1xx_hal_driver\\src\\stm32f1xx_hal_rcc.c 0x00000000   Number         0  stm32f1xx_hal_rcc.o ABSOLUTE
    stm32f1xx_hal_driver\\src\\stm32f1xx_hal_rcc_ex.c 0x00000000   Number         0  stm32f1xx_hal_rcc_ex.o ABSOLUTE
    stm32f1xx_hal_driver\\src\\stm32f1xx_hal_rtc.c 0x00000000   Number         0  stm32f1xx_hal_rtc.o ABSOLUTE
    stm32f1xx_hal_driver\\src\\stm32f1xx_hal_rtc_ex.c 0x00000000   Number         0  stm32f1xx_hal_rtc_ex.o ABSOLUTE
    stm32f1xx_hal_driver\\src\\stm32f1xx_hal_sd.c 0x00000000   Number         0  stm32f1xx_hal_sd.o ABSOLUTE
    stm32f1xx_hal_driver\\src\\stm32f1xx_hal_smartcard.c 0x00000000   Number         0  stm32f1xx_hal_smartcard.o ABSOLUTE
    stm32f1xx_hal_driver\\src\\stm32f1xx_hal_spi.c 0x00000000   Number         0  stm32f1xx_hal_spi.o ABSOLUTE
    stm32f1xx_hal_driver\\src\\stm32f1xx_hal_spi_ex.c 0x00000000   Number         0  stm32f1xx_hal_spi_ex.o ABSOLUTE
    stm32f1xx_hal_driver\\src\\stm32f1xx_hal_sram.c 0x00000000   Number         0  stm32f1xx_hal_sram.o ABSOLUTE
    stm32f1xx_hal_driver\\src\\stm32f1xx_hal_tim.c 0x00000000   Number         0  stm32f1xx_hal_tim.o ABSOLUTE
    stm32f1xx_hal_driver\\src\\stm32f1xx_hal_tim_ex.c 0x00000000   Number         0  stm32f1xx_hal_tim_ex.o ABSOLUTE
    stm32f1xx_hal_driver\\src\\stm32f1xx_hal_uart.c 0x00000000   Number         0  stm32f1xx_hal_uart.o ABSOLUTE
    stm32f1xx_hal_driver\\src\\stm32f1xx_hal_usart.c 0x00000000   Number         0  stm32f1xx_hal_usart.o ABSOLUTE
    stm32f1xx_hal_driver\\src\\stm32f1xx_hal_wwdg.c 0x00000000   Number         0  stm32f1xx_hal_wwdg.o ABSOLUTE
    stm32f1xx_hal_driver\\src\\stm32f1xx_it.c 0x00000000   Number         0  stm32f1xx_it.o ABSOLUTE
    stm32f1xx_hal_driver\\src\\stm32f1xx_ll_fsmc.c 0x00000000   Number         0  stm32f1xx_ll_fsmc.o ABSOLUTE
    stm32f1xx_hal_driver\\src\\stm32f1xx_ll_sdmmc.c 0x00000000   Number         0  stm32f1xx_ll_sdmmc.o ABSOLUTE
    stm32f1xx_hal_driver\\src\\stm32f1xx_ll_usb.c 0x00000000   Number         0  stm32f1xx_ll_usb.o ABSOLUTE
    stm32f1xx_hal_driver\src\stm32f1xx_hal.c 0x00000000   Number         0  stm32f1xx_hal.o ABSOLUTE
    stm32f1xx_hal_driver\src\stm32f1xx_hal_adc.c 0x00000000   Number         0  stm32f1xx_hal_adc.o ABSOLUTE
    stm32f1xx_hal_driver\src\stm32f1xx_hal_adc_ex.c 0x00000000   Number         0  stm32f1xx_hal_adc_ex.o ABSOLUTE
    stm32f1xx_hal_driver\src\stm32f1xx_hal_can.c 0x00000000   Number         0  stm32f1xx_hal_can.o ABSOLUTE
    stm32f1xx_hal_driver\src\stm32f1xx_hal_cec.c 0x00000000   Number         0  stm32f1xx_hal_cec.o ABSOLUTE
    stm32f1xx_hal_driver\src\stm32f1xx_hal_cortex.c 0x00000000   Number         0  stm32f1xx_hal_cortex.o ABSOLUTE
    stm32f1xx_hal_driver\src\stm32f1xx_hal_crc.c 0x00000000   Number         0  stm32f1xx_hal_crc.o ABSOLUTE
    stm32f1xx_hal_driver\src\stm32f1xx_hal_dac.c 0x00000000   Number         0  stm32f1xx_hal_dac.o ABSOLUTE
    stm32f1xx_hal_driver\src\stm32f1xx_hal_dac_ex.c 0x00000000   Number         0  stm32f1xx_hal_dac_ex.o ABSOLUTE
    stm32f1xx_hal_driver\src\stm32f1xx_hal_dma.c 0x00000000   Number         0  stm32f1xx_hal_dma.o ABSOLUTE
    stm32f1xx_hal_driver\src\stm32f1xx_hal_eth.c 0x00000000   Number         0  stm32f1xx_hal_eth.o ABSOLUTE
    stm32f1xx_hal_driver\src\stm32f1xx_hal_flash.c 0x00000000   Number         0  stm32f1xx_hal_flash.o ABSOLUTE
    stm32f1xx_hal_driver\src\stm32f1xx_hal_flash_ex.c 0x00000000   Number         0  stm32f1xx_hal_flash_ex.o ABSOLUTE
    stm32f1xx_hal_driver\src\stm32f1xx_hal_gpio.c 0x00000000   Number         0  stm32f1xx_hal_gpio.o ABSOLUTE
    stm32f1xx_hal_driver\src\stm32f1xx_hal_gpio_ex.c 0x00000000   Number         0  stm32f1xx_hal_gpio_ex.o ABSOLUTE
    stm32f1xx_hal_driver\src\stm32f1xx_hal_hcd.c 0x00000000   Number         0  stm32f1xx_hal_hcd.o ABSOLUTE
    stm32f1xx_hal_driver\src\stm32f1xx_hal_i2c.c 0x00000000   Number         0  stm32f1xx_hal_i2c.o ABSOLUTE
    stm32f1xx_hal_driver\src\stm32f1xx_hal_i2s.c 0x00000000   Number         0  stm32f1xx_hal_i2s.o ABSOLUTE
    stm32f1xx_hal_driver\src\stm32f1xx_hal_irda.c 0x00000000   Number         0  stm32f1xx_hal_irda.o ABSOLUTE
    stm32f1xx_hal_driver\src\stm32f1xx_hal_iwdg.c 0x00000000   Number         0  stm32f1xx_hal_iwdg.o ABSOLUTE
    stm32f1xx_hal_driver\src\stm32f1xx_hal_msp.c 0x00000000   Number         0  stm32f1xx_hal_msp.o ABSOLUTE
    stm32f1xx_hal_driver\src\stm32f1xx_hal_nand.c 0x00000000   Number         0  stm32f1xx_hal_nand.o ABSOLUTE
    stm32f1xx_hal_driver\src\stm32f1xx_hal_nor.c 0x00000000   Number         0  stm32f1xx_hal_nor.o ABSOLUTE
    stm32f1xx_hal_driver\src\stm32f1xx_hal_pccard.c 0x00000000   Number         0  stm32f1xx_hal_pccard.o ABSOLUTE
    stm32f1xx_hal_driver\src\stm32f1xx_hal_pcd.c 0x00000000   Number         0  stm32f1xx_hal_pcd.o ABSOLUTE
    stm32f1xx_hal_driver\src\stm32f1xx_hal_pcd_ex.c 0x00000000   Number         0  stm32f1xx_hal_pcd_ex.o ABSOLUTE
    stm32f1xx_hal_driver\src\stm32f1xx_hal_pwr.c 0x00000000   Number         0  stm32f1xx_hal_pwr.o ABSOLUTE
    stm32f1xx_hal_driver\src\stm32f1xx_hal_rcc.c 0x00000000   Number         0  stm32f1xx_hal_rcc.o ABSOLUTE
    stm32f1xx_hal_driver\src\stm32f1xx_hal_rcc_ex.c 0x00000000   Number         0  stm32f1xx_hal_rcc_ex.o ABSOLUTE
    stm32f1xx_hal_driver\src\stm32f1xx_hal_rtc.c 0x00000000   Number         0  stm32f1xx_hal_rtc.o ABSOLUTE
    stm32f1xx_hal_driver\src\stm32f1xx_hal_rtc_ex.c 0x00000000   Number         0  stm32f1xx_hal_rtc_ex.o ABSOLUTE
    stm32f1xx_hal_driver\src\stm32f1xx_hal_sd.c 0x00000000   Number         0  stm32f1xx_hal_sd.o ABSOLUTE
    stm32f1xx_hal_driver\src\stm32f1xx_hal_smartcard.c 0x00000000   Number         0  stm32f1xx_hal_smartcard.o ABSOLUTE
    stm32f1xx_hal_driver\src\stm32f1xx_hal_spi.c 0x00000000   Number         0  stm32f1xx_hal_spi.o ABSOLUTE
    stm32f1xx_hal_driver\src\stm32f1xx_hal_spi_ex.c 0x00000000   Number         0  stm32f1xx_hal_spi_ex.o ABSOLUTE
    stm32f1xx_hal_driver\src\stm32f1xx_hal_sram.c 0x00000000   Number         0  stm32f1xx_hal_sram.o ABSOLUTE
    stm32f1xx_hal_driver\src\stm32f1xx_hal_tim.c 0x00000000   Number         0  stm32f1xx_hal_tim.o ABSOLUTE
    stm32f1xx_hal_driver\src\stm32f1xx_hal_tim_ex.c 0x00000000   Number         0  stm32f1xx_hal_tim_ex.o ABSOLUTE
    stm32f1xx_hal_driver\src\stm32f1xx_hal_uart.c 0x00000000   Number         0  stm32f1xx_hal_uart.o ABSOLUTE
    stm32f1xx_hal_driver\src\stm32f1xx_hal_usart.c 0x00000000   Number         0  stm32f1xx_hal_usart.o ABSOLUTE
    stm32f1xx_hal_driver\src\stm32f1xx_hal_wwdg.c 0x00000000   Number         0  stm32f1xx_hal_wwdg.o ABSOLUTE
    stm32f1xx_hal_driver\src\stm32f1xx_it.c  0x00000000   Number         0  stm32f1xx_it.o ABSOLUTE
    stm32f1xx_hal_driver\src\stm32f1xx_ll_fsmc.c 0x00000000   Number         0  stm32f1xx_ll_fsmc.o ABSOLUTE
    stm32f1xx_hal_driver\src\stm32f1xx_ll_sdmmc.c 0x00000000   Number         0  stm32f1xx_ll_sdmmc.o ABSOLUTE
    stm32f1xx_hal_driver\src\stm32f1xx_ll_usb.c 0x00000000   Number         0  stm32f1xx_ll_usb.o ABSOLUTE
    uipkernel\uip_kernel_common.c            0x00000000   Number         0  uip_kernel_common.o ABSOLUTE
    uipkernel\uip_kernel_event.c             0x00000000   Number         0  uip_kernel_event.o ABSOLUTE
    uipkernel\uip_kernel_isr_cm.s            0x00000000   Number         0  uip_kernel_isr_cm.o ABSOLUTE
    uipkernel\uip_kernel_isr_engine.c        0x00000000   Number         0  uip_kernel_isr_engine.o ABSOLUTE
    uipkernel\uip_kernel_message.c           0x00000000   Number         0  uip_kernel_message.o ABSOLUTE
    uipkernel\uip_kernel_resource.c          0x00000000   Number         0  uip_kernel_resource.o ABSOLUTE
    uipkernel\uip_kernel_scheduler.c         0x00000000   Number         0  uip_kernel_scheduler.o ABSOLUTE
    uipkernel\uip_kernel_task.c              0x00000000   Number         0  uip_kernel_task.o ABSOLUTE
    uipkernel\uip_kernel_time.c              0x00000000   Number         0  uip_kernel_time.o ABSOLUTE
    RESET                                    0x08000000   Section      304  startup_stm32f10x_hd.o(RESET)
    !!!main                                  0x08000130   Section        8  __main.o(!!!main)
    !!!scatter                               0x08000138   Section       52  __scatter.o(!!!scatter)
    !!dczerorl2                              0x0800016c   Section       90  __dczerorl2.o(!!dczerorl2)
    !!handler_zi                             0x080001c8   Section       28  __scatter_zi.o(!!handler_zi)
    .ARM.Collect$$libinit$$00000000          0x080001e4   Section        2  libinit.o(.ARM.Collect$$libinit$$00000000)
    .ARM.Collect$$libinit$$00000002          0x080001e6   Section        0  libinit2.o(.ARM.Collect$$libinit$$00000002)
    .ARM.Collect$$libinit$$00000004          0x080001e6   Section        0  libinit2.o(.ARM.Collect$$libinit$$00000004)
    .ARM.Collect$$libinit$$0000000A          0x080001e6   Section        0  libinit2.o(.ARM.Collect$$libinit$$0000000A)
    .ARM.Collect$$libinit$$0000000C          0x080001e6   Section        0  libinit2.o(.ARM.Collect$$libinit$$0000000C)
    .ARM.Collect$$libinit$$0000000E          0x080001e6   Section        0  libinit2.o(.ARM.Collect$$libinit$$0000000E)
    .ARM.Collect$$libinit$$00000011          0x080001e6   Section        0  libinit2.o(.ARM.Collect$$libinit$$00000011)
    .ARM.Collect$$libinit$$00000013          0x080001e6   Section        0  libinit2.o(.ARM.Collect$$libinit$$00000013)
    .ARM.Collect$$libinit$$00000015          0x080001e6   Section        0  libinit2.o(.ARM.Collect$$libinit$$00000015)
    .ARM.Collect$$libinit$$00000017          0x080001e6   Section        0  libinit2.o(.ARM.Collect$$libinit$$00000017)
    .ARM.Collect$$libinit$$00000019          0x080001e6   Section        0  libinit2.o(.ARM.Collect$$libinit$$00000019)
    .ARM.Collect$$libinit$$0000001B          0x080001e6   Section        0  libinit2.o(.ARM.Collect$$libinit$$0000001B)
    .ARM.Collect$$libinit$$0000001D          0x080001e6   Section        0  libinit2.o(.ARM.Collect$$libinit$$0000001D)
    .ARM.Collect$$libinit$$0000001F          0x080001e6   Section        0  libinit2.o(.ARM.Collect$$libinit$$0000001F)
    .ARM.Collect$$libinit$$00000021          0x080001e6   Section        0  libinit2.o(.ARM.Collect$$libinit$$00000021)
    .ARM.Collect$$libinit$$00000023          0x080001e6   Section        0  libinit2.o(.ARM.Collect$$libinit$$00000023)
    .ARM.Collect$$libinit$$00000025          0x080001e6   Section        0  libinit2.o(.ARM.Collect$$libinit$$00000025)
    .ARM.Collect$$libinit$$0000002C          0x080001e6   Section        0  libinit2.o(.ARM.Collect$$libinit$$0000002C)
    .ARM.Collect$$libinit$$0000002E          0x080001e6   Section        0  libinit2.o(.ARM.Collect$$libinit$$0000002E)
    .ARM.Collect$$libinit$$00000030          0x080001e6   Section        0  libinit2.o(.ARM.Collect$$libinit$$00000030)
    .ARM.Collect$$libinit$$00000032          0x080001e6   Section        0  libinit2.o(.ARM.Collect$$libinit$$00000032)
    .ARM.Collect$$libinit$$00000033          0x080001e6   Section        2  libinit2.o(.ARM.Collect$$libinit$$00000033)
    .ARM.Collect$$libshutdown$$00000000      0x080001e8   Section        2  libshutdown.o(.ARM.Collect$$libshutdown$$00000000)
    .ARM.Collect$$libshutdown$$00000002      0x080001ea   Section        0  libshutdown2.o(.ARM.Collect$$libshutdown$$00000002)
    .ARM.Collect$$libshutdown$$00000004      0x080001ea   Section        0  libshutdown2.o(.ARM.Collect$$libshutdown$$00000004)
    .ARM.Collect$$libshutdown$$00000007      0x080001ea   Section        0  libshutdown2.o(.ARM.Collect$$libshutdown$$00000007)
    .ARM.Collect$$libshutdown$$0000000A      0x080001ea   Section        0  libshutdown2.o(.ARM.Collect$$libshutdown$$0000000A)
    .ARM.Collect$$libshutdown$$0000000C      0x080001ea   Section        0  libshutdown2.o(.ARM.Collect$$libshutdown$$0000000C)
    .ARM.Collect$$libshutdown$$0000000F      0x080001ea   Section        0  libshutdown2.o(.ARM.Collect$$libshutdown$$0000000F)
    .ARM.Collect$$libshutdown$$00000010      0x080001ea   Section        2  libshutdown2.o(.ARM.Collect$$libshutdown$$00000010)
    .ARM.Collect$$rtentry$$00000000          0x080001ec   Section        0  __rtentry.o(.ARM.Collect$$rtentry$$00000000)
    .ARM.Collect$$rtentry$$00000002          0x080001ec   Section        0  __rtentry2.o(.ARM.Collect$$rtentry$$00000002)
    .ARM.Collect$$rtentry$$00000004          0x080001ec   Section        6  __rtentry4.o(.ARM.Collect$$rtentry$$00000004)
    .ARM.Collect$$rtentry$$00000009          0x080001f2   Section        0  __rtentry2.o(.ARM.Collect$$rtentry$$00000009)
    .ARM.Collect$$rtentry$$0000000A          0x080001f2   Section        4  __rtentry2.o(.ARM.Collect$$rtentry$$0000000A)
    .ARM.Collect$$rtentry$$0000000C          0x080001f6   Section        0  __rtentry2.o(.ARM.Collect$$rtentry$$0000000C)
    .ARM.Collect$$rtentry$$0000000D          0x080001f6   Section        8  __rtentry2.o(.ARM.Collect$$rtentry$$0000000D)
    .ARM.Collect$$rtexit$$00000000           0x080001fe   Section        2  rtexit.o(.ARM.Collect$$rtexit$$00000000)
    .ARM.Collect$$rtexit$$00000002           0x08000200   Section        0  rtexit2.o(.ARM.Collect$$rtexit$$00000002)
    .ARM.Collect$$rtexit$$00000003           0x08000200   Section        4  rtexit2.o(.ARM.Collect$$rtexit$$00000003)
    .ARM.Collect$$rtexit$$00000004           0x08000204   Section        6  rtexit2.o(.ARM.Collect$$rtexit$$00000004)
    .text                                    0x0800020c   Section       60  startup_stm32f10x_hd.o(.text)
    .text                                    0x08000248   Section        0  heapauxi.o(.text)
    .text                                    0x0800024e   Section       74  sys_stackheap_outer.o(.text)
    .text                                    0x08000298   Section        0  exit.o(.text)
    .text                                    0x080002ac   Section        8  libspace.o(.text)
    .text                                    0x080002b4   Section        0  sys_exit.o(.text)
    .text                                    0x080002c0   Section        2  use_no_semi.o(.text)
    .text                                    0x080002c2   Section        0  indicate_semi.o(.text)
    CODE                                     0x080002c4   Section       72  uip_kernel_isr_cm.o(CODE)
    i.ADC1_2_IRQHandler                      0x0800030c   Section        0  chip_uip_interrupt.o(i.ADC1_2_IRQHandler)
    i.ADC3_IRQHandler                        0x08000320   Section        0  chip_uip_interrupt.o(i.ADC3_IRQHandler)
    i.AppIdleTask                            0x08000334   Section        0  demo.o(i.AppIdleTask)
    i.CAN1_RX1_IRQHandler                    0x08000364   Section        0  chip_uip_interrupt.o(i.CAN1_RX1_IRQHandler)
    i.CAN1_SCE_IRQHandler                    0x08000378   Section        0  chip_uip_interrupt.o(i.CAN1_SCE_IRQHandler)
    i.Chip_UIP_InterruptInit                 0x0800038c   Section        0  chip_uip_interrupt.o(i.Chip_UIP_InterruptInit)
    i.Chip_UIP_InterruptNullHandler          0x080003b8   Section        0  chip_uip_interrupt.o(i.Chip_UIP_InterruptNullHandler)
    Chip_UIP_InterruptNullHandler            0x080003b9   Thumb Code     4  chip_uip_interrupt.o(i.Chip_UIP_InterruptNullHandler)
    i.Chip_UIP_InterruptRegisterHandler      0x080003bc   Section        0  chip_uip_interrupt.o(i.Chip_UIP_InterruptRegisterHandler)
    i.DMA1_Channel1_IRQHandler               0x080003dc   Section        0  chip_uip_interrupt.o(i.DMA1_Channel1_IRQHandler)
    i.DMA1_Channel2_IRQHandler               0x080003f0   Section        0  chip_uip_interrupt.o(i.DMA1_Channel2_IRQHandler)
    i.DMA1_Channel3_IRQHandler               0x08000404   Section        0  chip_uip_interrupt.o(i.DMA1_Channel3_IRQHandler)
    i.DMA1_Channel4_IRQHandler               0x08000418   Section        0  chip_uip_interrupt.o(i.DMA1_Channel4_IRQHandler)
    i.DMA1_Channel5_IRQHandler               0x0800042c   Section        0  chip_uip_interrupt.o(i.DMA1_Channel5_IRQHandler)
    i.DMA1_Channel6_IRQHandler               0x08000440   Section        0  chip_uip_interrupt.o(i.DMA1_Channel6_IRQHandler)
    i.DMA1_Channel7_IRQHandler               0x08000454   Section        0  chip_uip_interrupt.o(i.DMA1_Channel7_IRQHandler)
    i.DMA2_Channel1_IRQHandler               0x08000468   Section        0  chip_uip_interrupt.o(i.DMA2_Channel1_IRQHandler)
    i.DMA2_Channel2_IRQHandler               0x0800047c   Section        0  chip_uip_interrupt.o(i.DMA2_Channel2_IRQHandler)
    i.DMA2_Channel3_IRQHandler               0x08000490   Section        0  chip_uip_interrupt.o(i.DMA2_Channel3_IRQHandler)
    i.DMA2_Channel4_5_IRQHandler             0x080004a4   Section        0  chip_uip_interrupt.o(i.DMA2_Channel4_5_IRQHandler)
    i.EXTI0_IRQHandler                       0x080004b8   Section        0  chip_uip_interrupt.o(i.EXTI0_IRQHandler)
    i.EXTI15_10_IRQHandler                   0x080004cc   Section        0  chip_uip_interrupt.o(i.EXTI15_10_IRQHandler)
    i.EXTI1_IRQHandler                       0x080004e0   Section        0  chip_uip_interrupt.o(i.EXTI1_IRQHandler)
    i.EXTI2_IRQHandler                       0x080004f4   Section        0  chip_uip_interrupt.o(i.EXTI2_IRQHandler)
    i.EXTI3_IRQHandler                       0x08000508   Section        0  chip_uip_interrupt.o(i.EXTI3_IRQHandler)
    i.EXTI4_IRQHandler                       0x0800051c   Section        0  chip_uip_interrupt.o(i.EXTI4_IRQHandler)
    i.EXTI9_5_IRQHandler                     0x08000530   Section        0  chip_uip_interrupt.o(i.EXTI9_5_IRQHandler)
    i.FLASH_IRQHandler                       0x08000544   Section        0  chip_uip_interrupt.o(i.FLASH_IRQHandler)
    i.FSMC_IRQHandler                        0x08000558   Section        0  chip_uip_interrupt.o(i.FSMC_IRQHandler)
    i.HAL_NVIC_SetPriority                   0x0800056c   Section        0  stm32f1xx_hal_cortex.o(i.HAL_NVIC_SetPriority)
    i.HAL_NVIC_SetPriorityGrouping           0x080005e8   Section        0  stm32f1xx_hal_cortex.o(i.HAL_NVIC_SetPriorityGrouping)
    i.HAL_RCC_GetHCLKFreq                    0x08000610   Section        0  stm32f1xx_hal_rcc.o(i.HAL_RCC_GetHCLKFreq)
    i.HAL_RCC_GetSysClockFreq                0x08000648   Section        0  stm32f1xx_hal_rcc.o(i.HAL_RCC_GetSysClockFreq)
    i.HAL_SYSTICK_CLKSourceConfig            0x08000700   Section        0  stm32f1xx_hal_cortex.o(i.HAL_SYSTICK_CLKSourceConfig)
    i.HAL_SYSTICK_Config                     0x08000728   Section        0  stm32f1xx_hal_cortex.o(i.HAL_SYSTICK_Config)
    i.Hardware_Init                          0x0800075c   Section        0  hardware_init.o(i.Hardware_Init)
    i.I2C1_ER_IRQHandler                     0x0800079c   Section        0  chip_uip_interrupt.o(i.I2C1_ER_IRQHandler)
    i.I2C1_EV_IRQHandler                     0x080007b0   Section        0  chip_uip_interrupt.o(i.I2C1_EV_IRQHandler)
    i.I2C2_ER_IRQHandler                     0x080007c4   Section        0  chip_uip_interrupt.o(i.I2C2_ER_IRQHandler)
    i.I2C2_EV_IRQHandler                     0x080007d8   Section        0  chip_uip_interrupt.o(i.I2C2_EV_IRQHandler)
    i.InterruptHandler                       0x080007ec   Section        0  chip_uip_interrupt.o(i.InterruptHandler)
    i.Kernel_System_Tick_Init                0x08000848   Section        0  hardware_init.o(i.Kernel_System_Tick_Init)
    i.NVIC_GetPriorityGrouping               0x08000880   Section        0  stm32f1xx_hal_cortex.o(i.NVIC_GetPriorityGrouping)
    NVIC_GetPriorityGrouping                 0x08000881   Thumb Code    10  stm32f1xx_hal_cortex.o(i.NVIC_GetPriorityGrouping)
    i.NVIC_SetPriority                       0x08000890   Section        0  stm32f1xx_hal_cortex.o(i.NVIC_SetPriority)
    NVIC_SetPriority                         0x08000891   Thumb Code    32  stm32f1xx_hal_cortex.o(i.NVIC_SetPriority)
    i.PVD_IRQHandler                         0x080008b8   Section        0  chip_uip_interrupt.o(i.PVD_IRQHandler)
    i.RCC_IRQHandler                         0x080008cc   Section        0  chip_uip_interrupt.o(i.RCC_IRQHandler)
    i.RTCAlarm_IRQHandler                    0x080008e0   Section        0  chip_uip_interrupt.o(i.RTCAlarm_IRQHandler)
    i.RTC_IRQHandler                         0x080008f4   Section        0  chip_uip_interrupt.o(i.RTC_IRQHandler)
    i.SDIO_IRQHandler                        0x08000908   Section        0  chip_uip_interrupt.o(i.SDIO_IRQHandler)
    i.SPI1_IRQHandler                        0x0800091c   Section        0  chip_uip_interrupt.o(i.SPI1_IRQHandler)
    i.SPI2_IRQHandler                        0x08000930   Section        0  chip_uip_interrupt.o(i.SPI2_IRQHandler)
    i.SPI3_IRQHandler                        0x08000944   Section        0  chip_uip_interrupt.o(i.SPI3_IRQHandler)
    i.StartOS                                0x08000958   Section        0  uip_kernel_common.o(i.StartOS)
    i.SystemInit                             0x08000988   Section        0  system_stm32f10x_cl.o(i.SystemInit)
    i.TAMPER_IRQHandler                      0x08000b44   Section        0  chip_uip_interrupt.o(i.TAMPER_IRQHandler)
    i.TASK_0                                 0x08000b58   Section        0  demo.o(i.TASK_0)
    i.TASK_1                                 0x08000b6e   Section        0  demo.o(i.TASK_1)
    i.TASK_2                                 0x08000b84   Section        0  demo.o(i.TASK_2)
    i.TASK_3                                 0x08000ba4   Section        0  demo.o(i.TASK_3)
    i.TASK_4                                 0x08000bbe   Section        0  demo.o(i.TASK_4)
    i.TIM1_BRK_IRQHandler                    0x08000bd0   Section        0  chip_uip_interrupt.o(i.TIM1_BRK_IRQHandler)
    i.TIM1_CC_IRQHandler                     0x08000be4   Section        0  chip_uip_interrupt.o(i.TIM1_CC_IRQHandler)
    i.TIM1_TRG_COM_IRQHandler                0x08000bf8   Section        0  chip_uip_interrupt.o(i.TIM1_TRG_COM_IRQHandler)
    i.TIM1_UP_IRQHandler                     0x08000c0c   Section        0  chip_uip_interrupt.o(i.TIM1_UP_IRQHandler)
    i.TIM2_IRQHandler                        0x08000c20   Section        0  chip_uip_interrupt.o(i.TIM2_IRQHandler)
    i.TIM3_IRQHandler                        0x08000c34   Section        0  chip_uip_interrupt.o(i.TIM3_IRQHandler)
    i.TIM4_IRQHandler                        0x08000c48   Section        0  chip_uip_interrupt.o(i.TIM4_IRQHandler)
    i.TIM5_IRQHandler                        0x08000c5c   Section        0  chip_uip_interrupt.o(i.TIM5_IRQHandler)
    i.TIM6_IRQHandler                        0x08000c70   Section        0  chip_uip_interrupt.o(i.TIM6_IRQHandler)
    i.TIM7_IRQHandler                        0x08000c84   Section        0  chip_uip_interrupt.o(i.TIM7_IRQHandler)
    i.TIM8_BRK_IRQHandler                    0x08000c98   Section        0  chip_uip_interrupt.o(i.TIM8_BRK_IRQHandler)
    i.TIM8_CC_IRQHandler                     0x08000cac   Section        0  chip_uip_interrupt.o(i.TIM8_CC_IRQHandler)
    i.TIM8_TRG_COM_IRQHandler                0x08000cc0   Section        0  chip_uip_interrupt.o(i.TIM8_TRG_COM_IRQHandler)
    i.TIM8_UP_IRQHandler                     0x08000cd4   Section        0  chip_uip_interrupt.o(i.TIM8_UP_IRQHandler)
    i.UART4_IRQHandler                       0x08000ce8   Section        0  chip_uip_interrupt.o(i.UART4_IRQHandler)
    i.UART5_IRQHandler                       0x08000cfc   Section        0  chip_uip_interrupt.o(i.UART5_IRQHandler)
    i.UIP_ActivateTask                       0x08000d10   Section        0  uip_kernel_task.o(i.UIP_ActivateTask)
    i.UIP_ClearEvent                         0x08000e14   Section        0  uip_kernel_event.o(i.UIP_ClearEvent)
    i.UIP_GetResource                        0x08000e64   Section        0  uip_kernel_resource.o(i.UIP_GetResource)
    i.UIP_ReceiveMessage                     0x08000f28   Section        0  uip_kernel_message.o(i.UIP_ReceiveMessage)
    i.UIP_ReleaseResource                    0x08001000   Section        0  uip_kernel_resource.o(i.UIP_ReleaseResource)
    i.UIP_SetEvent                           0x0800112c   Section        0  uip_kernel_event.o(i.UIP_SetEvent)
    i.UIP_TerminateTask                      0x08001264   Section        0  uip_kernel_task.o(i.UIP_TerminateTask)
    i.UIP_WaitEvent                          0x08001370   Section        0  uip_kernel_event.o(i.UIP_WaitEvent)
    i.USART1_IRQHandler                      0x080013f8   Section        0  chip_uip_interrupt.o(i.USART1_IRQHandler)
    i.USART2_IRQHandler                      0x0800140c   Section        0  chip_uip_interrupt.o(i.USART2_IRQHandler)
    i.USART3_IRQHandler                      0x08001420   Section        0  chip_uip_interrupt.o(i.USART3_IRQHandler)
    i.USBWakeUp_IRQHandler                   0x08001434   Section        0  chip_uip_interrupt.o(i.USBWakeUp_IRQHandler)
    i.USB_HP_CAN1_TX_IRQHandler              0x08001448   Section        0  chip_uip_interrupt.o(i.USB_HP_CAN1_TX_IRQHandler)
    i.USB_LP_CAN1_RX0_IRQHandler             0x0800145c   Section        0  chip_uip_interrupt.o(i.USB_LP_CAN1_RX0_IRQHandler)
    i.WWDG_IRQHandler                        0x08001470   Section        0  chip_uip_interrupt.o(i.WWDG_IRQHandler)
    i.main                                   0x08001484   Section        0  demo.o(i.main)
    i.uipAlarmHandler                        0x080014a0   Section        0  uip_kernel_time.o(i.uipAlarmHandler)
    i.uipAlarmInitialize                     0x0800151c   Section        0  uip_kernel_common.o(i.uipAlarmInitialize)
    i.uipAppInitialize                       0x08001548   Section        0  demo.o(i.uipAppInitialize)
    i.uipClearPrioGrpAndArrayBit             0x080015a8   Section        0  uip_kernel_scheduler.o(i.uipClearPrioGrpAndArrayBit)
    i.uipGetNextPriority                     0x08001610   Section        0  uip_kernel_scheduler.o(i.uipGetNextPriority)
    i.uipGetNextTask                         0x08001668   Section        0  uip_kernel_scheduler.o(i.uipGetNextTask)
    i.uipInterruptHandlingCallback           0x080016fc   Section        0  chip_uip_interrupt.o(i.uipInterruptHandlingCallback)
    i.uipInterruptServiceEngine              0x08001714   Section        0  uip_kernel_isr_engine.o(i.uipInterruptServiceEngine)
    i.uipKernelInitialize                    0x08001830   Section        0  uip_kernel_common.o(i.uipKernelInitialize)
    i.uipMsgInitialize                       0x08001958   Section        0  uip_kernel_common.o(i.uipMsgInitialize)
    i.uipPreContexSwitch                     0x080019a0   Section        0  uip_kernel_scheduler.o(i.uipPreContexSwitch)
    i.uipResInitialize                       0x080019f4   Section        0  uip_kernel_common.o(i.uipResInitialize)
    i.uipResetPrioGrpAndArrayBit             0x08001a48   Section        0  uip_kernel_scheduler.o(i.uipResetPrioGrpAndArrayBit)
    i.uipSystemCounterHandler                0x08001a98   Section        0  uip_kernel_time.o(i.uipSystemCounterHandler)
    i.uipTaskInitialize                      0x08001b18   Section        0  uip_kernel_common.o(i.uipTaskInitialize)
    i.uipTaskStackInit                       0x08001c24   Section        0  uip_kernel_common.o(i.uipTaskStackInit)
    x$fpl$dfixu                              0x08001c70   Section       90  dfixu.o(x$fpl$dfixu)
    x$fpl$dflt                               0x08001cca   Section       46  dflt_clz.o(x$fpl$dflt)
    x$fpl$dmul                               0x08001cf8   Section      340  dmul.o(x$fpl$dmul)
    x$fpl$dnaninf                            0x08001e4c   Section      156  dnaninf.o(x$fpl$dnaninf)
    x$fpl$dretinf                            0x08001ee8   Section       12  dretinf.o(x$fpl$dretinf)
    .constdata                               0x08001ef4   Section       16  stm32f1xx_hal_rcc.o(.constdata)
    x$fpl$usenofp                            0x08001ef4   Section        0  usenofp.o(x$fpl$usenofp)
    .data                                    0x20000000   Section       20  system_stm32f10x_cl.o(.data)
    .data                                    0x20000014   Section        4  system_stm32f1xx.o(.data)
    .data                                    0x20000018   Section      453  app_cfg.o(.data)
    .data                                    0x200001dd   Section        5  app_int_cfg.o(.data)
    .data                                    0x200001e4   Section       48  uip_kernel_common.o(.data)
    .data                                    0x20000214   Section      290  uip_kernel_scheduler.o(.data)
    .bss                                     0x20000338   Section     6284  app_cfg.o(.bss)
    .bss                                     0x20001bc4   Section       32  app_int_cfg.o(.bss)
    .bss                                     0x20001be4   Section     1304  uip_kernel_common.o(.bss)
    .bss                                     0x200020fc   Section       32  uip_kernel_scheduler.o(.bss)
    .bss                                     0x2000211c   Section       96  libspace.o(.bss)
    HEAP                                     0x20002180   Section      512  startup_stm32f10x_hd.o(HEAP)
    Heap_Mem                                 0x20002180   Data         512  startup_stm32f10x_hd.o(HEAP)
    STACK                                    0x20002380   Section     1024  startup_stm32f10x_hd.o(STACK)
    Stack_Mem                                0x20002380   Data        1024  startup_stm32f10x_hd.o(STACK)
    __initial_sp                             0x20002780   Data           0  startup_stm32f10x_hd.o(STACK)

    Global Symbols

    Symbol Name                              Value     Ov Type        Size  Object(Section)

    BuildAttributes$$THM_ISAv4$P$D$K$B$S$PE$A:L22UL41UL21$X:L11$S22US41US21$IEEE1$IW$USESV6$~STKCKD$USESV7$~SHL$OSPACE$ROPI$EBA8$UX$STANDARDLIB$REQ8$PRES8$EABIv2 0x00000000   Number         0  anon$$obj.o ABSOLUTE
    __ARM_use_no_argv                        0x00000000   Number         0  demo.o ABSOLUTE
    __ARM_exceptions_init                     - Undefined Weak Reference
    __alloca_initialize                       - Undefined Weak Reference
    __arm_preinit_                            - Undefined Weak Reference
    __cpp_initialize__aeabi_                  - Undefined Weak Reference
    __cxa_finalize                            - Undefined Weak Reference
    __rt_locale                               - Undefined Weak Reference
    __sigvec_lookup                           - Undefined Weak Reference
    _atexit_init                              - Undefined Weak Reference
    _call_atexit_fns                          - Undefined Weak Reference
    _clock_init                               - Undefined Weak Reference
    _fp_trap_init                             - Undefined Weak Reference
    _fp_trap_shutdown                         - Undefined Weak Reference
    _get_lc_collate                           - Undefined Weak Reference
    _get_lc_ctype                             - Undefined Weak Reference
    _get_lc_monetary                          - Undefined Weak Reference
    _get_lc_numeric                           - Undefined Weak Reference
    _get_lc_time                              - Undefined Weak Reference
    _getenv_init                              - Undefined Weak Reference
    _handle_redirection                       - Undefined Weak Reference
    _init_alloc                               - Undefined Weak Reference
    _init_user_alloc                          - Undefined Weak Reference
    _initio                                   - Undefined Weak Reference
    _rand_init                                - Undefined Weak Reference
    _signal_finish                            - Undefined Weak Reference
    _signal_init                              - Undefined Weak Reference
    _terminate_alloc                          - Undefined Weak Reference
    _terminate_user_alloc                     - Undefined Weak Reference
    _terminateio                              - Undefined Weak Reference
    __Vectors_Size                           0x00000130   Number         0  startup_stm32f10x_hd.o ABSOLUTE
    __Vectors                                0x08000000   Data           4  startup_stm32f10x_hd.o(RESET)
    __Vectors_End                            0x08000130   Data           0  startup_stm32f10x_hd.o(RESET)
    __main                                   0x08000131   Thumb Code     8  __main.o(!!!main)
    __scatterload                            0x08000139   Thumb Code     0  __scatter.o(!!!scatter)
    __scatterload_rt2                        0x08000139   Thumb Code    44  __scatter.o(!!!scatter)
    __scatterload_rt2_thumb_only             0x08000139   Thumb Code     0  __scatter.o(!!!scatter)
    __scatterload_null                       0x08000147   Thumb Code     0  __scatter.o(!!!scatter)
    __decompress                             0x0800016d   Thumb Code    90  __dczerorl2.o(!!dczerorl2)
    __decompress1                            0x0800016d   Thumb Code     0  __dczerorl2.o(!!dczerorl2)
    __scatterload_zeroinit                   0x080001c9   Thumb Code    28  __scatter_zi.o(!!handler_zi)
    __rt_lib_init                            0x080001e5   Thumb Code     0  libinit.o(.ARM.Collect$$libinit$$00000000)
    __rt_lib_init_alloca_1                   0x080001e7   Thumb Code     0  libinit2.o(.ARM.Collect$$libinit$$0000002E)
    __rt_lib_init_argv_1                     0x080001e7   Thumb Code     0  libinit2.o(.ARM.Collect$$libinit$$0000002C)
    __rt_lib_init_atexit_1                   0x080001e7   Thumb Code     0  libinit2.o(.ARM.Collect$$libinit$$0000001B)
    __rt_lib_init_clock_1                    0x080001e7   Thumb Code     0  libinit2.o(.ARM.Collect$$libinit$$00000021)
    __rt_lib_init_cpp_1                      0x080001e7   Thumb Code     0  libinit2.o(.ARM.Collect$$libinit$$00000032)
    __rt_lib_init_exceptions_1               0x080001e7   Thumb Code     0  libinit2.o(.ARM.Collect$$libinit$$00000030)
    __rt_lib_init_fp_1                       0x080001e7   Thumb Code     0  libinit2.o(.ARM.Collect$$libinit$$00000002)
    __rt_lib_init_fp_trap_1                  0x080001e7   Thumb Code     0  libinit2.o(.ARM.Collect$$libinit$$0000001F)
    __rt_lib_init_getenv_1                   0x080001e7   Thumb Code     0  libinit2.o(.ARM.Collect$$libinit$$00000023)
    __rt_lib_init_heap_1                     0x080001e7   Thumb Code     0  libinit2.o(.ARM.Collect$$libinit$$0000000A)
    __rt_lib_init_lc_collate_1               0x080001e7   Thumb Code     0  libinit2.o(.ARM.Collect$$libinit$$00000011)
    __rt_lib_init_lc_ctype_1                 0x080001e7   Thumb Code     0  libinit2.o(.ARM.Collect$$libinit$$00000013)
    __rt_lib_init_lc_monetary_1              0x080001e7   Thumb Code     0  libinit2.o(.ARM.Collect$$libinit$$00000015)
    __rt_lib_init_lc_numeric_1               0x080001e7   Thumb Code     0  libinit2.o(.ARM.Collect$$libinit$$00000017)
    __rt_lib_init_lc_time_1                  0x080001e7   Thumb Code     0  libinit2.o(.ARM.Collect$$libinit$$00000019)
    __rt_lib_init_preinit_1                  0x080001e7   Thumb Code     0  libinit2.o(.ARM.Collect$$libinit$$00000004)
    __rt_lib_init_rand_1                     0x080001e7   Thumb Code     0  libinit2.o(.ARM.Collect$$libinit$$0000000E)
    __rt_lib_init_return                     0x080001e7   Thumb Code     0  libinit2.o(.ARM.Collect$$libinit$$00000033)
    __rt_lib_init_signal_1                   0x080001e7   Thumb Code     0  libinit2.o(.ARM.Collect$$libinit$$0000001D)
    __rt_lib_init_stdio_1                    0x080001e7   Thumb Code     0  libinit2.o(.ARM.Collect$$libinit$$00000025)
    __rt_lib_init_user_alloc_1               0x080001e7   Thumb Code     0  libinit2.o(.ARM.Collect$$libinit$$0000000C)
    __rt_lib_shutdown                        0x080001e9   Thumb Code     0  libshutdown.o(.ARM.Collect$$libshutdown$$00000000)
    __rt_lib_shutdown_cpp_1                  0x080001eb   Thumb Code     0  libshutdown2.o(.ARM.Collect$$libshutdown$$00000002)
    __rt_lib_shutdown_fp_trap_1              0x080001eb   Thumb Code     0  libshutdown2.o(.ARM.Collect$$libshutdown$$00000007)
    __rt_lib_shutdown_heap_1                 0x080001eb   Thumb Code     0  libshutdown2.o(.ARM.Collect$$libshutdown$$0000000F)
    __rt_lib_shutdown_return                 0x080001eb   Thumb Code     0  libshutdown2.o(.ARM.Collect$$libshutdown$$00000010)
    __rt_lib_shutdown_signal_1               0x080001eb   Thumb Code     0  libshutdown2.o(.ARM.Collect$$libshutdown$$0000000A)
    __rt_lib_shutdown_stdio_1                0x080001eb   Thumb Code     0  libshutdown2.o(.ARM.Collect$$libshutdown$$00000004)
    __rt_lib_shutdown_user_alloc_1           0x080001eb   Thumb Code     0  libshutdown2.o(.ARM.Collect$$libshutdown$$0000000C)
    __rt_entry                               0x080001ed   Thumb Code     0  __rtentry.o(.ARM.Collect$$rtentry$$00000000)
    __rt_entry_presh_1                       0x080001ed   Thumb Code     0  __rtentry2.o(.ARM.Collect$$rtentry$$00000002)
    __rt_entry_sh                            0x080001ed   Thumb Code     0  __rtentry4.o(.ARM.Collect$$rtentry$$00000004)
    __rt_entry_li                            0x080001f3   Thumb Code     0  __rtentry2.o(.ARM.Collect$$rtentry$$0000000A)
    __rt_entry_postsh_1                      0x080001f3   Thumb Code     0  __rtentry2.o(.ARM.Collect$$rtentry$$00000009)
    __rt_entry_main                          0x080001f7   Thumb Code     0  __rtentry2.o(.ARM.Collect$$rtentry$$0000000D)
    __rt_entry_postli_1                      0x080001f7   Thumb Code     0  __rtentry2.o(.ARM.Collect$$rtentry$$0000000C)
    __rt_exit                                0x080001ff   Thumb Code     0  rtexit.o(.ARM.Collect$$rtexit$$00000000)
    __rt_exit_ls                             0x08000201   Thumb Code     0  rtexit2.o(.ARM.Collect$$rtexit$$00000003)
    __rt_exit_prels_1                        0x08000201   Thumb Code     0  rtexit2.o(.ARM.Collect$$rtexit$$00000002)
    __rt_exit_exit                           0x08000205   Thumb Code     0  rtexit2.o(.ARM.Collect$$rtexit$$00000004)
    Reset_Handler                            0x0800020d   Thumb Code     8  startup_stm32f10x_hd.o(.text)
    NMI_Handler                              0x08000215   Thumb Code     2  startup_stm32f10x_hd.o(.text)
    HardFault_Handler                        0x08000217   Thumb Code     2  startup_stm32f10x_hd.o(.text)
    MemManage_Handler                        0x08000219   Thumb Code     2  startup_stm32f10x_hd.o(.text)
    BusFault_Handler                         0x0800021b   Thumb Code     2  startup_stm32f10x_hd.o(.text)
    UsageFault_Handler                       0x0800021d   Thumb Code     2  startup_stm32f10x_hd.o(.text)
    SVC_Handler                              0x0800021f   Thumb Code     2  startup_stm32f10x_hd.o(.text)
    DebugMon_Handler                         0x08000221   Thumb Code     2  startup_stm32f10x_hd.o(.text)
    __user_initial_stackheap                 0x08000225   Thumb Code     0  startup_stm32f10x_hd.o(.text)
    __use_two_region_memory                  0x08000249   Thumb Code     2  heapauxi.o(.text)
    __rt_heap_escrow$2region                 0x0800024b   Thumb Code     2  heapauxi.o(.text)
    __rt_heap_expand$2region                 0x0800024d   Thumb Code     2  heapauxi.o(.text)
    __user_setup_stackheap                   0x0800024f   Thumb Code    74  sys_stackheap_outer.o(.text)
    exit                                     0x08000299   Thumb Code    18  exit.o(.text)
    __user_libspace                          0x080002ad   Thumb Code     8  libspace.o(.text)
    __user_perproc_libspace                  0x080002ad   Thumb Code     0  libspace.o(.text)
    __user_perthread_libspace                0x080002ad   Thumb Code     0  libspace.o(.text)
    _sys_exit                                0x080002b5   Thumb Code     8  sys_exit.o(.text)
    __I$use$semihosting                      0x080002c1   Thumb Code     0  use_no_semi.o(.text)
    __use_no_semihosting_swi                 0x080002c1   Thumb Code     2  use_no_semi.o(.text)
    __semihosting_library_function           0x080002c3   Thumb Code     0  indicate_semi.o(.text)
    uipDisableAllInterrupts                  0x080002c5   Thumb Code     0  uip_kernel_isr_cm.o(CODE)
    uipIntMaskStateRestore                   0x080002cd   Thumb Code     0  uip_kernel_isr_cm.o(CODE)
    uipPendSVHandler                         0x080002d3   Thumb Code     0  uip_kernel_isr_cm.o(CODE)
    ADC1_2_IRQHandler                        0x0800030d   Thumb Code    14  chip_uip_interrupt.o(i.ADC1_2_IRQHandler)
    ADC3_IRQHandler                          0x08000321   Thumb Code    14  chip_uip_interrupt.o(i.ADC3_IRQHandler)
    AppIdleTask                              0x08000335   Thumb Code    46  demo.o(i.AppIdleTask)
    CAN1_RX1_IRQHandler                      0x08000365   Thumb Code    14  chip_uip_interrupt.o(i.CAN1_RX1_IRQHandler)
    CAN1_SCE_IRQHandler                      0x08000379   Thumb Code    14  chip_uip_interrupt.o(i.CAN1_SCE_IRQHandler)
    Chip_UIP_InterruptInit                   0x0800038d   Thumb Code    36  chip_uip_interrupt.o(i.Chip_UIP_InterruptInit)
    Chip_UIP_InterruptRegisterHandler        0x080003bd   Thumb Code    28  chip_uip_interrupt.o(i.Chip_UIP_InterruptRegisterHandler)
    DMA1_Channel1_IRQHandler                 0x080003dd   Thumb Code    14  chip_uip_interrupt.o(i.DMA1_Channel1_IRQHandler)
    DMA1_Channel2_IRQHandler                 0x080003f1   Thumb Code    14  chip_uip_interrupt.o(i.DMA1_Channel2_IRQHandler)
    DMA1_Channel3_IRQHandler                 0x08000405   Thumb Code    14  chip_uip_interrupt.o(i.DMA1_Channel3_IRQHandler)
    DMA1_Channel4_IRQHandler                 0x08000419   Thumb Code    14  chip_uip_interrupt.o(i.DMA1_Channel4_IRQHandler)
    DMA1_Channel5_IRQHandler                 0x0800042d   Thumb Code    14  chip_uip_interrupt.o(i.DMA1_Channel5_IRQHandler)
    DMA1_Channel6_IRQHandler                 0x08000441   Thumb Code    14  chip_uip_interrupt.o(i.DMA1_Channel6_IRQHandler)
    DMA1_Channel7_IRQHandler                 0x08000455   Thumb Code    14  chip_uip_interrupt.o(i.DMA1_Channel7_IRQHandler)
    DMA2_Channel1_IRQHandler                 0x08000469   Thumb Code    14  chip_uip_interrupt.o(i.DMA2_Channel1_IRQHandler)
    DMA2_Channel2_IRQHandler                 0x0800047d   Thumb Code    14  chip_uip_interrupt.o(i.DMA2_Channel2_IRQHandler)
    DMA2_Channel3_IRQHandler                 0x08000491   Thumb Code    14  chip_uip_interrupt.o(i.DMA2_Channel3_IRQHandler)
    DMA2_Channel4_5_IRQHandler               0x080004a5   Thumb Code    14  chip_uip_interrupt.o(i.DMA2_Channel4_5_IRQHandler)
    EXTI0_IRQHandler                         0x080004b9   Thumb Code    14  chip_uip_interrupt.o(i.EXTI0_IRQHandler)
    EXTI15_10_IRQHandler                     0x080004cd   Thumb Code    14  chip_uip_interrupt.o(i.EXTI15_10_IRQHandler)
    EXTI1_IRQHandler                         0x080004e1   Thumb Code    14  chip_uip_interrupt.o(i.EXTI1_IRQHandler)
    EXTI2_IRQHandler                         0x080004f5   Thumb Code    14  chip_uip_interrupt.o(i.EXTI2_IRQHandler)
    EXTI3_IRQHandler                         0x08000509   Thumb Code    14  chip_uip_interrupt.o(i.EXTI3_IRQHandler)
    EXTI4_IRQHandler                         0x0800051d   Thumb Code    14  chip_uip_interrupt.o(i.EXTI4_IRQHandler)
    EXTI9_5_IRQHandler                       0x08000531   Thumb Code    14  chip_uip_interrupt.o(i.EXTI9_5_IRQHandler)
    FLASH_IRQHandler                         0x08000545   Thumb Code    14  chip_uip_interrupt.o(i.FLASH_IRQHandler)
    FSMC_IRQHandler                          0x08000559   Thumb Code    14  chip_uip_interrupt.o(i.FSMC_IRQHandler)
    HAL_NVIC_SetPriority                     0x0800056d   Thumb Code   124  stm32f1xx_hal_cortex.o(i.HAL_NVIC_SetPriority)
    HAL_NVIC_SetPriorityGrouping             0x080005e9   Thumb Code    32  stm32f1xx_hal_cortex.o(i.HAL_NVIC_SetPriorityGrouping)
    HAL_RCC_GetHCLKFreq                      0x08000611   Thumb Code    42  stm32f1xx_hal_rcc.o(i.HAL_RCC_GetHCLKFreq)
    HAL_RCC_GetSysClockFreq                  0x08000649   Thumb Code   146  stm32f1xx_hal_rcc.o(i.HAL_RCC_GetSysClockFreq)
    HAL_SYSTICK_CLKSourceConfig              0x08000701   Thumb Code    40  stm32f1xx_hal_cortex.o(i.HAL_SYSTICK_CLKSourceConfig)
    HAL_SYSTICK_Config                       0x08000729   Thumb Code    52  stm32f1xx_hal_cortex.o(i.HAL_SYSTICK_Config)
    Hardware_Init                            0x0800075d   Thumb Code    54  hardware_init.o(i.Hardware_Init)
    I2C1_ER_IRQHandler                       0x0800079d   Thumb Code    14  chip_uip_interrupt.o(i.I2C1_ER_IRQHandler)
    I2C1_EV_IRQHandler                       0x080007b1   Thumb Code    14  chip_uip_interrupt.o(i.I2C1_EV_IRQHandler)
    I2C2_ER_IRQHandler                       0x080007c5   Thumb Code    14  chip_uip_interrupt.o(i.I2C2_ER_IRQHandler)
    I2C2_EV_IRQHandler                       0x080007d9   Thumb Code    14  chip_uip_interrupt.o(i.I2C2_EV_IRQHandler)
    InterruptHandler                         0x080007ed   Thumb Code    78  chip_uip_interrupt.o(i.InterruptHandler)
    Kernel_System_Tick_Init                  0x08000849   Thumb Code    54  hardware_init.o(i.Kernel_System_Tick_Init)
    PVD_IRQHandler                           0x080008b9   Thumb Code    14  chip_uip_interrupt.o(i.PVD_IRQHandler)
    RCC_IRQHandler                           0x080008cd   Thumb Code    14  chip_uip_interrupt.o(i.RCC_IRQHandler)
    RTCAlarm_IRQHandler                      0x080008e1   Thumb Code    14  chip_uip_interrupt.o(i.RTCAlarm_IRQHandler)
    RTC_IRQHandler                           0x080008f5   Thumb Code    14  chip_uip_interrupt.o(i.RTC_IRQHandler)
    SDIO_IRQHandler                          0x08000909   Thumb Code    14  chip_uip_interrupt.o(i.SDIO_IRQHandler)
    SPI1_IRQHandler                          0x0800091d   Thumb Code    14  chip_uip_interrupt.o(i.SPI1_IRQHandler)
    SPI2_IRQHandler                          0x08000931   Thumb Code    14  chip_uip_interrupt.o(i.SPI2_IRQHandler)
    SPI3_IRQHandler                          0x08000945   Thumb Code    14  chip_uip_interrupt.o(i.SPI3_IRQHandler)
    StartOS                                  0x08000959   Thumb Code    38  uip_kernel_common.o(i.StartOS)
    SystemInit                               0x08000989   Thumb Code   386  system_stm32f10x_cl.o(i.SystemInit)
    TAMPER_IRQHandler                        0x08000b45   Thumb Code    14  chip_uip_interrupt.o(i.TAMPER_IRQHandler)
    TASK_0                                   0x08000b59   Thumb Code    22  demo.o(i.TASK_0)
    TASK_1                                   0x08000b6f   Thumb Code    22  demo.o(i.TASK_1)
    TASK_2                                   0x08000b85   Thumb Code    32  demo.o(i.TASK_2)
    TASK_3                                   0x08000ba5   Thumb Code    26  demo.o(i.TASK_3)
    TASK_4                                   0x08000bbf   Thumb Code    16  demo.o(i.TASK_4)
    TIM1_BRK_IRQHandler                      0x08000bd1   Thumb Code    14  chip_uip_interrupt.o(i.TIM1_BRK_IRQHandler)
    TIM1_CC_IRQHandler                       0x08000be5   Thumb Code    14  chip_uip_interrupt.o(i.TIM1_CC_IRQHandler)
    TIM1_TRG_COM_IRQHandler                  0x08000bf9   Thumb Code    14  chip_uip_interrupt.o(i.TIM1_TRG_COM_IRQHandler)
    TIM1_UP_IRQHandler                       0x08000c0d   Thumb Code    14  chip_uip_interrupt.o(i.TIM1_UP_IRQHandler)
    TIM2_IRQHandler                          0x08000c21   Thumb Code    14  chip_uip_interrupt.o(i.TIM2_IRQHandler)
    TIM3_IRQHandler                          0x08000c35   Thumb Code    14  chip_uip_interrupt.o(i.TIM3_IRQHandler)
    TIM4_IRQHandler                          0x08000c49   Thumb Code    14  chip_uip_interrupt.o(i.TIM4_IRQHandler)
    TIM5_IRQHandler                          0x08000c5d   Thumb Code    14  chip_uip_interrupt.o(i.TIM5_IRQHandler)
    TIM6_IRQHandler                          0x08000c71   Thumb Code    14  chip_uip_interrupt.o(i.TIM6_IRQHandler)
    TIM7_IRQHandler                          0x08000c85   Thumb Code    14  chip_uip_interrupt.o(i.TIM7_IRQHandler)
    TIM8_BRK_IRQHandler                      0x08000c99   Thumb Code    14  chip_uip_interrupt.o(i.TIM8_BRK_IRQHandler)
    TIM8_CC_IRQHandler                       0x08000cad   Thumb Code    14  chip_uip_interrupt.o(i.TIM8_CC_IRQHandler)
    TIM8_TRG_COM_IRQHandler                  0x08000cc1   Thumb Code    14  chip_uip_interrupt.o(i.TIM8_TRG_COM_IRQHandler)
    TIM8_UP_IRQHandler                       0x08000cd5   Thumb Code    14  chip_uip_interrupt.o(i.TIM8_UP_IRQHandler)
    UART4_IRQHandler                         0x08000ce9   Thumb Code    14  chip_uip_interrupt.o(i.UART4_IRQHandler)
    UART5_IRQHandler                         0x08000cfd   Thumb Code    14  chip_uip_interrupt.o(i.UART5_IRQHandler)
    UIP_ActivateTask                         0x08000d11   Thumb Code   220  uip_kernel_task.o(i.UIP_ActivateTask)
    UIP_ClearEvent                           0x08000e15   Thumb Code    68  uip_kernel_event.o(i.UIP_ClearEvent)
    UIP_GetResource                          0x08000e65   Thumb Code   162  uip_kernel_resource.o(i.UIP_GetResource)
    UIP_ReceiveMessage                       0x08000f29   Thumb Code   208  uip_kernel_message.o(i.UIP_ReceiveMessage)
    UIP_ReleaseResource                      0x08001001   Thumb Code   252  uip_kernel_resource.o(i.UIP_ReleaseResource)
    UIP_SetEvent                             0x0800112d   Thumb Code   268  uip_kernel_event.o(i.UIP_SetEvent)
    UIP_TerminateTask                        0x08001265   Thumb Code   228  uip_kernel_task.o(i.UIP_TerminateTask)
    UIP_WaitEvent                            0x08001371   Thumb Code   118  uip_kernel_event.o(i.UIP_WaitEvent)
    USART1_IRQHandler                        0x080013f9   Thumb Code    14  chip_uip_interrupt.o(i.USART1_IRQHandler)
    USART2_IRQHandler                        0x0800140d   Thumb Code    14  chip_uip_interrupt.o(i.USART2_IRQHandler)
    USART3_IRQHandler                        0x08001421   Thumb Code    14  chip_uip_interrupt.o(i.USART3_IRQHandler)
    USBWakeUp_IRQHandler                     0x08001435   Thumb Code    14  chip_uip_interrupt.o(i.USBWakeUp_IRQHandler)
    USB_HP_CAN1_TX_IRQHandler                0x08001449   Thumb Code    14  chip_uip_interrupt.o(i.USB_HP_CAN1_TX_IRQHandler)
    USB_LP_CAN1_RX0_IRQHandler               0x0800145d   Thumb Code    14  chip_uip_interrupt.o(i.USB_LP_CAN1_RX0_IRQHandler)
    WWDG_IRQHandler                          0x08001471   Thumb Code    14  chip_uip_interrupt.o(i.WWDG_IRQHandler)
    main                                     0x08001485   Thumb Code    22  demo.o(i.main)
    uipAlarmHandler                          0x080014a1   Thumb Code   116  uip_kernel_time.o(i.uipAlarmHandler)
    uipAlarmInitialize                       0x0800151d   Thumb Code    34  uip_kernel_common.o(i.uipAlarmInitialize)
    uipAppInitialize                         0x08001549   Thumb Code    60  demo.o(i.uipAppInitialize)
    uipClearPrioGrpAndArrayBit               0x080015a9   Thumb Code    96  uip_kernel_scheduler.o(i.uipClearPrioGrpAndArrayBit)
    uipGetNextPriority                       0x08001611   Thumb Code    74  uip_kernel_scheduler.o(i.uipGetNextPriority)
    uipGetNextTask                           0x08001669   Thumb Code   120  uip_kernel_scheduler.o(i.uipGetNextTask)
    uipInterruptHandlingCallback             0x080016fd   Thumb Code    20  chip_uip_interrupt.o(i.uipInterruptHandlingCallback)
    uipInterruptServiceEngine                0x08001715   Thumb Code   252  uip_kernel_isr_engine.o(i.uipInterruptServiceEngine)
    uipKernelInitialize                      0x08001831   Thumb Code   188  uip_kernel_common.o(i.uipKernelInitialize)
    uipMsgInitialize                         0x08001959   Thumb Code    62  uip_kernel_common.o(i.uipMsgInitialize)
    uipPreContexSwitch                       0x080019a1   Thumb Code    68  uip_kernel_scheduler.o(i.uipPreContexSwitch)
    uipResInitialize                         0x080019f5   Thumb Code    76  uip_kernel_common.o(i.uipResInitialize)
    uipResetPrioGrpAndArrayBit               0x08001a49   Thumb Code    62  uip_kernel_scheduler.o(i.uipResetPrioGrpAndArrayBit)
    uipSystemCounterHandler                  0x08001a99   Thumb Code   116  uip_kernel_time.o(i.uipSystemCounterHandler)
    uipTaskInitialize                        0x08001b19   Thumb Code   236  uip_kernel_common.o(i.uipTaskInitialize)
    uipTaskStackInit                         0x08001c25   Thumb Code    76  uip_kernel_common.o(i.uipTaskStackInit)
    __aeabi_d2uiz                            0x08001c71   Thumb Code     0  dfixu.o(x$fpl$dfixu)
    _dfixu                                   0x08001c71   Thumb Code    90  dfixu.o(x$fpl$dfixu)
    __aeabi_i2d                              0x08001ccb   Thumb Code     0  dflt_clz.o(x$fpl$dflt)
    _dflt                                    0x08001ccb   Thumb Code    46  dflt_clz.o(x$fpl$dflt)
    __aeabi_dmul                             0x08001cf9   Thumb Code     0  dmul.o(x$fpl$dmul)
    _dmul                                    0x08001cf9   Thumb Code   332  dmul.o(x$fpl$dmul)
    __fpl_dnaninf                            0x08001e4d   Thumb Code   156  dnaninf.o(x$fpl$dnaninf)
    __fpl_dretinf                            0x08001ee9   Thumb Code    12  dretinf.o(x$fpl$dretinf)
    __I$use$fp                               0x08001ef4   Number         0  usenofp.o(x$fpl$usenofp)
    aAPBAHBPrescTable                        0x08001ef4   Data          16  stm32f1xx_hal_rcc.o(.constdata)
    Region$$Table$$Base                      0x08001f04   Number         0  anon$$obj.o(Region$$Table)
    Region$$Table$$Limit                     0x08001f24   Number         0  anon$$obj.o(Region$$Table)
    SystemFrequency                          0x20000000   Data           4  system_stm32f10x_cl.o(.data)
    SystemFrequency_SysClk                   0x20000004   Data           4  system_stm32f10x_cl.o(.data)
    SystemFrequency_AHBClk                   0x20000008   Data           4  system_stm32f10x_cl.o(.data)
    SystemFrequency_APB1Clk                  0x2000000c   Data           4  system_stm32f10x_cl.o(.data)
    SystemFrequency_APB2Clk                  0x20000010   Data           4  system_stm32f10x_cl.o(.data)
    SystemCoreClock                          0x20000014   Data           4  system_stm32f1xx.o(.data)
    AppAlarmBase                             0x20000018   Data          24  app_cfg.o(.data)
    AppCounter                               0x20000030   Data          24  app_cfg.o(.data)
    AppAlarm                                 0x20000048   Data          48  app_cfg.o(.data)
    AppAlarmNumber                           0x20000078   Data           1  app_cfg.o(.data)
    AppRes                                   0x2000007c   Data          20  app_cfg.o(.data)
    AppResNumber                             0x20000090   Data           1  app_cfg.o(.data)
    AppMsg                                   0x20000094   Data          36  app_cfg.o(.data)
    AppMsgNumber                             0x200000b8   Data           1  app_cfg.o(.data)
    AppTask                                  0x200000bc   Data         288  app_cfg.o(.data)
    AppTaskNumber                            0x200001dc   Data           1  app_cfg.o(.data)
    ChipSTM32F103UARTIntHandlingData         0x200001dd   Data           4  app_int_cfg.o(.data)
    AppIntNumber                             0x200001e1   Data           1  app_int_cfg.o(.data)
    uipLowPowerMode                          0x200001e4   Data           1  uip_kernel_common.o(.data)
    uipTCBArray                              0x200001e8   Data           4  uip_kernel_common.o(.data)
    uipTaskNumber                            0x200001ec   Data           1  uip_kernel_common.o(.data)
    uipTaskIDNumber                          0x200001ed   Data           1  uip_kernel_common.o(.data)
    uipRCBArray                              0x200001f0   Data           4  uip_kernel_common.o(.data)
    uipResNumber                             0x200001f4   Data           1  uip_kernel_common.o(.data)
    uipACBArray                              0x200001f8   Data           4  uip_kernel_common.o(.data)
    uipAlarmNumber                           0x200001fc   Data           1  uip_kernel_common.o(.data)
    uipAlarmID                               0x200001fd   Data           1  uip_kernel_common.o(.data)
    uipMCBArray                              0x20000200   Data           4  uip_kernel_common.o(.data)
    uipMsgNumber                             0x20000204   Data           1  uip_kernel_common.o(.data)
    uipOSSurport                             0x20000205   Data           1  uip_kernel_common.o(.data)
    uipIdleTaskID                            0x20000206   Data           1  uip_kernel_common.o(.data)
    uipIdleTaskTCBPtr                        0x20000208   Data           4  uip_kernel_common.o(.data)
    uipIntTableID                            0x2000020c   Data           4  uip_kernel_common.o(.data)
    uipInSchedulerLoop                       0x20000210   Data           4  uip_kernel_common.o(.data)
    uipByteValue                             0x20000214   Data         256  uip_kernel_scheduler.o(.data)
    uipSchedulerLock                         0x20000314   Data           1  uip_kernel_scheduler.o(.data)
    uipNestedInterrupts                      0x20000318   Data           4  uip_kernel_scheduler.o(.data)
    uipSystemMode                            0x2000031c   Data           1  uip_kernel_scheduler.o(.data)
    uipPrioGroup                             0x20000320   Data           4  uip_kernel_scheduler.o(.data)
    uipLowHalfByteValue                      0x20000324   Data           1  uip_kernel_scheduler.o(.data)
    uipHighHalfByteValue                     0x20000325   Data           1  uip_kernel_scheduler.o(.data)
    uipCurrentTaskTCBPtr                     0x20000328   Data           4  uip_kernel_scheduler.o(.data)
    uipNextRunningTaskTCBPtr                 0x2000032c   Data           4  uip_kernel_scheduler.o(.data)
    uipSystemStackPtr                        0x20000330   Data           4  uip_kernel_scheduler.o(.data)
    uipCurrentTaskPriority                   0x20000334   Data           1  uip_kernel_scheduler.o(.data)
    uipNextRunningTaskPriority               0x20000335   Data           1  uip_kernel_scheduler.o(.data)
    AppMsgBuf                                0x20000338   Data         140  app_cfg.o(.bss)
    Task_0_Stack                             0x200003c4   Data        1024  app_cfg.o(.bss)
    Task_1_Stack                             0x200007c4   Data        1024  app_cfg.o(.bss)
    Task_2_Stack                             0x20000bc4   Data        1024  app_cfg.o(.bss)
    Task_3_Stack                             0x20000fc4   Data        1024  app_cfg.o(.bss)
    Task_4_Stack                             0x200013c4   Data        1024  app_cfg.o(.bss)
    Task_App_Idle_Stack                      0x200017c4   Data        1024  app_cfg.o(.bss)
    UIP_Exc_VectorTable                      0x20001bc4   Data          32  app_int_cfg.o(.bss)
    uipPriorityToTaskID                      0x20001be4   Data         256  uip_kernel_common.o(.bss)
    uipInitTaskStackPtr                      0x20001ce4   Data        1024  uip_kernel_common.o(.bss)
    uipSystemCounter                         0x200020e4   Data          12  uip_kernel_common.o(.bss)
    uipSystemAlarmBase                       0x200020f0   Data          12  uip_kernel_common.o(.bss)
    uipPrioGrpArray                          0x200020fc   Data          32  uip_kernel_scheduler.o(.bss)
    __libspace_start                         0x2000211c   Data          96  libspace.o(.bss)
    __temporary_stack_top$libspace           0x2000217c   Data           0  libspace.o(.bss)



==============================================================================

Memory Map of the image

  Image Entry point : 0x08000131

  Load Region LR_IROM1 (Base: 0x08000000, Size: 0x0000225c, Max: 0x00040000, ABSOLUTE, COMPRESSED[0x00001fd4])

    Execution Region ER_IROM1 (Exec base: 0x08000000, Load base: 0x08000000, Size: 0x00001f24, Max: 0x00040000, ABSOLUTE)

    Exec Addr    Load Addr    Size         Type   Attr      Idx    E Section Name        Object

    0x08000000   0x08000000   0x00000130   Data   RO            3    RESET               startup_stm32f10x_hd.o
    0x08000130   0x08000130   0x00000008   Code   RO         2532  * !!!main             c_w.l(__main.o)
    0x08000138   0x08000138   0x00000034   Code   RO         2708    !!!scatter          c_w.l(__scatter.o)
    0x0800016c   0x0800016c   0x0000005a   Code   RO         2706    !!dczerorl2         c_w.l(__dczerorl2.o)
    0x080001c6   0x080001c6   0x00000002   PAD
    0x080001c8   0x080001c8   0x0000001c   Code   RO         2710    !!handler_zi        c_w.l(__scatter_zi.o)
    0x080001e4   0x080001e4   0x00000002   Code   RO         2576    .ARM.Collect$$libinit$$00000000  c_w.l(libinit.o)
    0x080001e6   0x080001e6   0x00000000   Code   RO         2583    .ARM.Collect$$libinit$$00000002  c_w.l(libinit2.o)
    0x080001e6   0x080001e6   0x00000000   Code   RO         2585    .ARM.Collect$$libinit$$00000004  c_w.l(libinit2.o)
    0x080001e6   0x080001e6   0x00000000   Code   RO         2588    .ARM.Collect$$libinit$$0000000A  c_w.l(libinit2.o)
    0x080001e6   0x080001e6   0x00000000   Code   RO         2590    .ARM.Collect$$libinit$$0000000C  c_w.l(libinit2.o)
    0x080001e6   0x080001e6   0x00000000   Code   RO         2592    .ARM.Collect$$libinit$$0000000E  c_w.l(libinit2.o)
    0x080001e6   0x080001e6   0x00000000   Code   RO         2595    .ARM.Collect$$libinit$$00000011  c_w.l(libinit2.o)
    0x080001e6   0x080001e6   0x00000000   Code   RO         2597    .ARM.Collect$$libinit$$00000013  c_w.l(libinit2.o)
    0x080001e6   0x080001e6   0x00000000   Code   RO         2599    .ARM.Collect$$libinit$$00000015  c_w.l(libinit2.o)
    0x080001e6   0x080001e6   0x00000000   Code   RO         2601    .ARM.Collect$$libinit$$00000017  c_w.l(libinit2.o)
    0x080001e6   0x080001e6   0x00000000   Code   RO         2603    .ARM.Collect$$libinit$$00000019  c_w.l(libinit2.o)
    0x080001e6   0x080001e6   0x00000000   Code   RO         2605    .ARM.Collect$$libinit$$0000001B  c_w.l(libinit2.o)
    0x080001e6   0x080001e6   0x00000000   Code   RO         2607    .ARM.Collect$$libinit$$0000001D  c_w.l(libinit2.o)
    0x080001e6   0x080001e6   0x00000000   Code   RO         2609    .ARM.Collect$$libinit$$0000001F  c_w.l(libinit2.o)
    0x080001e6   0x080001e6   0x00000000   Code   RO         2611    .ARM.Collect$$libinit$$00000021  c_w.l(libinit2.o)
    0x080001e6   0x080001e6   0x00000000   Code   RO         2613    .ARM.Collect$$libinit$$00000023  c_w.l(libinit2.o)
    0x080001e6   0x080001e6   0x00000000   Code   RO         2615    .ARM.Collect$$libinit$$00000025  c_w.l(libinit2.o)
    0x080001e6   0x080001e6   0x00000000   Code   RO         2619    .ARM.Collect$$libinit$$0000002C  c_w.l(libinit2.o)
    0x080001e6   0x080001e6   0x00000000   Code   RO         2621    .ARM.Collect$$libinit$$0000002E  c_w.l(libinit2.o)
    0x080001e6   0x080001e6   0x00000000   Code   RO         2623    .ARM.Collect$$libinit$$00000030  c_w.l(libinit2.o)
    0x080001e6   0x080001e6   0x00000000   Code   RO         2625    .ARM.Collect$$libinit$$00000032  c_w.l(libinit2.o)
    0x080001e6   0x080001e6   0x00000002   Code   RO         2626    .ARM.Collect$$libinit$$00000033  c_w.l(libinit2.o)
    0x080001e8   0x080001e8   0x00000002   Code   RO         2646    .ARM.Collect$$libshutdown$$00000000  c_w.l(libshutdown.o)
    0x080001ea   0x080001ea   0x00000000   Code   RO         2659    .ARM.Collect$$libshutdown$$00000002  c_w.l(libshutdown2.o)
    0x080001ea   0x080001ea   0x00000000   Code   RO         2661    .ARM.Collect$$libshutdown$$00000004  c_w.l(libshutdown2.o)
    0x080001ea   0x080001ea   0x00000000   Code   RO         2664    .ARM.Collect$$libshutdown$$00000007  c_w.l(libshutdown2.o)
    0x080001ea   0x080001ea   0x00000000   Code   RO         2667    .ARM.Collect$$libshutdown$$0000000A  c_w.l(libshutdown2.o)
    0x080001ea   0x080001ea   0x00000000   Code   RO         2669    .ARM.Collect$$libshutdown$$0000000C  c_w.l(libshutdown2.o)
    0x080001ea   0x080001ea   0x00000000   Code   RO         2672    .ARM.Collect$$libshutdown$$0000000F  c_w.l(libshutdown2.o)
    0x080001ea   0x080001ea   0x00000002   Code   RO         2673    .ARM.Collect$$libshutdown$$00000010  c_w.l(libshutdown2.o)
    0x080001ec   0x080001ec   0x00000000   Code   RO         2546    .ARM.Collect$$rtentry$$00000000  c_w.l(__rtentry.o)
    0x080001ec   0x080001ec   0x00000000   Code   RO         2553    .ARM.Collect$$rtentry$$00000002  c_w.l(__rtentry2.o)
    0x080001ec   0x080001ec   0x00000006   Code   RO         2565    .ARM.Collect$$rtentry$$00000004  c_w.l(__rtentry4.o)
    0x080001f2   0x080001f2   0x00000000   Code   RO         2555    .ARM.Collect$$rtentry$$00000009  c_w.l(__rtentry2.o)
    0x080001f2   0x080001f2   0x00000004   Code   RO         2556    .ARM.Collect$$rtentry$$0000000A  c_w.l(__rtentry2.o)
    0x080001f6   0x080001f6   0x00000000   Code   RO         2558    .ARM.Collect$$rtentry$$0000000C  c_w.l(__rtentry2.o)
    0x080001f6   0x080001f6   0x00000008   Code   RO         2559    .ARM.Collect$$rtentry$$0000000D  c_w.l(__rtentry2.o)
    0x080001fe   0x080001fe   0x00000002   Code   RO         2580    .ARM.Collect$$rtexit$$00000000  c_w.l(rtexit.o)
    0x08000200   0x08000200   0x00000000   Code   RO         2628    .ARM.Collect$$rtexit$$00000002  c_w.l(rtexit2.o)
    0x08000200   0x08000200   0x00000004   Code   RO         2629    .ARM.Collect$$rtexit$$00000003  c_w.l(rtexit2.o)
    0x08000204   0x08000204   0x00000006   Code   RO         2630    .ARM.Collect$$rtexit$$00000004  c_w.l(rtexit2.o)
    0x0800020a   0x0800020a   0x00000002   PAD
    0x0800020c   0x0800020c   0x0000003c   Code   RO            4    .text               startup_stm32f10x_hd.o
    0x08000248   0x08000248   0x00000006   Code   RO         2530    .text               c_w.l(heapauxi.o)
    0x0800024e   0x0800024e   0x0000004a   Code   RO         2567    .text               c_w.l(sys_stackheap_outer.o)
    0x08000298   0x08000298   0x00000012   Code   RO         2569    .text               c_w.l(exit.o)
    0x080002aa   0x080002aa   0x00000002   PAD
    0x080002ac   0x080002ac   0x00000008   Code   RO         2577    .text               c_w.l(libspace.o)
    0x080002b4   0x080002b4   0x0000000c   Code   RO         2638    .text               c_w.l(sys_exit.o)
    0x080002c0   0x080002c0   0x00000002   Code   RO         2649    .text               c_w.l(use_no_semi.o)
    0x080002c2   0x080002c2   0x00000000   Code   RO         2651    .text               c_w.l(indicate_semi.o)
    0x080002c2   0x080002c2   0x00000002   PAD
    0x080002c4   0x080002c4   0x00000048   Code   RO          882    CODE                uip_kernel_isr_cm.o
    0x0800030c   0x0800030c   0x00000014   Code   RO           53    i.ADC1_2_IRQHandler  chip_uip_interrupt.o
    0x08000320   0x08000320   0x00000014   Code   RO           54    i.ADC3_IRQHandler   chip_uip_interrupt.o
    0x08000334   0x08000334   0x0000002e   Code   RO          624    i.AppIdleTask       demo.o
    0x08000362   0x08000362   0x00000002   PAD
    0x08000364   0x08000364   0x00000014   Code   RO           55    i.CAN1_RX1_IRQHandler  chip_uip_interrupt.o
    0x08000378   0x08000378   0x00000014   Code   RO           56    i.CAN1_SCE_IRQHandler  chip_uip_interrupt.o
    0x0800038c   0x0800038c   0x0000002c   Code   RO           57    i.Chip_UIP_InterruptInit  chip_uip_interrupt.o
    0x080003b8   0x080003b8   0x00000004   Code   RO           58    i.Chip_UIP_InterruptNullHandler  chip_uip_interrupt.o
    0x080003bc   0x080003bc   0x00000020   Code   RO           59    i.Chip_UIP_InterruptRegisterHandler  chip_uip_interrupt.o
    0x080003dc   0x080003dc   0x00000014   Code   RO           63    i.DMA1_Channel1_IRQHandler  chip_uip_interrupt.o
    0x080003f0   0x080003f0   0x00000014   Code   RO           64    i.DMA1_Channel2_IRQHandler  chip_uip_interrupt.o
    0x08000404   0x08000404   0x00000014   Code   RO           65    i.DMA1_Channel3_IRQHandler  chip_uip_interrupt.o
    0x08000418   0x08000418   0x00000014   Code   RO           66    i.DMA1_Channel4_IRQHandler  chip_uip_interrupt.o
    0x0800042c   0x0800042c   0x00000014   Code   RO           67    i.DMA1_Channel5_IRQHandler  chip_uip_interrupt.o
    0x08000440   0x08000440   0x00000014   Code   RO           68    i.DMA1_Channel6_IRQHandler  chip_uip_interrupt.o
    0x08000454   0x08000454   0x00000014   Code   RO           69    i.DMA1_Channel7_IRQHandler  chip_uip_interrupt.o
    0x08000468   0x08000468   0x00000014   Code   RO           70    i.DMA2_Channel1_IRQHandler  chip_uip_interrupt.o
    0x0800047c   0x0800047c   0x00000014   Code   RO           71    i.DMA2_Channel2_IRQHandler  chip_uip_interrupt.o
    0x08000490   0x08000490   0x00000014   Code   RO           72    i.DMA2_Channel3_IRQHandler  chip_uip_interrupt.o
    0x080004a4   0x080004a4   0x00000014   Code   RO           73    i.DMA2_Channel4_5_IRQHandler  chip_uip_interrupt.o
    0x080004b8   0x080004b8   0x00000014   Code   RO           74    i.EXTI0_IRQHandler  chip_uip_interrupt.o
    0x080004cc   0x080004cc   0x00000014   Code   RO           75    i.EXTI15_10_IRQHandler  chip_uip_interrupt.o
    0x080004e0   0x080004e0   0x00000014   Code   RO           76    i.EXTI1_IRQHandler  chip_uip_interrupt.o
    0x080004f4   0x080004f4   0x00000014   Code   RO           77    i.EXTI2_IRQHandler  chip_uip_interrupt.o
    0x08000508   0x08000508   0x00000014   Code   RO           78    i.EXTI3_IRQHandler  chip_uip_interrupt.o
    0x0800051c   0x0800051c   0x00000014   Code   RO           79    i.EXTI4_IRQHandler  chip_uip_interrupt.o
    0x08000530   0x08000530   0x00000014   Code   RO           80    i.EXTI9_5_IRQHandler  chip_uip_interrupt.o
    0x08000544   0x08000544   0x00000014   Code   RO           81    i.FLASH_IRQHandler  chip_uip_interrupt.o
    0x08000558   0x08000558   0x00000014   Code   RO           82    i.FSMC_IRQHandler   chip_uip_interrupt.o
    0x0800056c   0x0800056c   0x0000007c   Code   RO         1311    i.HAL_NVIC_SetPriority  stm32f1xx_hal_cortex.o
    0x080005e8   0x080005e8   0x00000028   Code   RO         1312    i.HAL_NVIC_SetPriorityGrouping  stm32f1xx_hal_cortex.o
    0x08000610   0x08000610   0x00000038   Code   RO         2148    i.HAL_RCC_GetHCLKFreq  stm32f1xx_hal_rcc.o
    0x08000648   0x08000648   0x000000b8   Code   RO         2152    i.HAL_RCC_GetSysClockFreq  stm32f1xx_hal_rcc.o
    0x08000700   0x08000700   0x00000028   Code   RO         1314    i.HAL_SYSTICK_CLKSourceConfig  stm32f1xx_hal_cortex.o
    0x08000728   0x08000728   0x00000034   Code   RO         1316    i.HAL_SYSTICK_Config  stm32f1xx_hal_cortex.o
    0x0800075c   0x0800075c   0x00000040   Code   RO          480    i.Hardware_Init     hardware_init.o
    0x0800079c   0x0800079c   0x00000014   Code   RO           83    i.I2C1_ER_IRQHandler  chip_uip_interrupt.o
    0x080007b0   0x080007b0   0x00000014   Code   RO           84    i.I2C1_EV_IRQHandler  chip_uip_interrupt.o
    0x080007c4   0x080007c4   0x00000014   Code   RO           85    i.I2C2_ER_IRQHandler  chip_uip_interrupt.o
    0x080007d8   0x080007d8   0x00000014   Code   RO           86    i.I2C2_EV_IRQHandler  chip_uip_interrupt.o
    0x080007ec   0x080007ec   0x0000005c   Code   RO           87    i.InterruptHandler  chip_uip_interrupt.o
    0x08000848   0x08000848   0x00000036   Code   RO          481    i.Kernel_System_Tick_Init  hardware_init.o
    0x0800087e   0x0800087e   0x00000002   PAD
    0x08000880   0x08000880   0x00000010   Code   RO         1318    i.NVIC_GetPriorityGrouping  stm32f1xx_hal_cortex.o
    0x08000890   0x08000890   0x00000028   Code   RO         1319    i.NVIC_SetPriority  stm32f1xx_hal_cortex.o
    0x080008b8   0x080008b8   0x00000014   Code   RO           88    i.PVD_IRQHandler    chip_uip_interrupt.o
    0x080008cc   0x080008cc   0x00000014   Code   RO           89    i.RCC_IRQHandler    chip_uip_interrupt.o
    0x080008e0   0x080008e0   0x00000014   Code   RO           90    i.RTCAlarm_IRQHandler  chip_uip_interrupt.o
    0x080008f4   0x080008f4   0x00000014   Code   RO           91    i.RTC_IRQHandler    chip_uip_interrupt.o
    0x08000908   0x08000908   0x00000014   Code   RO           92    i.SDIO_IRQHandler   chip_uip_interrupt.o
    0x0800091c   0x0800091c   0x00000014   Code   RO           93    i.SPI1_IRQHandler   chip_uip_interrupt.o
    0x08000930   0x08000930   0x00000014   Code   RO           94    i.SPI2_IRQHandler   chip_uip_interrupt.o
    0x08000944   0x08000944   0x00000014   Code   RO           95    i.SPI3_IRQHandler   chip_uip_interrupt.o
    0x08000958   0x08000958   0x00000030   Code   RO          763    i.StartOS           uip_kernel_common.o
    0x08000988   0x08000988   0x000001bc   Code   RO           12    i.SystemInit        system_stm32f10x_cl.o
    0x08000b44   0x08000b44   0x00000014   Code   RO           96    i.TAMPER_IRQHandler  chip_uip_interrupt.o
    0x08000b58   0x08000b58   0x00000016   Code   RO          625    i.TASK_0            demo.o
    0x08000b6e   0x08000b6e   0x00000016   Code   RO          626    i.TASK_1            demo.o
    0x08000b84   0x08000b84   0x00000020   Code   RO          627    i.TASK_2            demo.o
    0x08000ba4   0x08000ba4   0x0000001a   Code   RO          628    i.TASK_3            demo.o
    0x08000bbe   0x08000bbe   0x00000010   Code   RO          629    i.TASK_4            demo.o
    0x08000bce   0x08000bce   0x00000002   PAD
    0x08000bd0   0x08000bd0   0x00000014   Code   RO           97    i.TIM1_BRK_IRQHandler  chip_uip_interrupt.o
    0x08000be4   0x08000be4   0x00000014   Code   RO           98    i.TIM1_CC_IRQHandler  chip_uip_interrupt.o
    0x08000bf8   0x08000bf8   0x00000014   Code   RO           99    i.TIM1_TRG_COM_IRQHandler  chip_uip_interrupt.o
    0x08000c0c   0x08000c0c   0x00000014   Code   RO          100    i.TIM1_UP_IRQHandler  chip_uip_interrupt.o
    0x08000c20   0x08000c20   0x00000014   Code   RO          101    i.TIM2_IRQHandler   chip_uip_interrupt.o
    0x08000c34   0x08000c34   0x00000014   Code   RO          102    i.TIM3_IRQHandler   chip_uip_interrupt.o
    0x08000c48   0x08000c48   0x00000014   Code   RO          103    i.TIM4_IRQHandler   chip_uip_interrupt.o
    0x08000c5c   0x08000c5c   0x00000014   Code   RO          104    i.TIM5_IRQHandler   chip_uip_interrupt.o
    0x08000c70   0x08000c70   0x00000014   Code   RO          105    i.TIM6_IRQHandler   chip_uip_interrupt.o
    0x08000c84   0x08000c84   0x00000014   Code   RO          106    i.TIM7_IRQHandler   chip_uip_interrupt.o
    0x08000c98   0x08000c98   0x00000014   Code   RO          107    i.TIM8_BRK_IRQHandler  chip_uip_interrupt.o
    0x08000cac   0x08000cac   0x00000014   Code   RO          108    i.TIM8_CC_IRQHandler  chip_uip_interrupt.o
    0x08000cc0   0x08000cc0   0x00000014   Code   RO          109    i.TIM8_TRG_COM_IRQHandler  chip_uip_interrupt.o
    0x08000cd4   0x08000cd4   0x00000014   Code   RO          110    i.TIM8_UP_IRQHandler  chip_uip_interrupt.o
    0x08000ce8   0x08000ce8   0x00000014   Code   RO          111    i.UART4_IRQHandler  chip_uip_interrupt.o
    0x08000cfc   0x08000cfc   0x00000014   Code   RO          112    i.UART5_IRQHandler  chip_uip_interrupt.o
    0x08000d10   0x08000d10   0x00000104   Code   RO         1013    i.UIP_ActivateTask  uip_kernel_task.o
    0x08000e14   0x08000e14   0x00000050   Code   RO          848    i.UIP_ClearEvent    uip_kernel_event.o
    0x08000e64   0x08000e64   0x000000c4   Code   RO          951    i.UIP_GetResource   uip_kernel_resource.o
    0x08000f28   0x08000f28   0x000000d8   Code   RO          900    i.UIP_ReceiveMessage  uip_kernel_message.o
    0x08001000   0x08001000   0x0000012c   Code   RO          952    i.UIP_ReleaseResource  uip_kernel_resource.o
    0x0800112c   0x0800112c   0x00000138   Code   RO          850    i.UIP_SetEvent      uip_kernel_event.o
    0x08001264   0x08001264   0x0000010c   Code   RO         1018    i.UIP_TerminateTask  uip_kernel_task.o
    0x08001370   0x08001370   0x00000088   Code   RO          851    i.UIP_WaitEvent     uip_kernel_event.o
    0x080013f8   0x080013f8   0x00000014   Code   RO          113    i.USART1_IRQHandler  chip_uip_interrupt.o
    0x0800140c   0x0800140c   0x00000014   Code   RO          114    i.USART2_IRQHandler  chip_uip_interrupt.o
    0x08001420   0x08001420   0x00000014   Code   RO          115    i.USART3_IRQHandler  chip_uip_interrupt.o
    0x08001434   0x08001434   0x00000014   Code   RO          116    i.USBWakeUp_IRQHandler  chip_uip_interrupt.o
    0x08001448   0x08001448   0x00000014   Code   RO          117    i.USB_HP_CAN1_TX_IRQHandler  chip_uip_interrupt.o
    0x0800145c   0x0800145c   0x00000014   Code   RO          118    i.USB_LP_CAN1_RX0_IRQHandler  chip_uip_interrupt.o
    0x08001470   0x08001470   0x00000014   Code   RO          119    i.WWDG_IRQHandler   chip_uip_interrupt.o
    0x08001484   0x08001484   0x0000001c   Code   RO          630    i.main              demo.o
    0x080014a0   0x080014a0   0x0000007c   Code   RO         1060    i.uipAlarmHandler   uip_kernel_time.o
    0x0800151c   0x0800151c   0x0000002c   Code   RO          765    i.uipAlarmInitialize  uip_kernel_common.o
    0x08001548   0x08001548   0x00000060   Code   RO          631    i.uipAppInitialize  demo.o
    0x080015a8   0x080015a8   0x00000068   Code   RO          969    i.uipClearPrioGrpAndArrayBit  uip_kernel_scheduler.o
    0x08001610   0x08001610   0x00000058   Code   RO          970    i.uipGetNextPriority  uip_kernel_scheduler.o
    0x08001668   0x08001668   0x00000094   Code   RO          971    i.uipGetNextTask    uip_kernel_scheduler.o
    0x080016fc   0x080016fc   0x00000018   Code   RO          120    i.uipInterruptHandlingCallback  chip_uip_interrupt.o
    0x08001714   0x08001714   0x0000011c   Code   RO          885    i.uipInterruptServiceEngine  uip_kernel_isr_engine.o
    0x08001830   0x08001830   0x00000128   Code   RO          766    i.uipKernelInitialize  uip_kernel_common.o
    0x08001958   0x08001958   0x00000048   Code   RO          768    i.uipMsgInitialize  uip_kernel_common.o
    0x080019a0   0x080019a0   0x00000054   Code   RO          972    i.uipPreContexSwitch  uip_kernel_scheduler.o
    0x080019f4   0x080019f4   0x00000054   Code   RO          770    i.uipResInitialize  uip_kernel_common.o
    0x08001a48   0x08001a48   0x00000050   Code   RO          973    i.uipResetPrioGrpAndArrayBit  uip_kernel_scheduler.o
    0x08001a98   0x08001a98   0x00000080   Code   RO         1063    i.uipSystemCounterHandler  uip_kernel_time.o
    0x08001b18   0x08001b18   0x0000010c   Code   RO          772    i.uipTaskInitialize  uip_kernel_common.o
    0x08001c24   0x08001c24   0x0000004c   Code   RO          773    i.uipTaskStackInit  uip_kernel_common.o
    0x08001c70   0x08001c70   0x0000005a   Code   RO         2534    x$fpl$dfixu         fz_ws.l(dfixu.o)
    0x08001cca   0x08001cca   0x0000002e   Code   RO         2539    x$fpl$dflt          fz_ws.l(dflt_clz.o)
    0x08001cf8   0x08001cf8   0x00000154   Code   RO         2544    x$fpl$dmul          fz_ws.l(dmul.o)
    0x08001e4c   0x08001e4c   0x0000009c   Code   RO         2547    x$fpl$dnaninf       fz_ws.l(dnaninf.o)
    0x08001ee8   0x08001ee8   0x0000000c   Code   RO         2549    x$fpl$dretinf       fz_ws.l(dretinf.o)
    0x08001ef4   0x08001ef4   0x00000000   Code   RO         2551    x$fpl$usenofp       fz_ws.l(usenofp.o)
    0x08001ef4   0x08001ef4   0x00000010   Data   RO         2156    .constdata          stm32f1xx_hal_rcc.o
    0x08001f04   0x08001f04   0x00000020   Data   RO         2704    Region$$Table       anon$$obj.o


    Execution Region RW_IRAM1 (Exec base: 0x20000000, Load base: 0x08001f24, Size: 0x00002780, Max: 0x0000c000, ABSOLUTE, COMPRESSED[0x000000b0])

    Exec Addr    Load Addr    Size         Type   Attr      Idx    E Section Name        Object

    0x20000000   COMPRESSED   0x00000014   Data   RW           13    .data               system_stm32f10x_cl.o
    0x20000014   COMPRESSED   0x00000004   Data   RW          583    .data               system_stm32f1xx.o
    0x20000018   COMPRESSED   0x000001c5   Data   RW          607    .data               app_cfg.o
    0x200001dd   COMPRESSED   0x00000005   Data   RW          744    .data               app_int_cfg.o
    0x200001e2   COMPRESSED   0x00000002   PAD
    0x200001e4   COMPRESSED   0x00000030   Data   RW          775    .data               uip_kernel_common.o
    0x20000214   COMPRESSED   0x00000122   Data   RW          975    .data               uip_kernel_scheduler.o
    0x20000336   COMPRESSED   0x00000002   PAD
    0x20000338        -       0x0000188c   Zero   RW          606    .bss                app_cfg.o
    0x20001bc4        -       0x00000020   Zero   RW          743    .bss                app_int_cfg.o
    0x20001be4        -       0x00000518   Zero   RW          774    .bss                uip_kernel_common.o
    0x200020fc        -       0x00000020   Zero   RW          974    .bss                uip_kernel_scheduler.o
    0x2000211c        -       0x00000060   Zero   RW         2578    .bss                c_w.l(libspace.o)
    0x2000217c   COMPRESSED   0x00000004   PAD
    0x20002180        -       0x00000200   Zero   RW            2    HEAP                startup_stm32f10x_hd.o
    0x20002380        -       0x00000400   Zero   RW            1    STACK               startup_stm32f10x_hd.o


==============================================================================

Image component sizes


      Code (inc. data)   RO Data    RW Data    ZI Data      Debug   Object Name

         0          0          0        453       6284       5062   app_cfg.o
         0          0          0          5         32        836   app_int_cfg.o
      1396        390          0          0          0      45288   chip_uip_interrupt.o
       288         42          0          0          0       3701   demo.o
       118         10          0          0          0     236134   hardware_init.o
        60         26        304          0       1536        780   startup_stm32f10x_hd.o
       312         22          0          0          0      26096   stm32f1xx_hal_cortex.o
       240         52         16          0          0       2228   stm32f1xx_hal_rcc.o
       444         58          0         20          0       5945   system_stm32f10x_cl.o
         0          0          0          4          0        688   system_stm32f1xx.o
       888        178          0         48       1304      13833   uip_kernel_common.o
       528         74          0          0          0      10440   uip_kernel_event.o
        72          4          0          0          0        336   uip_kernel_isr_cm.o
       284         32          0          0          0        772   uip_kernel_isr_engine.o
       216          8          0          0          0       1037   uip_kernel_message.o
       496         82          0          0          0       1884   uip_kernel_resource.o
       504         84          0        290         32      11736   uip_kernel_scheduler.o
       528         80          0          0          0       1643   uip_kernel_task.o
       252         20          0          0          0       1284   uip_kernel_time.o

    ----------------------------------------------------------------------
      6632       1162        352        824       9188     369723   Object Totals
         0          0         32          0          0          0   (incl. Generated)
         6          0          0          4          0          0   (incl. Padding)

    ----------------------------------------------------------------------

      Code (inc. data)   RO Data    RW Data    ZI Data      Debug   Library Member Name

        90          0          0          0          0          0   __dczerorl2.o
         8          0          0          0          0         68   __main.o
         0          0          0          0          0          0   __rtentry.o
        12          0          0          0          0          0   __rtentry2.o
         6          0          0          0          0          0   __rtentry4.o
        52          8          0          0          0          0   __scatter.o
        28          0          0          0          0          0   __scatter_zi.o
        18          0          0          0          0         80   exit.o
         6          0          0          0          0        152   heapauxi.o
         0          0          0          0          0          0   indicate_semi.o
         2          0          0          0          0          0   libinit.o
         2          0          0          0          0          0   libinit2.o
         2          0          0          0          0          0   libshutdown.o
         2          0          0          0          0          0   libshutdown2.o
         8          4          0          0         96         68   libspace.o
         2          0          0          0          0          0   rtexit.o
        10          0          0          0          0          0   rtexit2.o
        12          4          0          0          0         68   sys_exit.o
        74          0          0          0          0         80   sys_stackheap_outer.o
         2          0          0          0          0         68   use_no_semi.o
        90          4          0          0          0         92   dfixu.o
        46          0          0          0          0         68   dflt_clz.o
       340         12          0          0          0        104   dmul.o
       156          4          0          0          0         92   dnaninf.o
        12          0          0          0          0         68   dretinf.o
         0          0          0          0          0          0   usenofp.o

    ----------------------------------------------------------------------
       988         36          0          0        100       1008   Library Totals
         8          0          0          0          4          0   (incl. Padding)

    ----------------------------------------------------------------------

      Code (inc. data)   RO Data    RW Data    ZI Data      Debug   Library Name

       336         16          0          0         96        584   c_w.l
       644         20          0          0          0        424   fz_ws.l

    ----------------------------------------------------------------------
       988         36          0          0        100       1008   Library Totals

    ----------------------------------------------------------------------

==============================================================================


      Code (inc. data)   RO Data    RW Data    ZI Data      Debug   

      7620       1198        352        824       9288     364903   Grand Totals
      7620       1198        352        176       9288     364903   ELF Image Totals (compressed)
      7620       1198        352        176          0          0   ROM Totals

==============================================================================

    Total RO  Size (Code + RO Data)                 7972 (   7.79kB)
    Total RW  Size (RW Data + ZI Data)             10112 (   9.88kB)
    Total ROM Size (Code + RO Data + RW Data)       8148 (   7.96kB)

==============================================================================

